:100000000C94B9190D94EE1A0D94C31A0D94981A04
:100010000D946D1A0D94421A0D94171A0D94EC1943
:100020000D94C1190C94EA190C94EA190C94EA196C
:100030000C94EA190C94EA190C94EA190D942336DD
:100040000C94EA190C94EA190C94EA190C94EA1924
:100050000C94EA190C94EA190C94EA190D943E17C1
:100060000C94EA190D949F1D0D94751D0C94EA19BA
:100070000C94EA190C94EA190C94EA190C94EA19F4
:100080000C94EA190C94EA190C94EA190C94EA19E4
:100090000D943F220D94B5210D94F7210C94256900
:1000A0000C94EA190C94EA190C94EA190C94EA19C4
:1000B0000C94EA190C94EA190C94EA190C94EA19B4
:1000C0000C94EA190C94EA190C94EA190D943F1D4A
:1000D0000D94151D0C94EA190C94EA190C94EA1964
:1000E0000C94EA1907634236B79BD8A71A396856A9
:1000F00018AEBAAB558C1D3CB7CC5763BD6DEDFD4A
:10010000753EF6177231BF000000803F0800000006
:10011000BE922449123EABAAAA2ABECDCCCC4C3EFC
:1001200000000080BEABAAAAAA3E00000000BF00EB
:100130000000803F0000000000084178D3BB4387E7
:10014000D1133D190E3CC3BD4282AD2B3E68EC82FB
:1001500076BED98FE1A93E4C80EFFFBE01C4FF7F80
:100160003F00000000000C94EC5B0D9495110D9481
:1001700007060C94DA230C9435540C94ECDD0C94A3
:100180000C1A0C94A1370C94F2860C941E240C9437
:10019000BE270C94DBAC0C94771A0C9463910D94ED
:1001A00068250C94641A0C94D4B10D94E3130D9447
:1001B000B4130C94FD5E0D945B070C9406240C9410
:1001C00086280D944B150C9415B20D9404070D94CC
:1001D0007B070C9403DA0C941E5F0C940B780C9440
:1001E000E4B20C945C560C94F5A30C94FBBB0D94F8
:1001F000FF120C945C290C940E600C9450DD0C944E
:10020000EF390D94E5110C9427290C94BF4C0C94F4
:10021000201C0C94FFF10C947FB30C94B17B0C94D4
:1002200084AC0C9417BD0C94F5190C94F9190C942A
:10023000F7990C941D290C94149B0C946D890C94C3
:10024000FEBC0C949B6D0C941AE20C94F1BB0C94C4
:10025000DD1C0D9465060C94485E0C9488280C9463
:100260004F5E0D94382B0C9437B70C94F1290C94F5
:100270009C290C94A2200C94A8280D940F040C9493
:1002800044630D9481110C94A0DA0D9421040C9414
:1002900095710C94E3790C94D6ED0C946DC10C948B
:1002A0002BBD0C944FE50C94EC5E0C942D360C9405
:1002B00007DA0C946CE20C949BE20C94D2790C94C7
:1002C0006E260C94D8BC0D942F2C0C94DA7A0D94D5
:1002D000C9140C9406A40C94855F0D941D070C940E
:1002E000D25D0D94702E0D94BB150C943FBD0C94F3
:1002F000F9230C9409880D946A130D94102C0C9416
:1003000021610C947B290C94F4BC0C941A8B0C94F2
:10031000C9900C944E290C941E6E0C94FFE10C9421
:10032000CD600C943E7D0D94CC100D9444110C9432
:10033000CD9A0D949C160C9447DA0C942A360C94A2
:1003400017860C9496400C94D3B20D944D080C94DF
:10035000E0BC0C94719B0D9472110C949F360C941C
:1003600001B20C9499220C943EB70C9470800C94BA
:100370003C540D94592C0D9441080C9427610C9415
:1003800033360D94F12A0C94F7D90C945D1C0C941F
:10039000895F0C945ADA0C9453B70C94BF940D9463
:1003A0008F120C9464A00C9469240D9486120D9401
:1003B00042110C949C370C940A230C9455E50D942F
:1003C000502A0C94C5220C94F5E10C94C1270C948E
:1003D00099290C94A89A0C94EDB20C94B8280C941A
:1003E0002E7B0C94C1910C947EF30C949A5B0C942C
:1003F000F7B10C94E0270C94A0ED0C940F240D940D
:1004000032120C9473DA0C944F5B0D948D160C948D
:1004100079280D94A3110C94B6B10D942F040C946B
:100420000A780C94E2860C94A4270D947F120C9405
:10043000071A0C943DDA0D9413150C94775B0C9409
:1004400023250C949D610C94C0BB0C94FAA30C94CE
:10045000839A0D94B9150D94FC340C9455E20C94C8
:1004600086DA0C9441E20C94E7BB0C94455E0C9444
:100470006D5F0C94C9600C946DB30C94D6270D94E9
:1004800072030C94E3BB0C940C780C9431DD0C9447
:1004900095800C946CC10C94847D0C9481640D94B3
:1004A000002B0C947DAC0C941F610C940F260C94C3
:1004B00028D90C94FA5E0C9453240C943B250C948C
:1004C000E5340C94ADBC0D946D310D94D4140C94A2
:1004D000D5520C9479880C9464F50C94CB5D0D94F2
:1004E00054390C9427640C94EDBB0D94A1340C94F6
:1004F000AF910C9489260C9446860C943BF20C9494
:10050000EABC0D9447080D940D030C94C4BB0C94E5
:10051000BABB0C94205B0C944E650D9437350D944A
:100520001F140C9441290D94912E0C94D85B0C94BB
:10053000ECE10C94A95D0C94CFBB0C94FFBB0D9423
:1005400018130C941F260C943E600C9481910C940B
:100550006D290D944D030C9408E20C946A5F0C9481
:10056000619A0D946E2F0C94148D0C9490370C940A
:100570005FE20D94B1060D946F080C9462880D949F
:1005800004040D94BC2F0C9447660C94E5640C9401
:100590000DBD0C9425610C94185B0C9438F30C94ED
:1005A0001C1A0C943F390D94A7310C944A6B0D948E
:1005B000F72F0D94E92E0C944D250C94D0BC0C947F
:1005C00047280C94FD190C9496AC0C949B910D94B7
:1005D0009A2F0C94D6280C945F840C94FABB0C943C
:1005E0000BB20C9477440D94B3140D9486030C94C1
:1005F000A6860C941C1B0C94A5260D9441040D9406
:10060000E4060C9491880C9482F30C94181A0C94C0
:1006100000710D9471390C94D1290C94F5BB0C9494
:10062000091A0D9499030C94615B0C9475780D94E0
:10063000562E0C946D610D9475080C94B2BC0C94FC
:1006400016890C944E1D0C9483F20D940D140C9489
:10065000C5600C942C1A0C945AB70C94EC190D9498
:100660002C040D94D1340D940A0F0C94FE280D9493
:100670000C300C94DEB10C94C6B10D94B02A0D94DC
:10068000D22E0C943E5F0C94EDB10C94E9280C949E
:10069000C81B0C9489270D9433150C94B8B30C9493
:1006A000AA740C941DDA0C94B3230C94B85D0C94CA
:1006B00060DA0C94C4AC0C94F3D90C943D240C94E3
:1006C000CC220C94A6360C9435BD0C9445B70C94F2
:1006D000845B0C9431ED0C94DFBB0C94C6BC0C9481
:1006E00021BD0C94D5850C94F8EC0C943D9B0C9496
:1006F0003D1A0C9493370C9409780C94DD5E0C949D
:100700005D280C9429F30C94FF240C94A75D0D94A0
:100710007A1C0D949D140C9409EE0C946AE20C94CE
:1007200062240C94CB230C94D9BB0C948A640D9452
:100730001E040D9489120C94A85D0D9412040C945F
:10074000A5AC0C945AF30C94BC230C94FF5D0C9450
:1007500042D90C94CCF20D94341C0D9488130C9453
:10076000A2250C9490E00C9468290C9406200C941B
:1007700061B70C94F2620C94B4DE0C942F1B0C94B1
:10078000362C0D9462350C94CB600D943B060C9482
:1007900043890C941B5A0C94F09A0D944F310C948D
:1007A00004B30D94CC120C94C8BB0C947BC10C9474
:1007B000CEDB0D94D5130D9440250C94A0600C94C1
:1007C0002DE20C943F230C94E2730C9496370C9416
:1007D000FBD90C9443E00D9494070D94D8310C94FC
:1007E0000BDA0C9430B70C9415560C943DA30C9472
:1007F00048240C940AF30C947EC10C9446E50C94A6
:10080000ADDA0C949CDA0C9463D90C9452A30C943A
:10081000345B0C945EDA0D9426140C94A5BC0D94F4
:1008200045110C94D8640C94DC1B0C949DF30C942F
:10083000FFD90C948BE10C94CCBB0D9443110D9417
:1008400055140C9429DD0D9497150C94141A0C94DE
:100850003C230C941F630D9497130C9423610C9408
:10086000D3230C94259B0C9499370C94C7600C945B
:10087000BCBC0C9466F50C9400240C9490F50C947C
:10088000D5BB4E414E494E495459494E46CDCCCC2C
:100890003D0AD7233C17B7D13877CC2B329595E654
:1008A000241FB14F0A000020410000C84200401C34
:1008B0004620BCBE4CCA1B0E5AAEC59D746364690B
:1008C0006E6F70737578585B005374617475732024
:1008D00064656666657265640A002D3E0050756247
:1008E0003A20002D3E005075623A20002D3E005007
:1008F00075623A20000000000000636D6400007320
:100900006574000076616C000064656C00004853FB
:10091000560000524742000066616E00006D6F6431
:1009200065006374726C0068756500007361740023
:100930000074656D700072617700002D3E00507587
:10094000623A20002D3E005075623A200053454E19
:10095000445354415455533A20556E6B6E6F776E25
:1009600020636D64200A0000000000000000000009
:10097000004F4E00000000000000004F46460000FF
:1009800000000000005245535400000000000054D5
:100990004F47474C450000000048414C54000000C0
:1009A000000000584F4E00000000000000584F4665
:1009B00046000000000000494E43524541534500A7
:1009C0000044454352454153450000454E41424C89
:1009D000450000000044495341424C450000005589
:1009E0004E465245455A450000465245455A450037
:1009F0000000004155544F00000000000046414EE9
:100A00005F4F4E4C59000048494748000000000025
:100A1000004D454449554D000000004C4F57000023
:100A20000000000000484541545F434F4F4C0048D0
:100A3000454154000000000000434F4F4C000000AF
:100A400000000044525900000000000000524742DC
:100A500000000000000000485356000000000000A5
:100A600000206661696C65643A004D6F646275735D
:100A7000206F7020004D423A206F6B003D004D42C8
:100A80003A205643230020636D643D003D004D42F3
:100A90003A2056435F6865617423004D423A204E08
:100AA0006F7420737570706F7274656420726567FF
:100AB00020747970650A002056616C3A3078002005
:100AC000543A00205265673A3078004D423A20414E
:100AD0006464723A00444D58000000000000444D28
:100AE00058524742570000444D58524742000000B8
:100AF00050574D0000000000004D42555344494DF1
:100B00000000544845524D4F00000052454C415999
:100B10000000000047524F5550000000005643545B
:100B2000454D500000004D425553564300000041D2
:100B300043484149455200005350494C4544000048
:100B4000004D4F544F520000000050494400000037
:100B50000000004D42555300000000005541525422
:100B6000425244470052454C415950574D00444D64
:100B70005852474257570056454E54530000000004
:100B8000454C455641544F5200434F554E544552E3
:100B9000000048554D0000000000004D45524355EF
:100BA0005259000020002D3E00436F6E766572742E
:100BB000696E6720002D3E0057726F6E672041738B
:100BC0007369676E6D656E742000524742783A20F3
:100BD0000020764C6576656C3A0020436F6E765641
:100BE0003A0020436F6E76533A0020486F743A0003
:100BF000436F6C643A0020436F6E7665727465646F
:100C000020563A00436F6E76657274656420533ADD
:100C1000002D3E0057726F6E672041737369676ED7
:100C20006D656E7420002D3E0057726F6E67204117
:100C3000737369676E6D656E7420004D41503A2084
:100C400076616C206D617070656420746F20200087
:100C50004D41503A2076616C75652061626F766512
:100C600020726967687420626F756E642000206965
:100C7000732062656C6F77206C65667420626F7597
:100C80006E6420004D41503A2076616C75652000FD
:100C90004D41503A20636D64206D61707065642031
:100CA000746F2000000000000000000000004F4EA4
:100CB00000000000000000004F4646000000000059
:100CC000000052455354000000000000544F4747B5
:100CD0004C450000000048414C540000000000005A
:100CE000584F4E00000000000000584F46460000DC
:100CF00000000000494E4352454153450000444521
:100D00004352454153450000454E41424C45000089
:100D1000000044495341424C45000000554E4652A4
:100D200045455A450000465245455A4500000000D9
:100D30004155544F00000000000046414E5F4F4EA9
:100D40004C590000484947480000000000004D454C
:100D50004449554D000000004C4F57000000000072
:100D60000000484541545F434F4F4C0048454154B3
:100D7000000000000000434F4F4C00000000000046
:100D80004452590000000000000052474200000099
:100D900000000000485356000000000000002053EF
:100DA0007566663A002041543A0053746F7070695A
:100DB0006E6720496E70757473002069732000445B
:100DC000656C6574696E6720636F6E662E20524194
:100DD0004D207761733A0053746F70706564006ED4
:100DE0006F7468696E6720746F2073746F7000533E
:100DF000746F7070696E67206368616E6E656C7386
:100E0000202E2E2E0043616E206E6F7420636C6561
:100E1000616E202D206C6F636B656400436F6E669E
:100E20006967206368616E676564206C6F63616CDD
:100E30006C792C20706F7274616C206469736162CC
:100E40006C6564002F636F6E6669672E6A736F6EE0
:100E5000007265626F6F742000436D643A20002F4A
:100E6000636F6D6D616E642F002F72616D2F002FA7
:100E70006974656D2F002F6974656D2F0022687489
:100E800074703A2F2F6C617A79686F6D652E727568
:100E90002F70776122004C6F636174696F6E3A2026
:100EA000687474703A2F2F003F6D61633D002669AE
:100EB000703D0026706F72743D00266E616D653D59
:100EC000002F0020004D5154543A20436F6D706C38
:100ED0006574652E2052656D6F766520746F70693C
:100EE00063200024636F6D6D616E64004D51545436
:100EF0003A20436C65616E55702072657461696E4D
:100F0000656420746F7069632000220022004F75B1
:100F1000744F664D656D6F727921005D20003A5BFC
:100F2000004D5154543A005D00456D7074793A207B
:100F30005B000A003A004D41433A005544502053AB
:100F400079736C6F6720696E697469616C697A6521
:100F5000642E0A005379736C6F6720706172616D43
:100F6000733A002E6C6F63616C005365727669632F
:100F700065207265636F72643A20006D444E5320A1
:100F8000726573706F6E64657220737461727465DC
:100F9000642E004572726F722073657474696E6797
:100FA000207570204D444E5320726573706F6E64CF
:100FB00065722100476F7420495020616464726536
:100FC00073733A00276970205B69705B2C646E73E1
:100FD0005B2C67775B2C7375626E65745D5D5D5D20
:100FE00027202D2073657420737461746963204910
:100FF000500A004661696C656420746F20636F6EEF
:101000006669677572652045746865726E657420DF
:101010007573696E6720444843502E20596F7520C0
:1010200063616E20736574206970206D616E7561F7
:101030006C6C792100204D41534B3A002047573AC0
:101040000020444E533A004C6F6164656420667220
:101050006F6D20666C6173682049503A000A7573A1
:10106000657320444843500A005374617274696E7A
:1010700067206C616E004142434445464748494AF7
:101080004B4C4D4E4F505152535455565758595A38
:101090006162636465666768696A6B6C6D6E6F70C8
:1010A0007172737475767778797A3031323334357A
:1010B000363738392B2F3D00426173696320003A7F
:1010C000004F544120696E697469616C697A656486
:1010D0000A0044454641554C542070617373776F44
:1010E000726420666F72204F5441204150492E2077
:1010F000557365206F746170776420636F6D6D61E7
:101100006E6420746F207365740070617373776F01
:101110007264004D5154543A2074727969796E6743
:10112000206E656E78742062726F6B6572004D512F
:1011300054543A20546F6F206D616E7920636F6E46
:101140006E656374696F6E206572726F72732E20A4
:1011500052657374617274204C414E002074727930
:1011600020616761696E20696E2035207365636F49
:101170006E6473004D5154543A206661696C656425
:101180002C2072633D004D5154543A2041776169DF
:1011900074696E6720666F722072657461696E652E
:1011A0006420746F7069637300636F6E6E6563743F
:1011B00065642061732000202E2E2E00207573653B
:1011C000723A003A000A4D5154543A204174746501
:1011D0006D7074696E6720636F6E6E656374696F9E
:1011E0006E20746F2000646973636F6E6E65637444
:1011F0006564005573696E67204D515454207061C9
:101200007373776F72642066726F6D20636F6E66A2
:101210006967002E6C6F63616C006D444E53206EE5
:10122000616D6520757064617465643A2000446581
:1012300076696365204E616D653A004D5154543AAC
:10124000204174206C656173742064657669636500
:10125000206E616D6520616E642062726F6B6572D5
:10126000204950206D75737420626520636F6E662F
:1012700069677572656400757074696D652C667256
:1012800065656865617000303864656436325F3268
:101290003032362D30312D3039004C696768744852
:1012A00075622000246E616D6500526562696E642E
:1012B00020737563636573732E20495020616464E5
:1012C000726573733A004572726F723A207265628A
:1012D000696E64206661696C0052656E657765644D
:1012E00020737563636573732E20495020616464B5
:1012F000726573733A004572726F723A2072656E4E
:1013000065776564206661696C000A4E6F206C69C0
:101310006E6B00436F6E74696E75652077697468D3
:101320002070726576696F75736C79206C6F61647B
:10133000656420636F6E66696700333073204545CE
:1013400050524F4D206973206E6F742072656C6F20
:10135000616465642E205265626F6F74004D515454
:10136000543A20416363657074696E6720636F6DE2
:101370006D616E64732E2E2E0A004E6F204D5154F7
:101380005420636F6E66696775726564004C6F61A7
:1013900064696E6720636F6E6669672066726F6D41
:1013A00020706F7274616C2064697361626C656433
:1013B0002E2075736520676574204F4E20746F2052
:1013C000656E61626C6500436F6E66696720697364
:1013D0002076616C696400436F6E74696E75652078
:1013E000776974682070726576696F75736C79209F
:1013F0006C6F6164656420636F6E66696700536536
:10140000747570204F5441004D5154543A20736507
:10141000742066697273742062726F6B6572004328
:10142000757272656E74204C414E20636F6E6669F2
:10143000672869702C646E732C67772C7375626EE5
:101440006574293A000A55736520746865736520D0
:10145000636F6D6D616E64733A202768656C7027E9
:10146000202D207468697320746578740A276D6173
:10147000632064653A61643A62653A65663A666516
:101480003A3030272073657420616E642073746F66
:101490007265204D41432D616464726573732069E8
:1014A0006E20454550524F4D0A276970205B697088
:1014B0005B2C646E735B2C67775B2C7375626E6557
:1014C000745D5D5D5D27202D2073657420737461EC
:1014D0007469632049500A277361766527202D209F
:1014E000736176652063757272656E7420636F6ECA
:1014F00066696720696E204E5652414D3B204F4E23
:101500007C4F4646202D20656E61626C652F6469B4
:101510007361626C65206175746F736176650A270B
:1015200067657427205B636F6E666967206164641A
:10153000725D27202D2067657420636F6E66696772
:101540002066726F6D207072652D636F6E666967BD
:10155000757265642055524C20616E642073746FFF
:10156000726520616464722C204F4E7C4F46462089
:101570002D20656E61626C652F64697361626C65B4
:1015800020646F776E6C6F6164206F6E207374617E
:10159000727475700A276C6F616427202D206C6F40
:1015A000616420636F6E6669672066726F6D204E9E
:1015B0005652414D0A2770776427202D20646566B6
:1015C000696E6520616E642073746F7265204D5181
:1015D00054542070617373776F72640A276F74615B
:1015E00070776427202D20646566696E6520616EC2
:1015F000642073746F7265204854545020415049E0
:101600002070617373776F72640A276C6F67205B59
:1016100073657269616C5F6C6F676C6576656C5D34
:10162000205B7564705F6C6F676C6576656C5D27B9
:10163000202D20646566696E65206C6F67206C657F
:1016400076656C2028302E2E37290A276B696C6C42
:1016500027202D2074657374207761746368646F2C
:10166000670A27636C65617227202D20636C6561B2
:101670007220454550524F4D0A2773656172636869
:1016800027202D2073656172636820312D77697280
:1016900065206465760A277265626F6F7427202D56
:1016A000207265626F6F7420636F6E74726F6C6C02
:1016B000657200536F6674207265626F6F74696E35
:1016C000672E2E2E00206E65770020697320003172
:1016D00057543A003157543A205365617263686930
:1016E0006E67206465760052414D3D000A53797360
:1016F0006C6F6720000A312D7769726520000A6DD2
:1017000071747420000A6D6F646275732076320004
:101710000A6D6F6462757320763120282B29000AC8
:10172000696E7075747320000A6974656D732000AA
:101730000A436F6E666967757265643A002F0049E7
:101740006E3A2000496E697469616C697A696E67E6
:1017500020496E70757473003157543A2073657464
:101760007570207265736F6C7574696F6E200031CF
:1017700057543A204453323438322D313030206EB1
:101780006F742070726573656E74003157543A201F
:101790004453323438322D313030204932432072B4
:1017A0006573746F726564003157543A20427573E3
:1017B000207265736574206572726F7200315754C0
:1017C0003A2042757320526573657420646F6E65AC
:1017D000003157543A204453323438322D313030AE
:1017E0002070726573656E742C2072657365740069
:1017F0004572726F7220312D7720696E69740031E5
:1018000057543A204453323438325F3130305F49D4
:1018100032435F544F5F31575F425249444745203E
:10182000696E697400444D584F75742E2046726578
:10183000653A00444D58696E2042756666657220AF
:10184000616C6C6F632065727200496E6974206907
:101850006E2063683A003B003D0050696E3A003BE1
:10186000003D4C4F5700546865726D6F3A004F6EE3
:101870006520776972652052656164790A00467255
:1018800065653A00444D58206F7574207374617219
:101890007465642E204368616E6E656C733A200037
:1018A000444D5820696E20737461727465642E20F3
:1018B0004368616E6E656C733A0042726F6B65725D
:1018C0007320636F6E666967757265643A00417074
:1018D000706C79696E6720636F6E666967004C6F24
:1018E0006164656420455441473A004E6F2073742B
:1018F0006F72656420636F6E666967004C6F616428
:1019000065642066726F6D20454550524F4D006CE6
:101910006F6164206661696C6564004A534F4E20B4
:101920006465746563746564004C6F6164696E67B7
:1019300020436F6E6669672066726F6D2045455063
:10194000524F4D00436F6E666967206175746F7307
:101950006176653A000A5379736C6F67206465623B
:101960007567206C6576656C3A0053657269616CC9
:10197000206465627567206C6576656C3A0053611A
:101980007665640A005365742064796E616D6963DD
:101990002049500A004F54412050617373776F7291
:1019A0006420757064617465640A004E6F2049504C
:1019B0002061647265737300205361766564004C26
:1019C0006F6164696E67204854545020636F6E667F
:1019D0006967206F6E20737461727475703A0000CD
:1019E0000000000000000000004F4E00000000005A
:1019F0000000004F46460000000000000052455322
:101A000054000000000000544F47474C45000000C0
:101A10000048414C54000000000000584F4E0000A8
:101A20000000000000584F4646000000000000493A
:101A30004E435245415345000044454352454153AE
:101A4000450000454E41424C4500000000444953CA
:101A500041424C45000000554E465245455A45000E
:101A600000465245455A45000000004155544F007C
:101A7000000000000046414E5F4F4E4C59000048A8
:101A80004947480000000000004D454449554D00BD
:101A90000000004C4F570000000000000048454186
:101AA000545F434F4F4C0048454154000000000034
:101AB00000434F4F4C00000000000044525900000A
:101AC00000000000005247420000000000000048F3
:101AD000535600000000000000636F756C64206EB8
:101AE0006F742070617273653A2000557064617480
:101AF00065640A00454550524F4D20636C65617224
:101B000065640A004D5154542050617373776F72AD
:101B10006420757064617465640A002B002D0045B3
:101B20005461673A200047657420455441473A2084
:101B300000485454502F312E310025733A2025731C
:101B40000D0A0020485454502F312E310D0A486F91
:101B500073743A2025730D0A4163636570743A20EB
:101B60002A2F2A0D0A436F6E6E656374696F6E3A91
:101B700020636C6F73650D0A0025730020000D0A49
:101B800000474554006661696C656420746F20638A
:101B90006F6E6E6563740A004552524F523A20537D
:101BA00065727665722072657475726E6564200068
:101BB000436F6E666967206E6F74206368616E673D
:101BC00065640A00446F6E652E0A00436F6E666995
:101BD000672070617273696E67206661696C656405
:101BE0000A004765742061626F7274656400676FF4
:101BF0007420436F6E6669670A006874747020729F
:101C00006574636F64652000667265652000436FCC
:101C10006E666967205552493A20687474703A2F8D
:101C20002F002044656661756C7420636F6E666971
:101C3000672073657276657220757365643A20005B
:101C40006C617A79686F6D652E7275000A282D298E
:101C50004352595054000A282D2950554C534520C1
:101C60006F6E2050494E3132000A282D2943414ED3
:101C7000000A282D294D455243555259000A282B58
:101C8000294D554C544956454E54000A282B29508D
:101C9000574D5F52454C4159000A282B294D444E5F
:101CA00053000A282D295541525442524944474570
:101CB000000A282B295359534C4F47000A282B2937
:101CC000504944000A282D294D43503233303137D2
:101CD000000A282D294152544E4554000A282B2928
:101CE0004F5441000A282D29535049204C454400A7
:101CF0000A282B294D4F544F5220435452000A2892
:101D00002D294143204841494552000A282D2943A5
:101D10004353383131202620484443313038300095
:101D20000A282B29524553544152545F4C414E5F6F
:101D30004F4E5F4D5154545F4552524F5253000A1B
:101D4000282D294841524452455345542C2075733F
:101D5000696E6720736F6674000A282B29434F55FC
:101D60004E544552000A282B29444854000A282B77
:101D7000294453323438322D313030000A282B298F
:101D80004F57495245000A282D2949504D4F44428A
:101D90005553000A282B294D4F4442555320307883
:101DA00030362061742053657269616C3220737023
:101DB0006565643A39363030000A282B29414441A0
:101DC0004652554954204C4544000A282B29444D7D
:101DD00058000A282B2957697A6E65743578303097
:101DE000000A282B294672656552616D2070726960
:101DF0006E74696E67000A282B2957415443484482
:101E00004F47006C617A79686F6D652E7275000AB4
:101E1000436F6E666967207365727665723A003249
:101E200030313130334C0020432B2B2076657273D8
:101E3000696F6E3A00303864656436325F32303232
:101E4000362D30312D3039000A4C617A79686F6D4A
:101E5000652E7275204C6967687448756220636FDF
:101E60006E74726F6C6C65722000204F46460020C5
:101E70004F4E0020425950415353005361766564E0
:101E800020746F20454550524F4D00536176696E66
:101E90006720636F6E66696720746F2045455052F6
:101EA0004F4D2E2E00556E6B6E6F776E20737566DC
:101EB0006669782000556E6B6E6F776E20636D6477
:101EC0002000436F756E7465723A2000444D582DA2
:101ED0004F757420496E69743A2000444D582D4F57
:101EE00075742073746F703A200041737369676E64
:101EF00065643A00444D58206374726C3A2000695E
:101F00003136000169333200027531360003753312
:101F1000320004693868000569386C000675386855
:101F2000000775386C000878313000093130300016
:101F30000A44656661756C742073657269616C2012
:101F40006D6F6465204E38312075736564003845C7
:101F500031002600384E31000600384532002E0090
:101F6000384E32000E00384F31003600384F320004
:101F70003E00374531002400374532002C00374FF2
:101F800031003400374F32003C00374E310004003E
:101F9000374E32000C002061646465642062792051
:101FA0006E756D20004D4255533A200041646469BE
:101FB0006E67207265677320776974682061637447
:101FC000696F6E733A00416464696E67207265667A
:101FD000657272656420726567733A004164646972
:101FE0006E672070726566657463682072656773DA
:101FF0003A004D4255533A204D6F64627573207418
:10200000656D706C617465206E6F7420666F756E9F
:10201000643A20004D4255533A20496E76616C690E
:10202000642074656D706C6174652E002C002C004A
:102030002C002C004D4255533A20636F6E66696741
:10204000206661696C65643A004D4255533A2063DD
:102050006F6E666967206572726F72004D425553EC
:102060003A20636F6E666967206C6F6164656420F7
:10207000004D4255533A204F7574206F66206D65B0
:102080006D6F7279004D4255533A20506F6C6C69F8
:102090006E67206572726F7220004D4255533A2070
:1020A0004E6F7420737570706F7274656420726502
:1020B0006720747970650A004D425553443A2049AF
:1020C000676E6F726564202D20657175616C207775
:1020D000697468207365747465642076616C004D62
:1020E000425553443A204D61707065643A004D4248
:1020F0005553443A204E65737465644D6170706544
:10210000643A004C6173744B6E6F776E2076616C2D
:1021100075653A2000536561726368696E67207265
:1021200065673A2000206F7574206F662072616EBB
:102130006765206275666665722C206665746368E3
:10214000696E6700646566207265672320004D42F2
:102150005553443A20536561726368696E67207213
:10216000656723003A002066726F6D207479706590
:1021700020004D425553443A2020676F74200020C0
:1021800076616C3A0020004D425553207265733AD7
:1021900020002076616C206E6F74206368616E672A
:1021A00065642E20436F6E74696E7565004D4255EF
:1021B000533A003A20657175616C207461726765ED
:1021C00072742E003D004D4255533A002076616CEA
:1021D000206368616E6765642E004D4255533A0076
:1021E000204E6F773A00204C6173743A0020230030
:1021F0002070726566657463682000205265672FE1
:10220000636F696C206D75737420626520696E74EC
:102210000020696E7465726E616C2073656E642057
:102220006572726F72202D206E6F207265672F634A
:102230006F696C0020696E7465726E616C207365E5
:102240006E64206572726F72202D206E6F2074652F
:102250006D706C6174650020696E7465726E616C7E
:102260002073656E64206572726F72202D206E6F10
:102270002073746F7265004D425553443A20656E69
:1022800064506F6C6C20004D425553443A20506F9F
:102290006C6C2000206E6F7420666F756E64004D4C
:1022A0004255533A2020706172616D2000207365A1
:1022B0006E64696E672063616E63656C6C65640053
:1022C0004D4255533A2020706172616D20004D429D
:1022D00055533A2020002073656E64206572726F3A
:1022E000722E20004D4255533A2020004164642054
:1022F00040563A20002056616C3A20004D4255531A
:10230000443A207375666669783A00206F722073CC
:10231000756666697820004D4255533A204E6F200D
:1023200074656D706C61746520666F7220004D6F0E
:10233000746F723A2074696D656F757400556E6BB9
:102340006E6F776E20636D64004D6F746F723A200C
:10235000466F7263656420657865637574696F6E36
:102360000056454E543A20636F6E66696720666179
:10237000696C65640056454E543A20696E69740074
:1023800056454E543A2050494420503D0056454E43
:10239000543A2044652D496E69740056454E543AAE
:1023A000204368616E2062616C616E63653D002050
:1023B0007365742052455645525345206D6F6465D0
:1023C0000056454E543A205049443A200020736547
:1023D0007420444952454354206D6F64650056454E
:1023E0004E543A205049443A2000207365742052DC
:1023F000455645525345206D6F64650056454E5411
:102400003A2050415353205049443A2000207365EC
:102410007420444952454354206D6F64650056450D
:102420004E543A2050415353205049443A20002002
:102430006F75743A00207365743A0020696E3A0033
:1024400056454E543A2000204F75743A002052658C
:10245000713A0056454E543A2000206D33002066F4
:10246000726F6D2000204D6178207265713A0020F6
:1024700066616E253A002061637469766520563A7C
:102480000056454E543A20546F74616C20563A0001
:1024900056454E543A2076616C75652000414320C4
:1024A00061697220726F6F6D74656D703A200056AD
:1024B000454E543A004143206D6F64653A20005602
:1024C000454E543A004143206169722074656D7035
:1024D0003A200056454E543A005049443A20616C27
:1024E000726561647920696E697469616C697A6585
:1024F00064005049443A20496E76616C69642070EA
:102500006172616D2061727261792E002C002C0065
:102510002C002C005049443A20636F6E6669672096
:102520006661696C65643A005049443A20636F6E95
:10253000666967206572726F72005049443A206381
:102540006F6E666967206C6F616465642000504936
:10255000443A204F7574206F66206D656D6F7279F7
:10256000005049443A2044652D496E69742000208A
:102570003C414C4D3E0020443A0020493A00205056
:102580003A0020696E3A00207365743A005049445D
:102590003A20005049443A20496E76616C696420C3
:1025A000706172616D2061727261792E0053657481
:1025B000206F757420746F20002050494420616C96
:1025C00061726D2E20002050494420616C61726D53
:1025D0003A20636C6F736564005049443A20556E2D
:1025E0006B6E6F776E207375666669782000504950
:1025F000443A20556E6B6E6F776E20636D642000D9
:1026000020536574706F696E743A005049443A20E3
:102610000020496E7075742076616C75653A0050C3
:1026200049443A200020696E697400200050574DDB
:102630002D4F75742023002073746F70002000509C
:10264000574D2D4F75742023003D0050696E3A00A0
:1026500020696E69740070696E230072656C61791F
:102660004374723A20002073746F700052656C617D
:10267000792D4F757420230072656C6179437472F3
:102680003A200069646C65006F6666006865617475
:10269000696E670066616E00647279696E670063D7
:1026A0006F6F6C696E6700616374696F6E0020699B
:1026B0007320004F7574200072656C6179437472E9
:1026C0003A2000556E6B6E6F776E20737566666983
:1026D00078200072656C61794374723A2000556EFF
:1026E0006B6E6F776E20636D64200072656C61792C
:1026F0004374723A2000616374696F6E0072656C96
:1027000061794374723A20005B305D3A2000202DDD
:10271000202D202D20EFBBBF003E003E31202D207C
:10272000005B305D3A2000202D202D202D20EFBBB6
:10273000BF003E003E31202D20005379736C6F673F
:1027400020726573756D6564005379736C6F6720D3
:10275000726573756D6564005379736C6F67207370
:10276000757370656E646564000000000000636D41
:10277000640000736574000076616C000064656C31
:1027800000004853560000524742000066616E0048
:10279000006D6F6465006374726C0068756500009D
:1027A000736174000074656D7000726177000020C1
:1027B000002E00696E00735F6F7574006D79686F2D
:1027C0006D65004354524C2F657865633A204F7510
:1027D000744F664D656D6F72793A2000202D3E2052
:1027E000004D5154543A2000202D3E2000456D6983
:1027F000743A203C00202D3E20004974656D436DE5
:10280000643A2000202D3E20004974656D3A200076
:102810003157543A20427573207265736574206590
:1028200072726F72003157543A20427573205265AC
:1028300073657420646F6E65003157543A204453B9
:10284000323438322070726573656E742C20726574
:10285000736574004932432052657365740000004B
:102860002100240027002A002D0030003300010140
:102870000000040107010A010000220025002800D1
:102880002B002E0031003400020100000501080178
:102890000B010505050507050808080802020202E4
:1028A0000A0A0808040404040101010101010101EC
:1028B0000303030303030303040707070C0C0C0CB7
:1028C0000C0C0C0C020202020606060606060606A0
:1028D0000B0B0B0B0B0B0B0B01021020200808102D
:1028E0002040102040800201020108040201010280
:1028F0000408102040808040201008040201800459
:1029000002018040201008040201080402010102B3
:1029100004081020408001020408102040800000BC
:102920000A0B02090C0D0E08070304010000000049
:102930000000000000000000000000000000000097
:102940000000000000000000000012111000000054
:102950000000000000000000000000000000000077
:10296000000000004D4255533A204164642040531A
:102970003A20006F637465742F73747265616D0023
:102980006170706C69636174696F6E2F6A736F6ECA
:1029900000746578742F706C61696E00436F6E749B
:1029A000656E742D547970653A2000436F6E6E65C4
:1029B0006374696F6E3A20636C6F73650041636383
:1029C0006573732D436F6E74726F6C2D416C6C6FF9
:1029D000772D4F726967696E3A202A00556E6B6ECB
:1029E0006F776E004E6F74204D6F64696669656421
:1029F000004F4B004D6F766564207065726D616E9F
:102A0000656E746C7900496E7465726E616C2053EA
:102A10006572766572204572726F72005061796CD2
:102A20006F616420546F6F204C61726765004E6F58
:102A30007420666F756E64005757572D4175746822
:102A4000656E7469636174653A20426173696320DD
:102A50007265616C6D3D22416363657373207265BD
:102A600073747269637465642200556E617574686D
:102A70006F72697A6564005061796C6F616420736C
:102A8000697A652077726F6E6700426164207265B3
:102A9000717565737400485454502F312E312000E5
:102AA000200057726F6E67207061796C6164004D11
:102AB0005154543A204354524C2F7478743A204F56
:102AC00075744F664D656D6F72793A2000202D3E0A
:102AD0002041543A004368616E20747970653A0071
:102AE0004E6F2073746F7265642076616C756573C8
:102AF000202D2064656661756C743A200053617600
:102B0000656420455441473A00536574204554415B
:102B1000473A2000556E6B6E6F776E207375666650
:102B200069782000556E6B6E6F776E20636D642040
:102B300000636C724374723A2000444D58494E3A17
:102B400000454F46003D00494E3A002500C2B043C3
:102B500020483D0020444854323220747970652E5C
:102B600020543D00494E3A00204E6F20656D697437
:102B70002064617461210020436F756E746572205A
:102B8000747970652E2076616C3D00494E3A0020C4
:102B9000436F756E74657220747970652E20494E8E
:102BA000434F525245435420496E7465727275709A
:102BB00074206E756D626572212121004952513A6F
:102BC00000416374697661746520696E2000416319
:102BD00074697661746520696E20002D3E002000C6
:102BE00023002D3E00200050656E6465643A20236A
:102BF000002D3E00456D69743A002D3E00456D691B
:102C0000743A002D3E00456D69743A002D3E004532
:102C10006D69743A003D004C454741435920494E87
:102C20003A0020666F7220286D73293A004354528F
:102C30004C3A205363686564756C6520636D64204D
:102C400000206D730020666F7220004354524C3A8E
:102C50002041726D656420002044697361726D6566
:102C600064004354524C3A20002074696D653A0068
:102C70004354524C3A205265733A004354524C3AF2
:102C8000206D6F6D656E74617279206576656E7406
:102C9000002054533A0020543A00544845524D3ACB
:102CA00000436C65616E696E6720616C61726D20B6
:102CB000003D0050696E3A004354524C3A20436F35
:102CC0006D6D616E6420626C6F636B656420627908
:102CD00020647269766572004354524C3A204F4E1C
:102CE0003A416C7265616479204163746976650A62
:102CF000004354524C3A2048414C543A416C72655E
:102D000061647920496E6163746976650A00435491
:102D1000524C3A20584F4E3A2044697361626C65B8
:102D2000640A004354524C3A20584F4E3A416C7258
:102D300065616479204163746976650A0043545281
:102D40004C3A20584F464620736B69707065642E6C
:102D5000205072657620636D643A004354524C3AB9
:102D6000205475726E6564206F66662066726F6DA2
:102D70003A004354524C3A20526573746F72656442
:102D80002066726F6D3A004354524C3A2049676E88
:102D90006F7265642C206368616E6E656C20636D74
:102DA000643D0020457865633A004354524C3A2014
:102DB0004163746976653A004354524C3A20484165
:102DC0004C543A416C726561647920496E61637458
:102DD0006976650A004354524C3A20584F4E3A20C7
:102DE00044697361626C65640A004354524C3A2032
:102DF000584F4E3A416C7265616479204163746941
:102E000076650A004354524C3A20584F4646207388
:102E10006B69707065642E205072657620636D64F6
:102E20003A004354524C3A205475726E6564206FD8
:102E300066662066726F6D3A004354524C3A2052D7
:102E40006573746F7265642066726F6D3A004469D1
:102E50007361726D696E67206E6F7420617574683E
:102E60006F72697A6564004354524C3A20636F6D07
:102E70006D616E64206A75737420666F7220004302
:102E800054524C3A204E6F7420656E6F75676820FF
:102E90006D656D6F727920666F722067726F7570E5
:102EA000206F7065726174696F6E00496E76616C37
:102EB00069642061726700496E76616C69642061A3
:102EC000726700496E76616C6964206172670043C5
:102ED00054524C3A20556E6B6E6F776E2073756648
:102EE00066697800536B697070696E6720736368F8
:102EF0006564756C65642067726F757020657865B0
:102F000063004354524C3A206368616E6E656C20D6
:102F100066726F7A656E004354524C3A2063686162
:102F20006E6E656C2066726F7A656E00536B6970A9
:102F300070656420686F6D696520737475666600DE
:102F40002000205375623D00204974656D3D0043AB
:102F500054524C3A2052414D3D004354524C3A2079
:102F60004F75744F664D656D6F72793A2000282D4C
:102F7000292000282B2920002076616C75652069A6
:102F800073200020756E6B6E6F776E0A005D3D00DA
:102F90005B0020696E76616C6964002000414354D7
:102FA0004956453A00206F6B003A00206661696C13
:102FB0006564003A005265747279696E6720564301
:102FC00054454D5020434D440A005265747279694E
:102FD0006E6720564320434D440A0052657472794F
:102FE000696E67206D6F6462757320434D440A00FB
:102FF0005265747279696E6720434D440A002065FA
:1030000072726F723D004D423A20706F6C6C696E47
:103010006720002056616C3A20004D423A20004D56
:10302000423A204E6F7420737570706F72746564CD
:103030002072656720747970650A004D423A2070ED
:103040006F6C6C696E672064696D6D657220004DF0
:10305000423A20496C6C6567616C20617267756DDE
:10306000656E74730A00206572726F723D004D4286
:103070003A20706F6C6C696E6720504920002D00FB
:103080004D423A2050492056616C203A004D423A58
:1030900020706F6C6C696E6720504920004D423A79
:1030A00020706F6C6C696E6720464D206661756C90
:1030B000742000206572726F723D004D423A20709C
:1030C0006F6C6C696E6720002D004D423A20464DB2
:1030D0002056616C203A004D423A20706F6C6C694A
:1030E0006E6720464D20004354524C2F706F6C6C1D
:1030F0003A204F75744F664D656D6F72793A2000B6
:10310000207365632072656D61696E696E6700008A
:103110005EBCE2613FDD83C29C7E20A3FD1F419D1A
:10312000C3217FFCA2401E5F01E3BD3E6082DC2321
:103130007D9FC1421CFEA0E1BF5D0380DE3C62BEFC
:10314000E0025CDF81633D7C22C09E1D43A1FF46FF
:1031500018FAA427799BC584DA3866E5BB5907DBE2
:10316000856739BAE406581947A5FB7826C49A65DD
:103170003BD987045AB8E6A7F91B45C6987A24F8C4
:10318000A6441A99C7257B3A6486D85B05E7B98CB3
:10319000D2306EEDB3510F4E10F2AC2F7193CD11B2
:1031A0004FADF3702ECC92D38D6F31B2EC0E50AF89
:1031B000F1134DCE90722C6D33D18F0C52B0EE3294
:1031C0006C8ED0530DEFB1F0AE4C1291CF2D73CA6F
:1031D000947628ABF517490856B4EA6937D58B576A
:1031E00009EBB536688AD495CB2977F4AA4816E955
:1031F000B7550B88D6346A2B7597C94A14F6A8744C
:103200002AC896154BA9F7B6E80A54D7896B353EFC
:103210003E2000496E76616C696420636F6D6D615C
:103220006E6400000020002300260029002C002FDF
:10323000003200000100000301060109013E3E3E8C
:10324000004E6F204D414320636F6E666967757253
:1032500065643A20736574206669726D7761726582
:103260002773204D41430A00454550524F4D20736E
:1032700069676E6174757265206F6B00496E697461
:1032800069616C697A696E6720454550524F4D2ED1
:10329000002072656164206572726F7220666F72C1
:1032A00020003E2000203C003157543A0031575452
:1032B0003A206E6F7420696E6974003157543A2059
:1032C000425553592074696D656F757400315754B8
:1032D0003A204453323438325F4552524F525F43A2
:1032E0004F4E464947003157543A20312D77697285
:1032F000652073686F72746564007265616479003B
:1033000024737461746500757074696D650066720C
:10331000656568656170002473746174730020458D
:103320007870697265640A00202D74617267657433
:10333000207A6F6E652D0020416C61726D2045789A
:1033400070697265640A0020636D643A00204375F9
:10335000723A00205365743A002054696D65723AE0
:1033600000204C6F636B733A0052414D3D000903DE
:103370006F0211241FBECFEFD1E2DEBFCDBF00E050
:103380000CBF19E0A0E0B2E0ECE7FCEA02E00BBF02
:1033900002C007900D92A83AB107D9F721E1A8EA37
:1033A000B9E001C01D92AD3BB207E1F719E1C8EBEE
:1033B000D9E100E006C021970109802FFE010F949A
:1033C0000E4EC73BD10780E00807A9F70F94FC3CDD
:1033D0000D942C560C9400008FE090E09093FF1019
:1033E0008093FE1088EC90E00895FC018481958123
:1033F0000895FC01768765870895DC01ED91FC91C5
:1034000002A0F3A1E02D199591E089270895862F58
:10341000089581E08627089521E0FC0184858830A5
:1034200008F020E0822F0895FC0184859585089599
:10343000FC0184899589089526E135E0FC013183FA
:103440002083FB014089518962897389FC01428391
:103450005383648375830895DC01ED91FC91048CA2
:10346000F58DE02D19946BE17BE1811102C06DE1D6
:103470007BE188E89EE00D94C91C63EB76E188E867
:103480009EE00F94C91CF0E0E0E0199584EF91E014
:1034900008958091230A8823B1F0E091240AF091E5
:1034A000250A309731F0868197819093220A809384
:1034B000210A68E074E188E89EE00F94C91C88E85E
:1034C0009EE00D94CA1B0895892B71F0FB01828147
:1034D00093810E94BFAD64E07BE188E89EE00F9499
:1034E000C91C88EC90E0089590E080E0F2CF0F9343
:1034F0001F93CF93DF93EB0102970CF483C00A81F3
:103500001B8169EE79E1C8010F942646892B51F49D
:1035100081E00E944DB088EC90E0DF91CF911F9147
:103520000F91089563EF79E1C8010F942646892B26
:1035300011F480E0EECF6FEB79E188E89EE00F9424
:10354000C91C0E94AFAF672F6095617070E088E87A
:103550009EE00E9457AC88E89EE00F94CA1B8091C1
:10356000640E9091650E892BE9F10A811B810E94FE
:1035700050AD8823B9F1F80101900020E9F73197A7
:10358000E01BF10BB09770F582E70E943BAD809194
:10359000640E9091650EDC01ED91FC910088F1893B
:1035A000E02D60E270E01995B8018091640E909171
:1035B000650E0F94721C8091640E9091650EDC0173
:1035C000ED91FC910190F081E02D60E019958091E2
:1035D000640E9091650EDC01ED91FC910488F589F3
:1035E000E02D19956A817B8188E89EE00F94721C1A
:1035F00068EB79E188E89EE00F94C91C88E89EE0BA
:103600000F94CA1B8091FE109091FF1002973CF01E
:1036100080EF9FEF9093FF108093FE107CCF6BEABA
:1036200079E182E99EE00F94C91C82E99EE00F9443
:10363000CA1B84EF91E071CF892B71F0FB0182816D
:1036400093810E940DAE65E979E188E89EE00F94D0
:10365000C91C88EC90E0089590E080E0F2CFEF92F2
:10366000FF920F931F93CF93DF93CDB7DEB72C97C5
:103670000FB6F894DEBF0FBECDBF8C017B0186E193
:1036800095E09A8389831B821C821D821E82988703
:103690008F8319861A861B861C8605301105ECF06F
:1036A000BE01695F7F4FF701808591850E94DD75BE
:1036B000892B99F0CE0107960E94B0AEBE01695FDA
:1036C0007F4FF701868197810E94DD75892B61F01C
:1036D000CE0107960E945AAF0EC0CE0101960E94FD
:1036E000B0AE0430110554F7CE0101960E945AAFD6
:1036F00003301105A4F1BE01695F7F4FF70184819A
:1037000095810E94DD75892B51F1CE0107960E94AB
:1037100005AFBE01695F7F4FF701828193810E94EF
:10372000DD75892B19F1CE0107960E945BAE6EE71D
:1037300079E188E89EE00F94C91C80E00E9444B0C3
:1037400088EC90E02C960FB6F894DEBF0FBECDBF8C
:10375000DF91CF911F910F91FF90EF900895CE01CF
:1037600001960E9405AF023011059CF6CE0101962C
:103770000E945BAE01301105D1F6CE0101960E9488
:103780005BAE65E879E188E89EE00F94C91CCFCF75
:10379000CF93C1E068EE73E080E090E00E9479BED4
:1037A0006C2F88E89EE00E9450ACCF5FC43191F747
:1037B00084EF91E0CF9108950F931F93CF93DF9300
:1037C0008C01EB010297C4F08A819B810F94D8454C
:1037D00080931E0299270E9457B00230110549F0CC
:1037E0008C819D810F94D84580931D0299270E945A
:1037F00061B0C8ECD0E002C0C0E9D1E06AE679E18E
:1038000088E89EE00F94C91C60911E0288E89EE043
:103810000E9450AC65E579E188E89EE00F94C91CF0
:1038200060911D0288E89EE00E9450AC88E89EE00E
:103830000F94CA1BCE01DF91CF911F910F91089574
:10384000CF93DF93EB010297ACF169EE79E18A81C6
:103850009B810F942646892B29F40E94AFAF7D7F70
:103860000E94F4AF63EF79E18A819B810F94264631
:10387000892B29F40E94AFAF72600E94F4AF64E418
:1038800079E188E89EE00F94C91C0E94AFAF71FBFC
:10389000662760F971E0672770E088E89EE00E9483
:1038A00057AC88E89EE00F94CA1B88EC90E0DF914B
:1038B000CF9108950E947678F8CF0F931F93CF93FE
:1038C000DF93CDB7DEB769970FB6F894DEBF0FBEB2
:1038D000CDBFE091F510F091F610309709F460C07B
:1038E0008091021190910311892B09F459C08FEF37
:1038F000838714861382148215821682178210869B
:103900001186128664ED76E188E89EE00F94C91C6A
:1039100088E89EE00F94CA1BBE016E5E7F4F8091C7
:10392000F5109091F6100F9459381816CCF5A8950B
:10393000AE014F5F5F4F68E0CE0142960E94496A38
:10394000198ABE016F5F7F4F809102119091031120
:103950000E94C6AB8C016FEC76E188E89EE00F9484
:10396000C91CBE016F5F7F4F88E89EE00F94721CF8
:103970000115110591F0C8010E94EA778C01892B8D
:1039800059F26AEC76E188E89EE00F94C91CB80110
:1039900088E89EE00F94721CBBCF65EC76E1B4CF53
:1039A00088EC90E069960FB6F894DEBF0FBECDBFED
:1039B000DF91CF911F910F9108950F931F93CF9394
:1039C000DF9300D000D0CDB7DEB70E94FA796FE167
:1039D00074E188E89EE00F94C91CCE0101960F9413
:1039E000E035CE0101960E94877506E115E01A8345
:1039F000098380917B0C90917C0CA0917D0CB091FF
:103A00007E0C8B839C83AD83BE83CE0101960E9486
:103A100087751A8309831B821C821D821E8280E5A2
:103A200091E00E9418B844E050E0BE016D5F7F4F06
:103A300081E090E00F941E260F942C29CE01019670
:103A40000E9487751A8309831B821C821D821E8235
:103A500080E591E00E9418B844E050E0BE016D5F3F
:103A60007F4F85E090E00F941E260F942C29CE0105
:103A700001960E94877565E474E188E89EE00F94E2
:103A8000C91C88EC90E026960FB6F894DEBF0FBEF6
:103A9000CDBFDF91CF911F910F9108950D94A74451
:103AA000CF92DF92EF92FF920F931F93CF93DF930A
:103AB00000D000D0CDB7DEB780912E0A81119AC018
:103AC0008091FE109091FF1002970CF493C08091AA
:103AD000270A9091280A009709F48CC062E375E0E8
:103AE0000E94C6AB8C01009709F484C00E94E1AC2F
:103AF000E82EF12CE114F10409F47CC070E060E0E0
:103B0000C8010E94A76A6C01EA94EF2809F481C0F9
:103B100061E0C8010E943EACFC0101851285CE0126
:103B200001960F94E035CE0101960E941BB864E522
:103B30007FE088E89EE00F94C91CB60188E89EE00B
:103B40000F94721C63EC77E088E89EE00F94721C7F
:103B5000B80188E89EE00E9457AC63EC77E088E803
:103B60009EE00F94721C65EA7BE088E89EE00F946B
:103B7000721C88E89EE00F94CA1B62E072E087E541
:103B80009FE00F944F31D0924D0FC0924C0F109385
:103B90004F0F00934E0F85EA9BE0892BE9F580E3F8
:103BA00095E09093510F8093500F8091210A90914E
:103BB000220A009741F070E060E00E94A76A9093AB
:103BC000300A80932F0A80912F0A9091300A009733
:103BD00031F19093530F8093520F1092550F109222
:103BE000540F81E080932E0A6BE37FE088E89EE02B
:103BF0000F94C91C26960FB6F894DEBF0FBECDBF3A
:103C0000DF91CF911F910F91FF90EF90DF90CF90B8
:103C1000089502E012E083CF85EA9BE0C2CF80E7FF
:103C200092E0D7CFEF92FF920F931F93CF93DF9342
:103C300000D000D0CDB7DEB77C018B016AE67AE018
:103C400089E39FE00F94C91CD7011296ED91FC9176
:103C50006081718189E39FE00F94721C61E67AE0D4
:103C600089E39FE00F94C91C012E000C220B330B3B
:103C700009831A832B833C8380E190E09E838D83AC
:103C8000BE016F5F7F4F89E39FE00E94D1FA0F94DE
:103C9000CA1B40E050E860E070E0C7010E94EBE022
:103CA00026960FB6F894DEBF0FBECDBFDF91CF9141
:103CB0001F910F91FF90EF900895CF92DF92EF92B6
:103CC000FF920F931F93CF93DF93CDB7DEB7C1540D
:103CD000D1090FB6F894DEBF0FBECDBF6C01AB01AA
:103CE00030E020E060E4CE0101967C010E94787211
:103CF000F70101900020E9F731978F010E191F0994
:103D0000A801B701C6010F948F52892B11F010E062
:103D100000E0C801CF5BDF4F0FB6F894DEBF0FBEE7
:103D2000CDBFDF91CF911F910F91FF90EF90DF906A
:103D3000CF9008953F924F925F926F927F928F92B1
:103D40009F92AF92BF92CF92DF92EF92FF920F932A
:103D50001F93CF93DF93CDB7DEB72C970FB6F894B0
:103D6000DEBF0FBECDBF5C01362E972E3A01690132
:103D70006BEC7AE089E39FE00F94C91C632D792DE9
:103D800089E39FE00E9457AC63EC7AE089E39FE00F
:103D90000F94C91CC301B0E0A0E08F839887A98766
:103DA000BA8730E1432E512C5C864B86BE01695F99
:103DB0007F4F89E39FE00E94D1FA4C016FEB7AE0DC
:103DC0000F94C91CB601C4010E9457AC67EB7AE09E
:103DD000C4010F94C91CC701B0E0A0E089839A8395
:103DE000AB83BC835E824D82BE016F5F7F4FC40197
:103DF0000E94D1FA0F94CA1B80912C0A90912D0A2F
:103E000070E060E0892B09F047C081E090E090937A
:103E10002D0A80932C0A26E040E855E260E070E02D
:103E200087EB9BE00F94D51D3092B60C87EB9BE09F
:103E30009093B50C8093B40C1092C40D1092C60DE3
:103E40001092C50D0130110509F44EC00CF041C0AF
:103E5000012B09F44EC0C114D10409F457C082E00B
:103E6000C816D10409F062C070923F0D60923E0DF9
:103E70001092410D1092400DF092430DE092420DD0
:103E800086E00E9406C010922D0A10922C0A882308
:103E900009F456C0682F70E0C5010E94121E90E020
:103EA00080E02C960FB6F894DEBF0FBECDBFDF9139
:103EB000CF911F910F91FF90EF90DF90CF90BF9027
:103EC000AF909F908F907F906F905F904F903F90BA
:103ED00008950330110581F00430110509F0BBCFBE
:103EE000FE24EF24FE24B7CFFE2CEE24EE24EA9429
:103EF000B2CFFF24FA94AFCFEF2821F492E0E92E5D
:103F0000F12CEECFEE24E394F12CEACF70923F0D2A
:103F100060923E0D90E080E0EE2011F080E09FEF97
:103F20009093410D8093400D85E0ABCF6BE97AE033
:103F300089E39FE00F94C91C10922D0A10922C0A5D
:103F400081E090E0AECFCF92DF92EF92FF921F938D
:103F5000CF93DF9300D000D0CDB7DEB766E37FE02C
:103F600088E89EE00F94C91C8CE6E82E8EE0F82EBF
:103F700010E090E1C92ED12CF70181917F018031B1
:103F800030F469E375E088E89EE00F94721C153008
:103F900041F1F7013197808190E0B0E0A0E08983A2
:103FA0009A83AB83BC83DE82CD82BE016F5F7F4F7D
:103FB00088E89EE00E94D1FA64E37FE00F94C91C78
:103FC0001F5F1630C9F626960FB6F894DEBF0FBEF7
:103FD000CDBFDF91CF911F91FF90EF90DF90CF90F9
:103FE00008958091710E90E0B0E0A0E089839A83FB
:103FF000AB83BC83DE82CD82BE016F5F7F4F88E8DA
:104000009EE00E94D1FA0F94CA1BDACFEF92FF9282
:104010000F931F93CF93DF9300D000D01F92CDB7A3
:10402000DEB77B01CE0107969F938F9301979F93F5
:104030008F9301979F938F9301979F938F930197EE
:104040009F938F9301979F938F938E010F5F1F4FC5
:104050001F930F938BE395E09F938F93DB01139650
:104060008C9113978F9312968C918F930F94245366
:104070000FB6F894DEBF0FBECDBF0697ECF469ED26
:104080007AE182E99EE00F94C91CD70112966D91E6
:104090007C9182E99EE00F94721C80E991E0279662
:1040A0000FB6F894DEBF0FBECDBFDF91CF911F9149
:1040B0000F91FF90EF9008958091640E9091650E9E
:1040C000892BA9F10E9450AD882389F182E70E94D3
:1040D0003BAD8091640E9091650EDC01ED91FC91F9
:1040E0000088F189E02D64E070E019958091640EFC
:1040F0009091650EDC01ED91FC910280F381E02D41
:1041000046E050E0B801199586E0F801ACE6BEE063
:1041100001900D928A95E1F78091640E9091650E61
:10412000DC01ED91FC910488F589E02D19950E9440
:10413000A31F6BEE7AE188E89EE00F94C91C88EC1F
:1041400090E0ADCF0895CF92DF92FF920F931F932F
:10415000CF93DF93F12C6115710509F48DC06A01CD
:10416000EB018C01CB010E94FBDEF82E882309F4C1
:1041700083C0D6FE0EC0D8018C918B3009F450C09C
:1041800008F041C040E051E060E070E08A3009F49E
:1041900050C0D4FE09C0F801608186EF860F8430DC
:1041A00018F0CE010E946FE2D5FE66C0D8011496C9
:1041B0004D915D916D917C91179711968C918F70B7
:1041C000873030F08930C8F18A50823008F45DC001
:1041D000CE010E94A8DFEE81FF81309709F44CC028
:1041E00080858F709EEF980F923010F0811144C03F
:1041F000D80111968C91982F9295907F80858F7021
:10420000892B808739C08C3081F040E056E060E037
:1042100070E08D3009F0BDCFCE010E94EBE0B9CF48
:1042200040E051E060E070E0F7CF40E056E060E051
:1042300070E0CE010E94C2E0ACCFEE81FF813097EA
:10424000D9F080858F709EEF980F923010F0811119
:1042500013C04187528763877487EE81FF81808511
:10426000807F83608087EE81FF818085982F907F9B
:104270008F708067903629F28F2DDF91CF911F913B
:104280000F91FF90DF90CF900895CE010E94A8DF9C
:10429000F3CFCF93DF9300D000D01F921F92CDB702
:1042A000DEB7FC01628398E0DE01119601900D9269
:1042B0009A95E1F729813A814B815C816D817E81FC
:1042C0008F81988528960FB6F894DEBF0FBECDBFBC
:1042D000DF91CF910895CF93DF9300D000D01F924C
:1042E0001F92CDB7DEB7FC01608398E0DE01119626
:1042F00001900D929A95E1F729813A814B815C8179
:104300006D817E818F81988528960FB6F894DEBFE7
:104310000FBECDBFDF91CF910895CF93DF9300D033
:1043200000D01F921F92CDB7DEB7FC019181907F24
:104330009A609183448355836683778388E0DE01A6
:10434000119601900D928A95E1F729813A814B816E
:104350005C816D817E818F81988528960FB6F89457
:10436000DEBF0FBECDBFDF91CF910895AF92BF9258
:10437000CF92DF92EF92FF920F931F93CF93DF9331
:1043800000D000D01F921F92CDB7DEB76115710526
:1043900009F45FC05A016B017C01CB010E94FBDE76
:1043A000082F882369F1D60116968D919C9100976C
:1043B00009F443C0FC011085212F2F703EEF320F0E
:1043C000323010F021112EC012951F70B4FE59C06A
:1043D000C6010E948EE2F7018083112381F1818161
:1043E000807F182B1183D6011696ED91FC91818563
:1043F0009285A385B485F70184839583A683B783CB
:10440000802F28960FB6F894DEBF0FBECDBFDF9188
:10441000CF911F910F91FF90EF90DF90CF90BF90C1
:10442000AF900895253049F460E00E943EAC0097BB
:1044300021F0DC0118961C91C7CF10E0C7CFD60140
:104440001696ED91FC9180858F70823021F083303B
:1044500051F000E0D5CF4185528563857485C70151
:104460000E948D21CDCF4185528563857485F701EA
:104470008181807F876081834483558366837783CE
:10448000BFCF1123E1F2F701AACFCF93DF9300D082
:1044900000D01F921F92CDB7DEB7FC016F3F7105B0
:1044A00019F014F06FEF70E077FD60E09181892FD3
:1044B0008F7081508230C8F4648388E0DE011196E9
:1044C00001900D928A95E1F729813A814B815C81B7
:1044D0006D817E818F81988528960FB6F894DEBF16
:1044E0000FBECDBFDF91CF910895907F91609183F2
:1044F000E3CFCF92DF92EF92FF92DC01362F11963D
:10450000EC911197EF70EC3008F0B6C0F0E088271E
:10451000E357FD4D8F4F0D940E4E3F23C522C5220C
:104520003C233C233C230A23CC223C233C239922DA
:10453000992214968D919D910D90BC91A02D66238A
:1045400099F0B7FD9FC08F3F9105A105B10529F0F6
:1045500024F08FEF90E0A0E0B0E02FEF30E0A90171
:10456000481B590BCA010CC0B7FD89C08F3F91058C
:10457000A105B10529F024F08FEF90E0A0E0B0E0B4
:10458000FF90EF90DF90CF90089514962C91822F9A
:1045900090E06623A9F3E1CF1496CD90DD90ED90E5
:1045A000FC901797662301F120E030E0A901C701D4
:1045B000B6010F94394C87FD65C020E030E04FE72D
:1045C00053E4C701B6010F94414F18160CF457C0BD
:1045D000A701960160E070E08FE793E40F942C4E02
:1045E0000F940B4FCB01CCCF20E030E0A901C701E5
:1045F000B6010F94394C87FD42C020E030E04FE710
:1046000053E4C701B6010F94414F1816DCF1C701FE
:10461000B601E6CF14966D917D918D919C9117977F
:104620003323B1F06D395FEF75078507950754F1B6
:10463000611524E67207810591050CF52CE93FEF21
:104640004FEF5FEF0F94A54DC90181509F4F98CF59
:104650006D394FEF7407840794078CF0611554E6A9
:1046600075078105910574F424E630E040E050E0E0
:104670000F94A54DC90184CF8FEF9FEF81CF90E0BC
:1046800080E07ECF8FEF90E07BCFCF93DF93EC0184
:10469000DB0189818F708630E1F128F4815082300E
:1046A000C8F080E014C0873009F18A508230C8F722
:1046B0002FEF30E00F94254E24E630E040E050E04C
:1046C0000F94A54D2C833D834E835F8381E0DF9162
:1046D000CF9108952FEF30E00F94254E24E630E07F
:1046E00040E050E00F94A54D2C83F0CF2FEF30E049
:1046F0000F94254E24E630E040E050E00F94A54DA5
:10470000CA01B9010F94404C6C837D838E839F83D3
:10471000DDCF2CE933E60F94254E24E630E040E06F
:1047200050E00F94A54D2C833D834E835F83B9CF1A
:10473000DC011196EC911197EF70E150EB3008F02D
:1047400039C0F0E08827E855FC4D8F4F0D940E4E90
:10475000CB23CB23DA23B323B323BC23D323D32309
:10476000D323B323B32314966D917D918D919C91A6
:1047700017970F94404C089514966D917D918D91EB
:104780009C91179724E630E040E050E00F94A54D4F
:10479000CA01B901EECF14966C9170E090E080E010
:1047A0000F943E4C089514966D917D918D919C913E
:1047B0001797089560E070E0CB010895DC01119631
:1047C000EC911197EF70E150EB3008F037C0F0E05A
:1047D0008827E251FC4D8F4F0D940E4E002400248B
:1047E0001E24F923F9230F24062406240624F92382
:1047F000F92314966D917D918D919C911797089551
:1048000014966C9170E090E080E0089514966D919C
:104810007D918D919C9117970F940B4F089514964D
:104820006D917D918D919C91179724E630E040E049
:1048300050E00F94A54DCA01B901089560E070E001
:10484000CB010895DC011196EC911197EF70E150C6
:10485000EB3008F03EC0F0E08827EE5CFB4D8F4F58
:104860000D940E4E4824482469243D243D2462249E
:104870005324532453243D243D2414962D913D91DB
:104880004D915C911797A4E6B0E00F94C44D089544
:1048900014966C9184E6689FB0011124072E000CD9
:1048A000880B990B089520E030E048EC52E4149610
:1048B0006D917D918D919C9117970F949F4C0F94C2
:1048C0000B4F089514966D917D918D919C91179742
:1048D000089560E070E0CB010895FC01A7812A2FC4
:1048E0002E7FC9F081818F7081508330A0F4A6950E
:1048F000A150BB0B2BE531E00F94254E24E630E0B0
:1049000040E050E00F94A54DDA01C90187569F4F52
:10491000AF4FBF4F08958FEF9FEF08952F923F92B3
:104920004F925F926F927F928F929F92AF92BF92BF
:10493000CF92DF92EF92FF920F93CF93DF9300D04D
:104940001F92CDB7DEB77C017A8369835C834B838A
:10495000DB011C92FC0160818FEF860F883108F02B
:104960004BC034FF49C0FAE06F9FB00111246C5571
:10497000734FCD010F947B46D70111968C918F70A8
:1049800041F04B815C816CEB76E089819A810F94D8
:104990007F52E981FA8101900020E9F7319729815E
:1049A0003A81E21BF30B19012E0E3F1E4B815C81F5
:1049B0004E1B5F0B415051095C834B83D70111960D
:1049C000EC911197EF7009F4F5C0E150EC3008F06C
:1049D000F1C0F0E08827E051FB4D8F4F0D940E4E53
:1049E000FF24A2250F266E2689264D251F261F2669
:1049F0001F263B252325A52629803A80DFCFF701F6
:104A00008481282F30E050E040E0002359F030E06E
:104A1000A4E6B0E00F94D74D2FEF30E040E050E037
:104A20000F94A54D5F934F933F932F938FE495E0A1
:104A30009F938F93FC81FF932B812F933F922F9213
:104A40000F94B752B2C017968C9117978F93169602
:104A50008C9116978F9315968C9115978F9314962A
:104A60008C918F9382E595E09F938F93BC81BF9348
:104A7000EB81EF93E3CF17968C9117978F93169650
:104A80008C9116978F9315968C9115978F931496FA
:104A90008C918F9386E595E0E7CF1496CD90DD90CD
:104AA000ED90FC901797F7FE34C084E6882E912C89
:104AB000A12CB12CC701B601A50194010F94A54DFD
:104AC0009B01AC0188279927DC01821B930BA40B67
:104AD000B50BBF93AF939F938F9366277727CB0137
:104AE0006C197D098E099F09A50194010F94A54DAC
:104AF0005F934F933F932F938AE595E09F938F9316
:104B00003C813F934B814F933F922F920F94B7522A
:104B10004CC0C701B60124E630E040E050E00F94FD
:104B2000A54D9F938F937F936F935F934F933F9385
:104B30002F938BE595E09F938F939C819F93AB81FF
:104B4000AF93E2CFC7010E946D24BC01D701169636
:104B5000CC9016971796DC901797D0FADD24D0F8F2
:104B600014969C9114971596FC90EB80BC80292F8D
:104B700030E050E040E077FD35C0011135C07F9353
:104B80006F931F921F921F929F931F92FF92DF922B
:104B9000CF9284E695E09F938F93FC81FF932B81C6
:104BA0002F933F922F920F94B7520FB6F894DEBF17
:104BB0000FBECDBF89819A810F900F900F900F90FB
:104BC000DF91CF910F91FF90EF90DF90CF90BF904A
:104BD000AF909F908F907F906F905F904F903F909D
:104BE0002F900895002361F0292F30E0A4E6B0E073
:104BF0000F94D74D2FEF30E040E050E00F94A54DDB
:104C00005F934F933F932F931F92FF92DF92CF9228
:104C100087E695E09F938F93BF92EF9275CF15969D
:104C20008C9115971F928F9316969C9116971796B5
:104C30008C9181708F939F938AE695E015CF14969F
:104C40008D909D90AD90BC90179720E030E0A90129
:104C5000C501B4010F94394C2401350187FF04C00C
:104C600077FA709477F87094C301B2010F940B4FE8
:104C70006B01072E000C880B990B0F94404C9B0185
:104C8000AC01C301B2010F942C4E20E030E04AE7A2
:104C900054E40F949F4C0F94964F0F940B4F062F94
:104CA000772E20E030E0A901C501B4010F94394C02
:104CB00087FF07C07F920F93DF92CF9280E795E046
:104CC000D3CE7F920F93DF92CF9281E795E09F93AF
:104CD0008F933C813F934B814F93B0CE14968C9130
:104CE00014971F928F9315968C9115971F928F93FF
:104CF00016968C911F928F9387E695E09F938F93E2
:104D0000BC81BF93EB81EF933F922F920F94B752E8
:104D10004CCF17968C9117971F928F9314968C9166
:104D200014971F928F9315968C9115971F928F93BE
:104D300016968C911F928F9384E695E09F938F93A4
:104D4000BC81BF93EB81EF93DFCE14966D917C9184
:104D50004B815C81C1010F949D522CCFEF92FF9249
:104D60000F93CF93DF93CDB7DEB7A0970FB6F8942C
:104D7000DEBF0FBECDBF7C0100E020E030E340E2AB
:104D800050E0BE016F5F7F4F0E948E24BE016F5FB7
:104D90007F4F89E39FE00F94721C65EA7DE089E311
:104DA0009FE00F94C91CF70161816F7089E39FE058
:104DB0000E9450AC6EE97DE089E39FE00F94C91C2E
:104DC000F701628189E39FE00E9450AC89E39FE094
:104DD0000F94CA1BA0960FB6F894DEBF0FBECDBFCE
:104DE000DF91CF910F91FF90EF900895CF93DF93D4
:104DF000EC016115710539F48F8181708F8381E039
:104E0000DF91CF9108958981982F9F7029F180E0DB
:104E10009430B0F79B01770F440B550B295931099A
:104E200041095109A4E6B0E00F94C44D2BE531E0EF
:104E300040E050E00F94A54D37FF02C030E020E085
:104E40002536310514F024E630E02F5F220F8F81E4
:104E50008170282B2F83D3CF807F82608983DACF24
:104E60002F923F924F925F926F927F928F929F927A
:104E7000AF92BF92CF92DF92EF92FF920F931F9368
:104E8000CF93DF93CDB7DEB768970FB6F894DEBF48
:104E90000FBECDBF6C0109871A872B873C874D87D2
:104EA0005E876F87788B22E1E216F10480F5F701C7
:104EB000E75EFC4F3081398BCE0109960E946D244C
:104EC00097FD04C0BC01C6010E94F6268B85D60161
:104ED00012968C93129789858C931196EC91119769
:104EE000EF70EC3008F06CC0F0E08827E558F84D22
:104EF0008F4F0D940E4ED628A427A4271D2989274D
:104F00009929E928272927292729E928E928198A19
:104F1000D3CFF12C9A859F709D3008F0A7C4E92F5C
:104F2000F0E08827E956F84D8F4F0D940E4EE0279C
:104F3000D129F129D1299C299C29D129D129362C83
:104F4000362CD129D129A8289A859F709D3008F048
:104F50000FC1E92FF0E08827EF54F84D8F4F0D94E3
:104F60000E4EE02786287928D627C127BE275D2840
:104F70008828B828B82847284728A8288889F6010B
:104F800087838F85D60116968C9316978E851596F6
:104F90008C9315978D8514968C93149711968C91FC
:104FA0001197807F892B11968C930AC08F859889E1
:104FB000F6018683878190FB80F987838E858583C0
:104FC000B989BB2309F460C0F60181818F702B2F52
:104FD00030E08217130609F457C069EA7BE089E3E1
:104FE0009FE00F94C91CD60111966C916F7089E3F4
:104FF0009FE00E9450AC66EA7BE089E39FE00F945B
:10500000C91C698989E39FE00E9450AC64EA7BE097
:1050100089E39FE00F94C91CF601008119821A826E
:105020001B821C821D821E821F82188689898F70B6
:105030009A81907F892B8A830983EE24EA94FE2C3F
:105040001181228133814481558166817781CE012E
:1050500001960E943027D6012C9311963C9311970C
:1050600012964C93129713965C93139714966C9325
:10507000149715967C93159716968C9316971796FA
:105080009C93C6010E94AE2688E0F60163C18D851F
:105090009E85AF85B889B7FD0EC08F3F9105A105EC
:1050A000B10529F024F08FEF90E0A0E0B0E0D60148
:1050B00014968C9385CF80E0FACF6D857E858F85A1
:1050C000988920E06D39BFEF7B078B079B076CF059
:1050D0002FEF6115E4E67E078105910534F424E69F
:1050E00030E040E050E00F94A54DD60114962C938B
:1050F00067CF8F859889F6018683878190FB80F939
:1051000087838E8585838D8584835ACF8D85CFCF88
:105110008D849E84AF84B88820E030E0A901C50169
:10512000B4010F94394C60E087FD0FC020E030E0FF
:105130004FE753E4C501B4010F94414F6FEF1816C8
:1051400024F0C501B4010F94124FF601648338CFE7
:10515000D60111968C911197807F8C6011968C935B
:1051600011978D859E8515969C938E93149728CFC5
:1051700069E27CE089E39FE00F94C91C6A856F7047
:1051800089E39FE00E9450AC66E27CE089E39FE007
:105190000F94C91CF60161816F7089E39FE00E9442
:1051A00050AC89E39FE00F94CA1B0ACF9A859F7089
:1051B00011968C911197807F892B11968C938D85F8
:1051C0009E85AF85B889F60184839583A683B783CE
:1051D000F7CE9A859F70933089F09C3009F4B8CF50
:1051E0004D855E856F857889F60144835583668396
:1051F00077838181807F892B8183E2CE60E0C60145
:105200000E947922D60114968C9314978F859889E1
:1052100016968C93169717968C91179790FB80F99A
:1052200017968C9317978E8515968C9315971196D4
:105230008C911197807F8260B6CE60E0CE01099696
:105240000E947922D60114968C931497F0CF9A85F8
:105250009F709D3008F057C0E92FF0E08827EC5C84
:10526000F64D8F4F0D940E4EE0274E297B29FE28D8
:105270007B297B2941296D296D296D295C296829A4
:10528000A8288D859E85AF85B889F601848395838E
:10529000A683B7838181807F8660AECF6D8570E005
:1052A00090E080E00F943E4CD60114966D937D9370
:1052B0008D939C93179784CE6D857E858F85988975
:1052C0000F94404CF601648375838683978378CE70
:1052D0006D857E858F859889E5CFF6018181807FF8
:1052E000982B91838D859E85AF85B889848395831E
:1052F000A683B78365CE11968C911197807F982BEA
:1053000011969C935CCF64E17CE089E39FE00F946D
:10531000C91C6A856F7089E39FE00E9450AC61E10F
:105320007CE089E39FE00F94C91CD60111966C9133
:1053300033CFFF24F394EECD4D855E856F8578895C
:10534000F60144835583668377838181807F982B20
:10535000918388E0DE01119601900D928A95E1F724
:1053600029813A814B815C816D817E818F81988515
:1053700068960FB6F894DEBF0FBECDBFDF91CF9118
:105380001F910F91FF90EF90DF90CF90BF90AF9063
:105390009F908F907F906F905F904F903F902F9055
:1053A0000895963009F437C148F46D85913071F055
:1053B0006FEF70E0933051F060E008C0973009F46F
:1053C00036C19A506D857E859230B0F784E68F871E
:1053D00088898E7F888B1E868A85807F82608A87F7
:1053E0006D872E8530E0AFEFB0E00F94D74D812C64
:1053F000912C54018A946115F4E67F07810591058B
:1054000044F424E630E040E050E00F94A54D49011B
:105410005A0114012D852A8B022F10E0FF2009F478
:1054200070C088898695A82FA150BB0B7D01BFEF66
:10543000EB16FB0609F01BC1E0E88E1691040CF098
:10544000FDC08FE790E088199909809FD001819F66
:10545000B00D909FB00D11242FEF30E00F94254E2A
:1054600021E83EE740E050E00F94A54DD6011796A5
:105470002C93ABE9B0E0A50194010F94C44D3FE734
:10548000432E512C612C712CA30192010F94A54D38
:105490002C593F4F4F4F5F4F1901AEEFB1E0A501BF
:1054A00094010F94C44DA30192010F94A54DD8010E
:1054B0000F94C44D2FEF30E040E050E00F94A54D25
:1054C00089012F3F310519F014F00FEF10E064E06F
:1054D0007CE089E39FE00F94C91CB10189E39FE060
:1054E0000E9457AC66EF7BE089E39FE00F94C91CF4
:1054F000B80189E39FE00E9457AC89E39FE00F94D5
:10550000CA1BE2E9F8E2E491F0E0EE0FFF1FE85871
:10551000F74D85919491E8EDF8E2E4912F85388973
:105520003170AFEFBFEF0F94D74D2DE631E040E083
:1055300050E00F94A54D44275527AAEFB5E00F94EE
:10554000C44DDC01CB019058AF4FBF4FCD01BB27FD
:1055500097FDB095AB2F8E3FE1E09E0708F05FC14D
:10556000382F8F3F910508F47CC14EEF481B50E067
:105570003FEF0F5F1F4FF101FF2731962094312C31
:105580003E9FC0013F9F900D1124292F3327220DEC
:10559000331DD8010F94254E4B015C018824AA24A9
:1055A000BB245E9F90015F9F300D1124232F332772
:1055B000220D331D0F94254EBB27A92F982F872F1F
:1055C000882A992AAA2A4E9F90014F9F300D1124B4
:1055D000232F3327220D331DD8010F94254EB82FCA
:1055E000A72F962F882788279927BB2788299929AD
:1055F000AA29F601A683958384836AEC7BE089E37C
:105600009FE00F94C91CC6010E94AE2660E080E0B6
:105610000E9431BCD5CC6D857E858F85988924E626
:1056200030E040E050E00F94A54DB901CFCE6D853C
:105630007E858F8598890F940B4FC8CEA501940164
:105640002058310941095109ABE9B0E00F94C44D2C
:105650002FE730E040E050E00F94A54D2C593F4F2C
:105660004F4F5F4F1901D60117961C9230CF97010B
:10567000AAEBBFEF0F941D4E24E630E040E050E06F
:105680000F94A54D29013A01B4E64B0E511C611C43
:10569000711C26E430E0D7010F94254E24E630E05B
:1056A00040E050E00F94A54DDA01C9014E96A11DCE
:1056B000B11D8D8B9E8BAF8BB88F90E889169104AE
:1056C0000CF092C08FE790E088199909809FD00173
:1056D000819FB00D909FB00D11242D893E894F8977
:1056E000588D0F94CF4D9B01AC01AFEFB0E00F94FC
:1056F000C44D24E63AE640E050E00F94A54DD601B3
:1057000017962C93A5019401240D351D461D571D98
:10571000AEEFB1E00F94C44D23EE30E040E050E036
:105720000F94A54D79018A013C8B2B8BAFEFB0E034
:10573000A50194010F94C44D2FE730E040E050E004
:105740000F94A54D1901EA89AE2FB0E0A801970189
:105750000F94C44D2FEF30E040E050E00F94A54D82
:1057600089012F3F310519F014F00FEF10E060EFC1
:105770007BE089E39FE00F94C91C2AE030E0B3018D
:10578000A20189E39FE00F94EC1B6AEE7BE089E3C2
:105790009FE00F94C91C2AE030E04D895E896F8933
:1057A000788D89E39FE00F94EC1B62EE7BE089E348
:1057B0009FE00F94C91CB10189E39FE00E9457ACA0
:1057C0006AED7BE089E39FE00F94C91CB80189E38F
:1057D0009FE00E9457AC61ED7BE089E39FE00F946E
:1057E000C91C6B897C8985CEA5019401205831099B
:1057F00041095109ABE9B0E00F94C44D2FE730E007
:1058000040E050E00F94A54D2C593F4F4F4F5F4F54
:105810001901D60117961C921C8A1B8AA8CF8C3FAF
:10582000F3E09F0768F48D3F22E0920728F452E0EE
:10583000580F3FEF40E09DCE3CEF381B5FEFFACFB3
:105840008A3F35E0930781F08B3FE4E09E0728F420
:1058500044E0480F5FEF30E08CCE5AEF581B30E049
:1058600001C050E04FEF85CE50E0F9CF68EB7BE010
:1058700089E39FE00F94C91C6A856F7089E39FE0FC
:105880000E9450AC65EB7BE04CCDFC019181892FEF
:105890008F7021F0823029F080E00895907F92602F
:1058A00091839B0177FF02C030E020E02E3681E03B
:1058B000380714F02DE631E02683878130FB80F92C
:1058C000878381E00895EF92FF920F931F93CF9308
:1058D000DF93FC01892B69F19081992351F19D326D
:1058E00091F180ED890F8A3070F1C8E0D0E09532F7
:1058F00011F1CEEFDFEF9B37F1F0C7E1D0E093324B
:10590000D1F08F018EEAE82E8CE0F82EC1E0D0E0D5
:10591000C7010F945446AC01B701C8010F946D46FE
:10592000892B49F021968AE0E80EF11CC931D10596
:1059300079F7CFEFDFEFCE01DF91CF911F910F917C
:10594000FF90EF900895D0E0C0E0F5CFEF92FF9286
:105950000F931F93CF93DF93EC01892B51F188852F
:105960008F70843009F5E984FA84C7010E94632CA2
:105970008C0118161906ECF4C7010F948423C80192
:10598000012E000CAA0BBB0B89879A87AB87BC87BB
:105990008885807F82608887C801DF91CF911F91C1
:1059A0000F91FF90EF900895823019F409851A85C0
:1059B000F3CF10E000E0F0CF2F923F924F925F9232
:1059C0006F927F928F929F92AF92BF92CF92DF920F
:1059D000EF92FF920F931F93CF93DF93CDB7DEB774
:1059E000A4970FB6F894DEBF0FBECDBF7C016B014C
:1059F00066E577E0C6010E94C6ABFC01892B09F47D
:105A000022C180858F70843009F455C0853009F03B
:105A10001AC1068117810115110509F414C1D801B5
:105A200018968C9118978F70823019F412960D91F8
:105A30001C910115110509F406C1F80180858F70CC
:105A4000853011F0D801F2CFC8010E94E1AC82305C
:105A5000C9F760E0C8010E943EAC5C010E94A62C20
:105A600061E0C8010E943EAC4C01FC0180858F7052
:105A7000823041F7C7010E94DE23D40119964D9070
:105A80005D906D907C901C97641575058605970553
:105A9000C9F6A114B10409F4D6C019861A861B866A
:105AA0001C861D861E861F86188A8A85807F8A87A7
:105AB000F50161854DC069E775E0818592850F9498
:105AC0006F52892B09F0BFC0C7010E94DE23611508
:105AD00071058105910509F49CC0660F771F881F29
:105AE000991F2FEF30E040E050E00F94A54D57FD97
:105AF00016C023303105410551050CF070C0DA01A4
:105B0000C9010196A11DB11D82309105A105B10504
:105B100009F44BC00397A105B10509F460C0198AC7
:105B20001A8A1B8A1C8A1D8A1E8A1F8A188E8A89D5
:105B3000807F8A8B67E0CE0141960E9449212987A8
:105B40003A874B875C876D877E878F87988B62E16A
:105B5000CE0109960E946B2129833A834B835C8393
:105B60006D837E838F83988729813A814B815C8105
:105B70006D817E818F819885A4960FB6F894DEBFE3
:105B80000FBECDBFDF91CF911F910F91FF90EF908E
:105B9000DF90CF90BF90AF909F908F907F906F904D
:105BA0005F904F903F902F900895198A1A8A1B8A10
:105BB0001C8A1D8A1E8A1F8A188E8A89807F8A8B7A
:105BC00067E0CE0141960E94492129873A874B8799
:105BD0005C876D877E878F87988B61E1B9CF198A43
:105BE0001A8A1B8A1C8A1D8A1E8A1F8A188E8A8915
:105BF000807F8A8B67E0CE0141960E9449212987E8
:105C00003A874B875C876D877E878F87988B60E1AB
:105C10009FCF198A1A8A1B8A1C8A1D8A1E8A1F8A8C
:105C2000188E8A89807F8A8B67E0CE0141960E9418
:105C3000492129873A874B875C876D877E878F87C5
:105C4000988B62E085CF6DE775E0C6010E94C6AB18
:105C50008C01009709F41CC1DC0118968C918F709F
:105C6000853009F0FEC0C8010E94E1AC843008F420
:105C70000FC160E0C8010E943EAC5C0161E0C80158
:105C80000E943EAC3C0162E0C8010E943EACDC01D7
:105C900019962D913D914D915C911C97298F3A8FCA
:105CA0004B8F5C8F63E0C8010E943EAC4C0165E005
:105CB000C8010E943EAC6C0167E0C8010E943EAC86
:105CC0008C01C7010E94DE23298D3A8D4B8D5C8D9E
:105CD000621773078407950714F5C114D10409F4FA
:105CE000C2C0D60118968C9118978F70823009F037
:105CF000BAC019861A861B861C861D861E861F86BC
:105D0000188A8A85807F8A8719964D915D916D9159
:105D10007C911C97CE0109960E948D211DCFD40144
:105D200019962D913D914D915C911C972D8F3E8F31
:105D30004F8F58A32617370748075907D4F4011582
:105D4000110509F490C0F80180858F70823009F048
:105D50008AC019861A861B861C861D861E861F868B
:105D6000188A8A85807F8A874185528563857485F4
:105D7000D1CFD5011996CD90DC90F30121843284E6
:105D800019861A861B861C861D861E861F86188A03
:105D90008A85807F8A872101032C000C660877089A
:105DA00046010D2C000CAA08BB08098D1A8D012E86
:105DB000000C220B330B09A31AA32BA33CA3C7018E
:105DC0000E94DE239B01AC01E9A0FAA00BA11CA15B
:105DD0002E193F09400B510BC301B2016819790913
:105DE0008A099B090F94734D0D8D1E8D9801110F1B
:105DF000440B550BE9A0FAA00BA11CA12E193F09D9
:105E0000400B510B0F94A54D820E931EA41EB51E80
:105E1000C1018C199D096D8D7E8D098D1A8D601BB8
:105E2000710B0F94FA4D77FF02C06F5F7F4F75952E
:105E30006795CB01770FAA0BBB0B880D991DAA1D87
:105E4000BB1D40E050E0BA01B7FD64CFB301A20131
:105E500084179507A607B7070CF05CCFAC01BD010E
:105E600059CF811115C019861A861B861C868A8512
:105E7000807F8A871D861E861F86188A88E0FE011D
:105E80003996DE01119601900D928A95E1F76CCE5C
:105E900088E0F701F6CF2F923F924F925F926F9278
:105EA0007F928F929F92AF92BF92CF92DF92EF92AA
:105EB000FF920F931F93CF93DF93CDB7DEB7659714
:105EC0000FB6F894DEBF0FBECDBF6115710549F561
:105ED00028E0FC01DE01119601900D922A95E1F770
:105EE00029813A814B815C816D817E818F8198858A
:105EF00065960FB6F894DEBF0FBECDBFDF91CF9190
:105F00001F910F91FF90EF90DF90CF90BF90AF90D7
:105F10009F908F907F906F905F904F903F902F90C9
:105F200008953B018C0166E577E0C3010E94C6AB92
:105F30006C01D801FC90FF2009F45AC0009709F4C5
:105F400057C0FC0180858F70843009F4DEC0853035
:105F500009F04EC080911E02893020F480911D020C
:105F6000893050F061E875E089E39FE00F94721C7E
:105F700089E39FE00F94CA1BD6011696ED90FC9022
:105F8000E114F104A9F1F70180858F705701823087
:105F900069F0B12CA12CE114F10409F436C1D70148
:105FA00018968C918F70853021F0F701E280F38094
:105FB000F2CFC7010E94E1AC8230B9F760E0C701BF
:105FC0000E943EAC0E94A62C4C0161E0C7010E94D9
:105FD0003EAC6C01D8018C918815190431F7F6019B
:105FE00080858F70823009F7C114D10409F017C180
:105FF0006DE775E0C3010E94C6AB7C01D801119624
:106000008C918F7009F43BC1E114F10409F43BC198
:10601000F70180858F70853009F0D0C1C7010E94DB
:10602000E1AC843008F4CAC164E0C7010E943EAC10
:106030006C0166E0C7010E943EAC1C01C8010E94D1
:10604000DE234B015C0160E0C7010E943EACDC0135
:1060500019964D905D906D907C901C97B0911E02AA
:10606000B98B84149504A604B7040CF016C1B9309A
:1060700020F480911D02893050F164E87CE089E3CE
:106080009FE00F94C91CC8010E94DE23AB01BC0134
:106090002AE030E089E39FE00F94EC1B6EE67CE0A1
:1060A00089E39FE00F94C91C60E0C7010E943EACE9
:1060B000FC0141855285638574852AE030E089E3DF
:1060C0009FE00F94EC1B89E39FE00F94CA1BC1145F
:1060D000D10409F479C1D60118968C9118978F7064
:1060E000823009F071C119821A821B821C821D82C2
:1060F0001E821F8218868A81807F8A8319964D911D
:106100005D916D917C911C9743C069E775E0818535
:1061100092850F946F52892B09F06ACFB0E1FB167C
:1061200009F463C0BF1580F0E2E0FE1619F1D80152
:106130004D915D916D917C91139714968D919D91E8
:106140000D90BC91A02D38C0F1E1FF16F1F122E1D4
:10615000F212EDCF19821A821B821C821D821E82CE
:106160001F8218868A81807F8A8344E150E060E044
:1061700070E00EC019821A821B821C821D821E8250
:106180001F8218868A81807F8A8340E050E0BA01AE
:10619000CE0101960E948D2129873A874B875C8723
:1061A0006D877E878F87988B49855A856B857C851F
:1061B0008D859E85AF85B88949835A836B837C839F
:1061C0008D839E83AF83B8878BCE19821A821B8200
:1061D0001C821D821E821F8218868A81807F8A838C
:1061E00040E850E060E070E0D3CF19821A821B8251
:1061F0001C821D821E821F8218868A81807F8A836C
:106200004FEF50E060E070E0C3CFA114B10409F497
:10621000EFCEF50180858F7009F4EACE650180919B
:106220001E02893020F480911D028930B8F060E9A7
:106230007CE089E39FE00F94C91CD60119964D912B
:106240005D916D917C911C972AE030E089E39FE09D
:106250000F94EC1B89E39FE00F94CA1B19821A82EA
:106260001B821C821D821E821F8218868A81807F6B
:106270008A83F601418552856385748589CFE1144F
:10628000F10409F09BC0F801408151816281738162
:1062900084819581A681B7818FCF61E0C7010E947B
:1062A0003EACDC0119962D913D914D915C911C976E
:1062B0002A8B3B8B4C8B5D8B281539054A055B057A
:1062C0003CF5B989B93020F480911D02893050F035
:1062D00060E57CE089E39FE00F94C91C89E39FE0BF
:1062E0000F94CA1B2114310409F46EC0F10180859A
:1062F0008F70823009F068C019821A821B821C825A
:106300001D821E821F8218868A81807F8A83B2CF77
:1063100063E0C7010E943EAC8C0162E0C7010E94AD
:106320003EACDC011996CD90DD90ED90FC901C9771
:10633000F80121853285438554852C193D094E0984
:106340005F09C501B40164197509860997090F949D
:10635000734D2A893B894C895D8924193509460981
:1063600057090F94A54DC20ED31EE41EF51EF989E0
:10637000F93020F480911D02893090F06BE37CE0CD
:1063800089E39FE00F94C91C2AE030E0B701A60121
:1063900089E39FE00F94EC1B89E39FE00F94CA1BF5
:1063A00019821A821B821C821D821E821F821886FD
:1063B0008A81807F8A83B701A601EACED701189629
:1063C0008C918F7009F05FCF19821A821B821C8218
:1063D0008A81807F8A8349815A816B817C8180E0B8
:1063E00090E0DC01E9CE8F929F92AF92BF92CF9264
:1063F000DF92FF920F931F93CF93DF93EC018A817B
:106400009B810E94E1AC082F10E00430110554F488
:106410000E946BB1BC018A819B810E9478B10F5FA1
:106420001F4FF3CFEA81FB8106811781011511050A
:1064300031F0D80112968D919C919D838C83EC81D3
:10644000FD81309721F0828193819F838E83EE813D
:10645000FF81309749F00280F381E02D309721F0E1
:1064600082819381998788870115110541F0F80190
:1064700080858F70843059F128F4823071F0FF24C8
:10648000FA940CC0853001F18630C9F76FE875E0E9
:10649000C8010E94C6AB8C01E7CFF184FA86CE0119
:1064A0000E94FBDE811138C010E000E01C870B87E2
:1064B000DF91CF911F910F91FF90DF90CF90BF9010
:1064C000AF909F908F90089506811781CDCFC184A2
:1064D000D284C114D10499F2F6018081882379F223
:1064E00095ED892E9AE0992EB12CA12CFA2CC4019D
:1064F0000F945446AC01B401C6010F946D46892B2C
:10650000B9F1FFEFAF1ABF0A89E0880E911CA7E12D
:10651000AA16B10459F7B3CFCE010E947EB08C0108
:106520000097B1F0FC0182819381892B39F08F2D86
:106530000E9496B18C01892B09F4B6CFD801ED9158
:10654000FC910684F785E02DBE01C8011995AECFF8
:106550008F2D0E9496B18C01892B09F4A5CFEA8575
:10656000F0E0EE0FFF1FE858F04F11830083E6CFF5
:10657000C6010F9484238A2D90E0B0E0A0E0F801DA
:1065800081879287A387B4878085807F8260808798
:1065900085CFCF92DF92EF92FF920F931F93CF930D
:1065A000DF9300D000D01F921F92CDB7DEB77C01E1
:1065B00009831A832B833C834D835E836F837887A3
:1065C000CE0101960E945FAC8C018981882351F035
:1065D0009B81923008F0B6C0823011F0853011F402
:1065E00010E000E070E060E0C7010E9418E0D82EE3
:1065F000C92E6EE77AE089E39FE00F94C91C6D2DE8
:106600007C2D89E39FE00E9457AC6CE77AE089E338
:106610009FE00F94C91CB80189E39FE00E9457AC2A
:1066200089E39FE00F94CA1B80912C0A90912D0A58
:10663000892BE9F040E050E3B701CE0101960E94BA
:10664000A32070E060E0C7010E94121E90E080E08D
:1066500028960FB6F894DEBF0FBECDBFDF91CF9165
:106660001F910F91FF90EF90DF90CF90089581E000
:1066700090E090932D0A80932C0A26E040E855E2A2
:1066800060E070E087EB9BE00F94D51DD092B60CD4
:1066900087EB9BE09093B50C8093B40C1092C40DE3
:1066A0001092C60D1092C50D80ED97E090933F0DAE
:1066B00080933E0D1092410D1092400D0115110571
:1066C000E1F185E090E09093430D8093420D86E0E8
:1066D0000E9406C0D82E64E670E080E090E00E9440
:1066E00079BED1100AC065E77AE089E39FE00F9494
:1066F000C91C89E39FE00F94CA1B82ED97E0909339
:106700003F0D80933E0D1092410D1092400D24E6F6
:10671000209FC001219F900D11249093430D8093E1
:10672000420D86E00E9406C010922D0A10922C0A9B
:10673000882359F0682F70E086CF1092430D109295
:10674000420DC5CF8FEF9FEF83CF81E090E080CFE8
:106750002F923F924F925F926F927F928F929F9271
:10676000AF92BF92CF92DF92EF92FF920F931F935F
:10677000CF93DF93CDB7DEB72C970FB6F894DEBF7B
:106780000FBECDBF5C0109831A832B833C834D83ED
:106790005E836F837887CE0101960E945FAC1C01F7
:1067A000023011F0053011F4312C212CF501048157
:1067B0001581F80180858F70853009F07FC0C80190
:1067C0000E94E1ACE82EF12CF2E0EF16F1040CF49B
:1067D00075C060E0C8010E943EACFC0181859285D5
:1067E0009C878B8761E0C8010E943EACFC0141841C
:1067F00052846384748488248A94982CF2E0EF167F
:10680000F10459F062E0C8010E943EACFC018184B1
:106810009284F3E0EF16F104A1F48FE390E09A87FD
:10682000898792E0C92ED12C29853A85D1010F9410
:106830001D4E24E630E040E050E00F94A54D790174
:106840001CC063E0C8010E943EACFC0181859285BA
:106850009A87898782E0C82ED12CF4E0EF16F104E4
:1068600039F064E0C8010E943EACFC01C184D284CE
:1068700089859A857101892BB9F684019601A20157
:106880006B857C85C5010E949A1E2C960FB6F894E4
:10689000DEBF0FBECDBFDF91CF911F910F91FF9053
:1068A000EF90DF90CF90BF90AF909F908F907F90B0
:1068B0006F905F904F903F902F90089590E080E010
:1068C000E4CF2F923F924F925F926F927F928F927E
:1068D000AF92BF92CF92DF92EF92FF920F931F93EE
:1068E000CF93DF93CDB7DEB7C457D1090FB6F89475
:1068F000DEBF0FBECDBF3C01AE960FAFAE97AF96D9
:106900001FAFAF97E0962FAFE097E1963FAFE197CB
:10691000E2964FAFE297E3965FAFE397E4966FAFEF
:10692000E497E5967FAFE59723961FAE1EAE2397BB
:10693000FE01ED5BFF4F82E1DF011D928A95E9F7D1
:106940007296119211928EE0DF011D928A95E9F7FD
:1069500064E975E089E39FE00F94721CB50189E357
:106960009FE00F94721C6CEB76E089E39FE00F943C
:10697000721CCE0183599F4F0E94AE26D4FE2CC0BC
:10698000AE96EFADAE97E83108F067C1F0E088272A
:10699000E353FB4C8F4F0D940E4E3336E5342A36BD
:1069A0002D362D362A36E5342D362D362D362D361C
:1069B0002D362D362D36E534E5342D362D362D3653
:1069C000E534E534E534E534333661E779E0CE018A
:1069D0008B5A9F4F0F944D460E94E4AB882309F4D5
:1069E00019C18091F910811115C1A114B10409F0E8
:1069F0005FC030E020E043E050E060E4CE0101966B
:106A00000E947872D3011296ED91FC9160817181A0
:106A10004FE350E0CE0101960F947F52D5FE26C180
:106A2000AE968FADAE97823009F420C1853009F45F
:106A30001DC1AF968FADAF978F709FE0980F9F707D
:106A4000923018F0883009F011C101E020E030E206
:106A500044E150E0BE016F5B7F4FCE0183599F4FF1
:106A60000E948E24482DBE016F5B7F4FCE010196A0
:106A70000E947ABF67E479E089E39FE00F94C91C24
:106A8000BE016F5F7F4F89E39FE00F94721C64E447
:106A900079E089E39FE00F94C91CBE016F5B7F4FD3
:106AA00089E39FE00F94721C89E39FE00F94CA1B57
:106AB000AF968FADAF978F70160127012224332434
:106AC000B0E14B225524882311F0D5FC06C02114D7
:106AD00031044104510409F409C130E020E043E0ED
:106AE00050E060E4CE0101960E947872D3011296C4
:106AF000ED91FC91608171814FE350E0CE010196F0
:106B00000F947F52A114B10469F061EA75E0CE01DF
:106B100001960F9459524FE350E0B501CE01019612
:106B20000F947F5261EA75E0CE0101960F9459529D
:106B30004FE350E069E079E021143104410451044D
:106B400059F4E0968FADE0974FE350E068E179E0CB
:106B5000873011F06FEF78E0CE0101960F945D461B
:106B6000AF968FADAF978F708450823008F0A5C07C
:106B700067E1CE0183599F4F0E946B21A6962FAFEC
:106B8000A697A7963FAFA797A8964FAFA897A996A5
:106B90005FAFA997AA966FAFAA97AB967FAFAB9757
:106BA000AC968FAFAC97AD969FAFAD9700E020E06D
:106BB00030E344E150E0BE016F5B7F4FCE0183596B
:106BC0009F4F0E948E246FEE78E089E39FE00F9440
:106BD000C91CBE016F5F7F4F89E39FE00F94721C59
:106BE0006CEE78E089E39FE00F94C91CBE016F5BF7
:106BF0007F4F89E39FE00F94721C89E39FE00F941D
:106C0000CA1B0E94E4AB882329F08091F9108823E5
:106C100009F45DC0B701A601C3010E94EBE090E05A
:106C200080E0CC58DF4F0FB6F894DEBF0FBECDBF6B
:106C3000DF91CF911F910F91FF90EF90DF90CF9058
:106C4000BF90AF908F907F906F905F904F903F90EC
:106C50002F9008956BE779E0BACE6DE479E089E38F
:106C60009FE00F94C91CE894D4F8B6CED4FE20CF90
:106C700066968FAD6697882309F41ACF482DBE011A
:106C80006B5A7F4FCE0101960E947ABF6EE379E086
:106C900089E39FE00F94C91CBE016F5F7F4F89E3BA
:106CA0009FE00F94721C6BE379E089E39FE00F94FF
:106CB000C91CBE016B5A7F4FF3CE20E030E323287E
:106CC0002428252811F420E030E200E072CF482D7E
:106CD000BE016F5B7F4FCE0101960E947ABF40E0FC
:106CE00050E260E070E0C3010E94C2E0D4FE97C0B1
:106CF000A114B10409F028C1AE96EFADAE97E150F2
:106D0000E63120F5F0E08827E757F94C8F4F0D94D6
:106D10000E4E9C37A636A636A636A6369C37A63625
:106D2000A636A636A636A636A636A636A137993793
:106D3000A636A636A6369F3690379337963765E245
:106D40007AE0CE018B5A9F4F0F944D4630E020E001
:106D500043E050E060E4CE0101960E947872D301D6
:106D60001296ED91FC91608171814FE350E0CE016C
:106D700001960F947F52A114B10469F061EA75E0A5
:106D8000CE0101960F9459524FE350E0B501CE0168
:106D900001960F947F5261EA75E0CE0101960F943F
:106DA00059524FE350E06AEF78E0CE0101960F941C
:106DB0005D4666EE78E089E39FE00F94C91CBE0152
:106DC0006F5F7F4F89E39FE00F94721C63EE78E062
:106DD00089E39FE00F94C91CBE016B5A7F4F89E382
:106DE0009FE00F94721C89E39FE00F94CA1B0E94DE
:106DF000E4AB882309F40ECF8091F91081110ACFFA
:106E0000482DBE016B5A7F4FCE0101960E947ABF7A
:106E100040E050E160E070E0C3010E94C2E0D6FEB5
:106E20007CC040E051E060E070E0C3010E9414E1EA
:106E3000672B682B692B09F495C065ED79E0CE01CD
:106E40008B5A9F4F0F944D4630E020E043E050E0D6
:106E500060E4CE0101960E947872D3011296ED9102
:106E6000FC91608171814FE350E0CE0101960F9457
:106E70007F52A114B10469F061EA75E0CE01019678
:106E80000F9459524FE350E0B501CE0101960F9493
:106E90007F5261EA75E0CE0101960F9459524FE39B
:106EA00050E062E279E0CE0101960F945D466DED0F
:106EB00078E089E39FE00F94C91CBE016F5F7F4FAC
:106EC00089E39FE00F94721C6AED78E089E39FE00C
:106ED0000F94C91CBE016B5A7F4F89E39FE00F944A
:106EE000721C89E39FE00F94CA1B0E94E4AB8823C5
:106EF00009F490CE8091F91081118CCE482DBE01FD
:106F00006B5A7F4FCE0101960E947ABF40E050E459
:106F100060E070E0C3010E94C2E081E090E081CEB9
:106F20006FE27AE00ECF69E37AE00BCF63E47AE0B8
:106F300008CF6DEF79E005CFF3018285853009F048
:106F400005CF63EF79E0FDCE00E020E030E340E1E3
:106F500050E0BE016B5A7F4FCE0183599F4F0E9474
:106F60008E24F4CE40E056E060E070E0C3010E9461
:106F700014E1611576408105910519F469EE79E017
:106F80005ECF6BEC79E05BCF6F927F928F92AF9286
:106F9000BF92CF92DF92EF92FF920F931F93CF9306
:106FA000DF9300D000D01F921F92CDB7DEB73C0117
:106FB0006A017B01590140FF03C0E894C0F8D3F88F
:106FC000D3FC0DC00E941B766639710581059105C1
:106FD00030F08091FE109091FF10059729F5B701D0
:106FE000A6014427507766277727C3010E94EBE06C
:106FF00069EC78E089E39FE00F94C91C8FEF9FEF65
:1070000028960FB6F894DEBF0FBECDBFDF91CF91AB
:107010001F910F91FF90EF90DF90CF90BF90AF90B6
:107020008F907F906F90089519821A821B821C8224
:107030001D821E821F8218868A81807F8A8340E09B
:1070400050E3B301CE0101960E94B62140E050E723
:1070500060E070E0C3010E9414E1C62AD72AE82A42
:10706000F92A8824839409811A812B813C814D81DE
:107070005E816F817885C3010E946134C1CF8F9298
:107080009F92AF92BF92CF92DF92EF92FF920F93B7
:107090001F93CF93DF93CDB7DEB760970FB6F89409
:1070A000DEBF0FBECDBF8C017B0140E050E860E049
:1070B00070E00E9414E1672B682B692B09F0B5C0C2
:1070C00062E070E0C8010E9418E06C0119861A861F
:1070D0001B861C861D861E861F86188A8A85807FD1
:1070E0008A87D7FCA2C040E050E2B801CE010996E1
:1070F0000E94B62163E070E0C8010E9418E0AC0174
:107100001816190614F04FE350E081E0C816D104B8
:1071100029F4EF2CFF0CFF08FF2404C082E0C816FE
:10712000D104D4F32FEF30E0D7010F94254E9A010C
:10713000550F440B550B0F94A54D49016901C8012A
:107140000E948EE2E82EF12C60E0CE0109960E94AA
:10715000792288169906F9F4CD2841F082E0E816E4
:10716000F10419F185E0E816F104F9F081E090E00E
:1071700060960FB6F894DEBF0FBECDBFDF91CF9102
:107180001F910F91FF90EF90DF90CF90BF90AF9045
:107190009F908F900895CD2899F186E0E816F1042C
:1071A00041F081E0E816F10421F061E0C8010E949D
:1071B0006FE2B401CE0109960E94452240E050E200
:1071C000B801CE0109960E94A32082E0E816F104DE
:1071D00021F085E0E816F10449F430E020E040E0D9
:1071E00050E160E070E0C8010E94C43730E020E068
:1071F00040E050E260E070E0C8010E94C437B6CFC2
:1072000085E0E816F10409F4B1CF82E0E816F10454
:1072100009F4ACCF62E0C8010E946FE230E020E0E8
:1072200040E050E160E070E0E7CF90E080E0A0CF88
:10723000CF93DF93EC0140E050E360E070E00E9408
:1072400014E1AB01BC014115510561057105A1F0C7
:107250008091FE109091FF10069771F430E020E0CD
:10726000CE010E94C43740E050E360E070E0CE0100
:10727000DF91CF910C94C2E0DF91CF910895EF920E
:10728000FF920F931F93CF93DF9300D000D0CDB721
:10729000DEB78091640E9091650E892B09F46CC065
:1072A00087E70E943BAD8091640E9091650EDC01F2
:1072B000ED91FC910088F189E02D70E060E0199576
:1072C00010E000E08091640E9091650EDC01ED917C
:1072D000FC9111971C962D913C910217130740F4D5
:1072E0000190F081E02D60E019950F5F1F4FEACF0C
:1072F0000088F189E02D70E060E019950FE114E05D
:1073000083E2E82E84E0F82E8091640E9091650E61
:10731000F80161918F01DC01ED91FC910190F08108
:10732000E02D1995E016F10679F78091640E9091A1
:10733000650EDC01ED91FC910488F589E02D19952D
:107340006FE479E0CE0101960F946A19CE0101969F
:107350000E94E9C8CE0101960F942B1987E090E0B6
:107360000E9457B087E090E00E9461B064EF7AE13C
:1073700088E89EE00F94C91C1092840E1092830E30
:1073800080E090E190937F0E80937E0E84E890E001
:107390009093860E8093850E81E08093800E80E02E
:1073A00090E29093820E8093810E82E78093870E05
:1073B00082E79EE00E9447DA82E79EE00E94ADDA13
:1073C00088EC90E026960FB6F894DEBF0FBECDBFD6
:1073D000DF91CF911F910F91FF90EF900895FF9251
:1073E0000F931F93CF93DF9300D000D0CDB7DEB7BC
:1073F0008C01BC01CE0101960F946119BE016F5F33
:107400007F4F89E39FE00F94BB1C89E39FE00F94BB
:10741000CA1BCE0101960F942B196FE17BE1CE01BF
:1074200001960F943319BE016F5F7F4FC8010F940F
:107430009917F82ECE0101960F942B19FF2069F0B1
:10744000B801CE0101960F946119CE0101960E94F8
:10745000E9C8CE0101960F942B1926960FB6F89421
:10746000DEBF0FBECDBFDF91CF911F910F91FF9077
:1074700008958F929F92BF92CF92DF92EF92FF92E8
:107480000F931F93CF93DF93CDB7DEB7AE970FB6B1
:10749000F894DEBF0FBECDBF8091270A9091280AD5
:1074A000892B09F43CC68091FA10811138C680916D
:1074B000FA108F5F8093FA106EEC78E188E89EE016
:1074C0000F94C91C88E89EE00F94CA1B0091270AFC
:1074D0001091280A63EA75E0C8010E94C6AB909338
:1074E00001118093001169EA75E0C8010E94C6ABE2
:1074F0009093320A8093310A6AE479E0C8010E94CD
:10750000C6AB9093FD108093FC1060EB75E0C80152
:107510000E94C6AB9093250A8093240A009739F104
:10752000DC011696ED91FC91309709F120852F70C2
:107530002530E9F46AEB78E188E89EE00F94C91CF5
:107540008091240A9091250A0E94E1AC8093230A3D
:10755000682F88E89EE00E9450AC88E89EE00F9477
:10756000CA1BE091240AF091250A868197819093A5
:10757000220A8093210A0E94501D65EB75E08091DC
:10758000270A9091280A0E94C6AB9093AD09809378
:10759000AC09009709F4B0C00E94E1AC082F10E0DC
:1075A0000115110509F4A8C0000F111F000F111FCC
:1075B0008091AA099091AB09892B09F08EC07801BE
:1075C000013811051CF020E8E22EF12CC7010F94C0
:1075D0000B449093AB098093AA09E092A9091092F9
:1075E000EE101092ED101092200A10921F0A1092C5
:1075F000EC101092F0101092EF10C70101960F944A
:107600000B449093F2108093F1109093EB108093C1
:10761000EA108E0D9F1D9093E5108093E4100E9458
:10762000ACBE6093E6107093E7108093E8109093DF
:10763000E91090E080E0E091F110F091F210E80F95
:10764000F91F10820196E816F906ACF782E090E087
:107650009093EE108093ED1080911F0A9091200A74
:10766000009741F061E00E9431BC60E080911F0A08
:107670000E9403BC80E98093C9001092C800109258
:10768000CD0083E08093CC008EE08093CA00F0921E
:107690001C02E0921B022091F1103091F2108091B7
:1076A0001B0290911C02820F931F9093E510809310
:1076B000E410232B09F45DC06AE478E189E39FE0DC
:1076C0000F94C91CB70189E39FE00E946CB08CEE57
:1076D0009DED9093E3108093E21060EA78E188E8F2
:1076E0009EE00F94C91CB80188E89EE00E9457AC48
:1076F00088E89EE00F94CA1B6BEB75E08091270A27
:107700009091280A0E94C6AB8C01009709F46BC0C7
:107710000E94E1AC882309F466C06FEF680FC801CE
:107720000E943EACFC01E184F2849091E110992327
:1077300059F0809170008E7F809370001092E1105C
:10774000109219021092180282E18093170291118F
:107750000F94B036C7010F94D83601E010E0E01660
:10776000F10674F060E0C8010F940C370F5F1F4FF3
:10777000F6CF63E378E189E39FE00F94ED1CA7CF98
:1077800065E278E189E39FE00F94C91C0E941B76B3
:10779000AB01BC0189E39FE00E944DAC89E39FE00F
:1077A0000F94CA1B64E878E188E89EE00F94C91C36
:1077B000B70188E89EE00E9457AC88E89EE00F94ED
:1077C000CA1B6EE778E189E39FE00F94C91C0E9411
:1077D0001B76AB01BC0189E39FE00E944DAC89E3BD
:1077E0009FE00F94CA1B0091270A1091280A6FEBA3
:1077F00075E0C8010E94C6AB90932B0A80932A0AB9
:1078000066EC75E0C8010E94C6AB909303118093AB
:107810000211892B09F448C080910411811144C0E0
:107820008091F5109091F610892B09F0D8C16FEF77
:1078300077E189E39FE00F94C91C89E39FE00F94EF
:10784000CA1B8FE090E00F940B448C0188E1D801B3
:1078500011968C93119712961C9212971C921E9659
:107860001C921E921D970E9459B81093F610009317
:10787000F510012B09F08CC060EF77E182E99EE002
:107880000F94C91C82E99EE00F94CA1B80E08170AE
:107890008093041180910411882331F06EE678E121
:1078A00088E89EE00F94C91C1092F8101092F7100F
:1078B000E0910011F0910111309709F4BFC2C68028
:1078C000D78000910011109101110115110509F4E3
:1078D000AEC2C114D10409F4AAC2F60180858F702A
:1078E000853099F7C6010E94E1AC823070F3A8019F
:1078F000B601CE0101960E94AAE3CE0101960E9434
:10790000FBDE8823E1F18C859D85009709F406C292
:10791000DC01ED91FC910284F385E02D1995892B12
:1079200049F08C859D85DC01ED91FC910084F18509
:10793000E02D19958C859D85DC01ED91FC910680EB
:10794000F781E02D1995892BD1F0CE0101960E9487
:107950008EE2882341F040E050E160E070E0CE012B
:1079600001960E94EBE08F819885892B41F040E0E1
:1079700050E260E070E0CE0101960E94EBE0D6019B
:107980001296CD90DC90CE0101960E9477E399CFBC
:107990000E9459B88091F5109091F6100E9491675D
:1079A000882309F489C061ED77E188E89EE00F94AF
:1079B000ED1C8091F5109091F6100E948367E09184
:1079C000F510F091F61081E080838091F510909190
:1079D000F6100F947F376DEB77E1811102C068EAF2
:1079E00077E189E39FE00F94ED1C80910211909163
:1079F0000311892B09F44ACF8091F3109091F41070
:107A0000892B09F0DEC083E190E00F940B448C01D8
:107A10008091F5109091F61027ED31E0F801328B4E
:107A2000218B968385831482108289E0818381E093
:107A3000828383831093F4100093F3100E94ACBEF2
:107A40006B017C01F0E1CF0EF7E2DF1EE11CF11CBF
:107A5000D8011596ED91FC9116978FEF83871486C8
:107A6000138214821582168217821086118612865E
:107A700014961C92BB24B394BE01605E7F4FF80144
:107A8000858196810F94593818160CF095C00E9484
:107A9000ACBE6C157D058E059F0508F08DC0DE011E
:107AA000909698E080E0915019F1ED91E827F0E090
:107AB000E15FFE4C8491F7CF0E94BD6A8091F51082
:107AC0009091F6100E949167882359F06BE877E156
:107AD00088E89EE00F94C91C88E89EE00F94CA1BBA
:107AE00084CF6FE677E182E99EE00F94ED1CCECE65
:107AF0009FA19813C1CFD8018C91811138C01596E0
:107B00008D919C910F947F37BE01605E7F4FF8018D
:107B1000858196810F94603740E064EBD80115961B
:107B20008D919C910F943A37F80185809680C4011D
:107B30000E94A068C4010E94666767E88FE79CE026
:107B40000E94FF5D60E88FE79CE00E94FF5D0E945D
:107B500076BEC4010E94A068982ED80115968D911A
:107B60009C910F947F3795FC02C0F801B082AE0162
:107B70004F5F5F4FBE01605E7F4FC8010F94C037FB
:107B8000D80111969C9088A1803109F4CAC2BE0127
:107B9000605E7F4FC8010F942F38891510F5F801EA
:107BA0008181D80111968C93119714968C9114971A
:107BB0008F5F14968C9360CFE091F310F091F410E6
:107BC0001282E0910211F0910311E680F7809FE7A5
:107BD000D92E8091021190910311892B71F481E0CB
:107BE00056CE88A1803111F48CE0DBCFBE01605EFF
:107BF0007F4FC8010F942F38D4CFE114F10479F3EB
:107C0000BE01605E7F4FF701808191810E94B07755
:107C1000882329F368E577E189E39FE00F94C91C85
:107C2000D7016D917C9189E39FE00F94721C89E3E9
:107C30009FE00F94CA1B0091F3101091F410AE0155
:107C40004F5F5F4FBE01605E7F4FC8010F941538D4
:107C5000882309F45EC088A1803109F45AC0DD820E
:107C6000F801858196810F947F37BE01605E7F4F5A
:107C7000D80115968D919C910F94603740E06EE489
:107C8000F801858196810F943A3740E06B81D801E5
:107C900015968D919C910F943A3740E06C81F801D4
:107CA000858196810F943A3788A1803141F040E078
:107CB0006D81D80115968D919C910F943A37F801FA
:107CC000858196810F947F37BE01605E7F4FD8011A
:107CD00015968D919C910F946037F801408168E46E
:107CE000858196810F943A3764E170E080E090E0FE
:107CF0000E9479BED8018C91882331F06AE070E04F
:107D000080E090E00E9479BEF801858196810F9411
:107D10007F37D7011296ED90FC905BCF70E060E06A
:107D2000CE0101960E9418E08C01912C812C97FFC6
:107D300006C011950195110988248394912CCE01D8
:107D400001960E948EE2E82EF12C8B85853091F011
:107D5000863009F014CEB02E61E0802F0E9431BC35
:107D600061E0892809F441C0EA94EF2809F041C094
:107D700060E03FC0EF2829F462E0CE0101960E9446
:107D80006FE240E050E160E070E0CE0101960E94B9
:107D9000EBE08F819885892B41F040E050E260E074
:107DA00070E0CE0101960E94EBE061E0802F0E941E
:107DB00031BC60E0802F0E9403BC66E678E189E375
:107DC0009FE00F94C91CB80189E39FE00E9457AC63
:107DD00061E678E189E39FE00F94C91C6FE578E1E3
:107DE00089E39FE00F94C91CCACDEA94EF2809F0FB
:107DF000BFCFE62EF12C8B2D0E9403BC6AE578E103
:107E000089E39FE00F94C91CB80189E39FE00E94B9
:107E100057AC68E578E189E39FE00F94C91CB7018E
:107E200089E39FE00E9457AC66E578E1D9CFF8017D
:107E3000868197819093F8108093F71089E39FE0F3
:107E40000F94CA1B64E477E188E89EE00F94C91C94
:107E500088E89EE00F94CA1BE091FC10F091FD10A1
:107E6000309709F4A8C08091FA108F5F8093FA10C0
:107E7000E680F780E114F10409F498C0D701189660
:107E80008C918F70863009F07EC0F9A6E8A670E06C
:107E900060E0CE0188960F94B9018DA59EA5892B2F
:107EA00009F471C08091270A9091280A892B09F45E
:107EB0006AC0C8A4D9A4C114D104B9F1F60180855F
:107EC0008F70863091F5D9A2C8A270E060E0CE0133
:107ED00080960F94B901EDA1FEA110821182128249
:107EE000138269EC75E0C6010E94C6ABFC01892BC8
:107EF000E1F090859F7095509230B8F4068117811B
:107F00000115110591F01A830983B601CE0101967E
:107F10000F94B901EE81FF811082118212821382C7
:107F2000D80112960D911C91EBCF6FE377E189E3B5
:107F30009FE00F94C91C6BA589E39FE00E9450ACA1
:107F40006DE377E189E39FE00F94C91C6AA589E39B
:107F50009FE00E9450AC89E39FE00F94CA1BEDA5FF
:107F6000FEA510821182128213828AA5843078F4D1
:107F7000823098F060E08BA50E9431BCEDA5FEA593
:107F80008181807F8183F701E280F38073CF803429
:107F900059F0823421F08032B1F762E0ECCF60E03A
:107FA0008BA50E9431BCEFCF62E0FACF8091FA102E
:107FB00081508093FA1060E377E188E89EE00F94A7
:107FC000C91C68E277E188E89EE00F94C91C81E053
:107FD0002091001130910111232B09F480E00E94BF
:107FE000331A6FE177E188E89EE00F94C91C81E0C5
:107FF0002091FC103091FD10232B09F480E00E94A9
:10800000331A60E177E188E89EE00F94C91C65E0CF
:1080100077E188E89EE00F94C91C81E020912A0A4C
:1080200030912B0A232B09F480E00E94331A6EEF63
:1080300076E188E89EE00F94C91C81E02091210A36
:108040003091220A232B09F480E00E94331A65EF55
:1080500076E188E89EE00F94C91C81E0209102112E
:1080600030910311232B09F480E00E94331A6CEE47
:1080700076E188E89EE00F94C91C80912E0A0E9448
:10808000331A88E89EE00F94CA1B67EE76E188E811
:108090009EE00F94C91C0E941B76AB01BC0188E8CE
:1080A0009EE00E944DAC88E89EE00F94CA1B81E0E0
:1080B0008093260A85E59EE00F949A2F882351F03D
:1080C00085E59EE00F94BC2F84E090E09093FF1034
:1080D0008093FE108091FE109091FF10079731F46D
:1080E00084E090E09093FF108093FE108091FA104E
:1080F00081508093FA108091260AAE960FB6F894BC
:10810000DEBF0FBECDBFDF91CF911F910F91FF90CA
:10811000EF90DF90CF90BF909F908F90089580E078
:10812000ECCFFCE0F91508F43ACD5ECD4F925F92AA
:108130006F927F928F929F92AF92BF92CF92DF9277
:10814000EF92FF920F931F93CF93DF93CDB7DEB7DC
:10815000C157D1090FB6F894DEBF0FBECDBF8C0159
:108160004B01F42E642F89E39FE00E9450AC63EC36
:108170007EE089E39FE00F94C91CB401CE01019613
:108180005C010F946119B50189E39FE00F94BB1C5A
:1081900089E39FE00F94CA1BC5010F942B1992E04D
:1081A000F91280C161EC7EE0C5010F943319D4014E
:1081B00014962D913C9115978D819E812817390732
:1081C00011F58D919C9169817A81009759F0611523
:1081D000710509F064C1232B09F4A3C1DC018C9162
:1081E00090E00DC06115710509F49BC1232B09F4C2
:1081F00098C1FB01808190E0919581959109FF24C0
:10820000F394892B09F0F12CC5010F942B19FF2051
:1082100009F4D3C240E06DE271E0C8010E94EED7DC
:1082200080902F0A9090300A6AEB7EE0CE0184594C
:108230009F4F0F94331963EB7EE0CE018A599F4F15
:108240000F943319CE01865A9F4F0F94E035A096B4
:10825000FFACA0976F96EFAC6F976E96DFAC6E9702
:108260006D96CFAC6D976FE479E0CE0181960F9457
:108270006A19BE016F5D7F4FC5010F9461196C2DA6
:10828000C5010F947C186DEC75E00F94AD186D2D41
:108290000F947C186DEC75E00F94AD186E2D0F9453
:1082A0007C186DEC75E00F94AD186F2D0F947C1851
:1082B000BC01CE01805A9F4F0F946119C5010F94E4
:1082C0002B19CE0181960F942B196EEA7EE0CE0118
:1082D0008C5A9F4F0F9433196E01EEE4CE0ED11CD1
:1082E0006FE479E0C6010F946A1994E6E92E9EE0E6
:1082F000F92E2AE6622E2EE0722E2601D70118965C
:108300006C9170E084E0759567958A95E1F7C501F9
:108310000E940FAD4D815E8169817A81C2010F9407
:108320002A18C5010F942B19F70160856F7070E052
:10833000C5010E940FAD4D815E8169817A81C201C4
:108340000F942A18C5010F942B19FFEFEF1AFF0A9B
:108350006E147F0499F668EA7EE0CE01885B9F4F39
:108360000F94331966E97EE0CE0181960F9433199C
:10837000BE016F5D7F4FCE01805C9F4F0F946119EE
:108380002696EEACFFAC269788E1E80EF11CB7010B
:10839000CE01805C9F4F0F9402188111C5C0CE01A1
:1083A000805C9F4F0F946A18BE01685B7F4FCE01BF
:1083B000805C9F4F0F94C718B6010F94C718BE0179
:1083C0006C5A7F4F0F94C718BE01605A7F4F0F94AD
:1083D000C718BE016A597F4F0F94C7187C014AE045
:1083E000B50180E590E00F94C046F50101900020B2
:1083F000E9F73197AF014A195B09B501C7010F943D
:108400002A18811103C0C7010F946A18BE0164596C
:108410007F4FC7010F94C718B4010F94AD18BC016A
:10842000C8010F94BB1CC8010F94CA1BCE01805C0D
:108430009F4F0F942B19CE0181960F942B19CE01CB
:10844000885B9F4F0F942B19C2010F942B19CE01FB
:108450008C5A9F4F0F942B19CE01805A9F4F0F9427
:108460002B19CE018A599F4F0F942B19CE01845995
:108470009F4F0F942B19C8010F94CA1B64E670E03C
:1084800080E090E00E9479BED801ED91FC910488D3
:10849000F589E02DC801199501E010E0EDC00F94B9
:1084A0006F52ADCEB1E0FB1220C266E77EE0C5019F
:1084B0000F943319B501C4010F949917582EC501B3
:1084C0000F942B19552009F4D8C1EE2009F473C17B
:1084D00066E070E0C4010E94EEB94AE0B801CE0146
:1084E000885B9F4F0F94471B4091001150910111E1
:1084F000F40160817181CE0181960E94DAE2CE01A1
:1085000081960E94FBDE811122C000E911E0CE01BC
:1085100081960E9477E3CE01885B9F4F0F942B19C1
:10852000ABC0FF24F39470CE22962EAD3FAD2297C0
:1085300026968EAD9FAD26976DE77EE0820F931F46
:108540000F944D462696FFAEEEAE26972DCF2A9677
:108550006EAD7FAD2A97CE0181960E942AB4892BF9
:10856000A1F224961CAE1DAE1EAE1FAE2497289617
:108570001CAE1DAE1EAE1FAE289722968FAD229761
:10858000807F22968FAF229740E050E3BE016F5D5F
:108590007F4FCE01805C9F4F0E94B62100E020E01B
:1085A00030E340E250E0B501CE01805C9F4F0E9475
:1085B0008E24BC01C6010F94051908EC10E1A7CF69
:1085C000EE2009F4F8C066E070E0C4010E94EEB944
:1085D0004091001150910111D4016D917C91CE0117
:1085E00081960E94DAE2CE0181960E94FBDE00E9CC
:1085F00011E08823E9F18BA5873061F4CE018196E3
:108600000E94B3E461E0892B09F462E0CE01819617
:108610000E946FE224961CAE1DAE1EAE1FAE2497C4
:1086200028961CAE1DAE1EAE1FAE289722968FADAB
:108630002297807F22968FAF229740E050E3BE01C1
:108640006F5D7F4FCE01805C9F4F0E94B62100E09E
:1086500020E030E340E250E0B501CE01805C9F4F66
:108660000E948E24BC01C6010F94051908EC10E18C
:10867000CE0181960E9477E3C801CF58DF4F0FB635
:10868000F894DEBF0FBECDBFDF91CF911F910F9148
:10869000FF90EF90DF90CF90BF90AF909F908F9022
:1086A0007F906F905F904F900895F4016081718189
:1086B0000E94C6AB7C01892B09F0C5C004E911E01A
:1086C000DBCFEE2009F477C069E070E0C4010E94BE
:1086D000EEB94AE0B801C5010F94471B41E050E0F4
:1086E0006CEB76E0C4010F942A184D815E8169819C
:1086F0007A81C4010F942A1869E57EE089E39FE03E
:108700000F94C91CB401CE0181960F946119BE016A
:108710006F5D7F4F89E39FE00F94BB1C89E39FE06F
:108720000F94CA1BCE0181960F942B1961E57EE050
:10873000CE0181960F943319F401848195812DA186
:108740003EA182179307E1F4892B91F1E080F1803B
:1087500069A07AA0D7018D917D01882349F1082E67
:10876000000C990B0F94F4516C01F30181913F01BE
:10877000082E000C990B0F94F451C816D90651F32A
:10878000CE0181960F942B19552031F041E068EC11
:1087900070E0C8010E94EED7D4018D919C910F9496
:1087A000CD22009711F484E991E08C01C501B6CE89
:1087B00055245394E5CF01E982CF6FE67EE0C501F1
:1087C0000F943319B501C4010F949917F82EC50100
:1087D0000F942B19F110F4CE69E67EE0C5010F94D9
:1087E0003319B501C4010F949917F82EC5010F94E0
:1087F0002B19FF2009F479C0EE20E9F265E070E062
:10880000C4010E94EEB96DEC75E0C4010F94B41779
:10881000882339F0E0900011F0900111E114F10487
:1088200091F46FE479E0C4010F94B417811107C08B
:108830008091001190910111009709F036CFE090DE
:10884000270AF090280A40E068EC70E2C8010E9414
:10885000EED7C8010F94CA1B1C821B8285EC92E0E4
:108860009A8389831E830D838FEF9FEF98878F8371
:10887000B701C5010E94AAB201CE6FE57EE0C50135
:108880000F943319B501C4010F949917F82EC5013F
:108890000F942B19F11015CF64E47EE0C5010F94FD
:1088A0003319B501C4010F949917182FC5010F94FE
:1088B0002B1900E0112309F4DFCE80E00E944DB0B7
:1088C0006CE17EE088E89EE00F94C91C88E89EE099
:1088D0000F94CA1B6FE479E0C5010F946A19C501B2
:1088E0000E94E9C8C5010F942B1900E0D6CD8F92E4
:1088F0009F92AF92BF92CF92DF92EF92FF920F932F
:108900001F93CF93DF93CDB7DEB7CF55D1090FB605
:10891000F894DEBF0FBECDBF8C016B0161157105F0
:1089200019F04115510579F562E37FE089E39FE095
:108930000F94C91C69E27FE089E39FE00F94C91C92
:10894000B80189E39FE00F94721C67E27FE089E33E
:108950009FE00F94C91C89E39FE00F94CA1BC15A82
:10896000DF4F0FB6F894DEBF0FBECDBFDF91CF91C2
:108970001F910F91FF90EF90DF90CF90BF90AF903D
:108980009F908F900895460F571FDA011C920E9406
:108990001B764B0161E27FE089E39FE00F94C91CE5
:1089A000B40189E39FE00E9457AC6EE17FE089E368
:1089B0009FE00F94C91CB80189E39FE00F94721CDB
:1089C0006BE17FE089E39FE00F94C91CBAE38B164B
:1089D000B1E09B064CF46EE07FE082E99EE00F94EC
:1089E000C91C82E99EE0B9CF6CE07FE089E39FE09B
:1089F0000F94C91CB60189E39FE00F94721C6AE0D2
:108A00007FE089E39FE00F94C91C89E39FE00F9406
:108A1000CA1B1A821982FE0133968EE3DF011D9272
:108A20008A95E9F78091FE109091FF10059791F5D6
:108A300063E070E0C8010E945D1E7C01892BD1F5C6
:108A4000E091910CF091920C808180FF88CF61E0E1
:108A500070E0C8010E945D1E892B09F480CF64E29A
:108A600070E0C8010F94AC52892B09F078CF6CEEFE
:108A70007EE089E39FE00F94C91CB80189E39FE081
:108A80000F94721C89E39FE00F94CA1BC8010E94D7
:108A900011BA65CF61E070E0C8010E945D1E7C01E3
:108AA000892B09F465C04FE350E0B801CE0101966F
:108AB0000F949D52A12CBB24B394E00EF11E63EEE3
:108AC0007EE0C7010F944446892B09F45EC064E23E
:108AD00070E0C8010F94AC52892B09F040CFB1105F
:108AE00003C0AA2009F43BCF40910011509101111D
:108AF000B701CE018F5B9F4F0E94DAE2CE018F5B00
:108B00009F4F0E94FBDE182F882359F0B601CE013B
:108B10008F5B9F4F0E942AB411E0181619060CF0C3
:108B200010E0CE018F5B9F4F0E9477E3112309F481
:108B300016CF8981882309F412CF8091FE1090917D
:108B4000FF10059709F40BCF65EC7EE089E39FE009
:108B50000F94C91CBE016F5F7F4F89E39FE00F94A4
:108B6000721C89E39FE00F94CA1BCE0101968FCF40
:108B700062E070E0C8010E945D1E7C01892B09F44F
:108B8000EECEAA24A394B12C98CFF6010190002038
:108B9000E9F73197EC19FD09329708F498CFC8012D
:108BA0000E9411BAB11003C0AA2009F4D8CEC601A0
:108BB0000F94CD22D4CE0F931F93CF93DF93CDB7D5
:108BC000DEB76F970FB6F894DEBF0FBECDBF209112
:108BD000270A3091280A232B09F413C12091FA1097
:108BE000022E000C330B82179307B4F465E07EE08D
:108BF00082E99EE00F94C91C82E99EE00F94CA1B93
:108C000080E06F960FB6F894DEBF0FBECDBFDF9148
:108C1000CF911F910F9108956FEE7DE089E39FE062
:108C20000F94C91C89E39FE00F94CA1B8091AE0981
:108C30008F5F8093AE096AEA7DE088E89EE00F943A
:108C4000C91C88E89EE00F94CA1BE091FC10F091CB
:108C5000FD10309709F18091FA108F5F8093FA1020
:108C6000068117810115110591F0D80118968C9194
:108C70008F70863041F41A83098370E060E0CE0182
:108C800001960F94B901F80102811381EBCF809115
:108C9000FA1081508093FA10E0910011F0910111C7
:108CA0003097A1F10681178101151105C9F1D8018D
:108CB00018968C918F70853029F5C8010E94E1AC1F
:108CC000882301F14091001150910111F801608158
:108CD0007181CE0101960E94DAE2CE0101960E94D6
:108CE000FBDE882359F08C859D85009739F0DC01E7
:108CF000ED91FC910084F185E02D1995CE0101964E
:108D00000E9477E3F80102811381CECF6FED7DE001
:108D100089E39FE00F94C91C89E39FE00F94CA1B6D
:108D20001092F8101092F71067ED7DE089E39FE054
:108D30000F94C91C89E39FE00F94CA1B64E670E09E
:108D400080E090E00E9479BE10922E0A1092260ACE
:108D50006FEB7DE089E39FE00F94C91C0E941B76B6
:108D6000AB01BC0189E39FE00E944DAC8091270AD2
:108D70009091280A009711F00E947CB71092280A5F
:108D80001092270A1092FD101092FC1010920111FF
:108D9000109200111092320A1092310A1092250A94
:108DA0001092240A1092220A1092210A1092300A7C
:108DB00010922F0A1092230A1092AD091092AC095A
:108DC000109203111092021110922B0A10922A0A8B
:108DD0006AEB7DE089E39FE00F94C91C0E941B763B
:108DE000AB01BC0189E39FE00E944DAC89E39FE0A9
:108DF0000F94CA1B10921D0A8091AE098150809376
:108E0000AE0981E0FECE4F925F926F927F928F9279
:108E10009F92AF92BF92CF92DF92EF92FF920F9309
:108E20001F93CF93DF93CDB7DEB7C859D1090FB6E3
:108E3000F894DEBF0FBECDBF8E010F5B1F4FD80170
:108E40001D921C92FE01ED5BFF4F8EE1DF011D9232
:108E50008A95E9F78091640E9091650E892B09F44B
:108E6000CEC10E9450AD882309F4C9C182E70E9497
:108E70003BAD8091640E9091650EDC01ED91FC910B
:108E80000088F189E02D60E270E019954FE150E033
:108E9000B8018091640E9091650E0E9495AD7C01A1
:108EA0008091640E9091650EDC01ED91FC91048837
:108EB000F589E02D1995E114F10409F4A0C1F80138
:108EC000EE0DFF1D10828091710E1F928F93809185
:108ED000700E1F928F9380916F0E1F928F938091CF
:108EE0006E0E1F928F9380916D0E1F928F938091C3
:108EF0006C0E1F928F938FEC95E09F938F931F9230
:108F000080E48F93FE0131966F01FF93EF930F94EE
:108F1000B7526EE07CE188E89EE00F94C91CB8016E
:108F200088E89EE00F94721CB60188E89EE00F94DA
:108F3000721C88E89EE00F94CA1B7E01F1E6EF0EDA
:108F4000F11CD70113961C921E92129788EE93E0A3
:108F5000A0E0B0E0F70184839583A683B78388E01F
:108F6000848788EE93E0968785878DE792E09183EA
:108F70008083108A1786128B018B148A138A80E5EE
:108F800090E0968B858B118E66E27BE189E39FE012
:108F90000F94C91C66E67EE0CE0185589F4F0F9462
:108FA0006119BE0165587F4F89E39FE00F94BB1C98
:108FB00089E39FE00F94CA1BCE0185589F4F0F9401
:108FC0002B196EEF75E0CE0183579F4F0F946A19EE
:108FD0006EEF75E0CE0185589F4F0F946A19BE0160
:108FE00065587F4FCE018B579F4F0F94611966E6EE
:108FF0007EE0CE018B579F4F0F94C718BE01635779
:109000007F4F0F94C718BC01CE018D569F4F0F9410
:109010006119CE018B579F4F0F942B19CE018558A4
:109020009F4F0F942B19CE0183579F4F0F942B19ED
:1090300080E096E0CB57DF4F99838883C558D040B6
:10904000C757DF4F19821882C958D040C557DF4F24
:1090500019821882CB58D040CD56DF4F8881998134
:10906000C359D040C957DF4F99838883C758D04030
:1090700068E07CE189E39FE00F94C91C0E941B76A5
:10908000AB01BC0189E39FE00E944DAC89E39FE006
:109090000F94CA1B64E670E080E090E00E9479BE05
:1090A0008FEE99E3D70150969C938E931F9763E7B9
:1090B00071E08FEC90E00F944E478C010FB6F8945E
:1090C000DEBF0FBECDBF892B09F4F4C083E090E072
:1090D0000F940B44D8011D969C938E931C97FC0112
:1090E000F182E0821282C7010F949A2F882319F02F
:1090F000C7010F94BC2FD70153966D917C91549763
:109100005596AD90BC906115710509F48FC0CE01E4
:1091100085589F4F0F94091DA501BE0165587F4FCB
:10912000C7010F946235181619060CF0C0C0D7019C
:109130005196BC9051975296AC90DF92CF9281E8B5
:109140009BE19F938F931F930F930F94D547DF92CB
:10915000CF928CE79BE19F938F931F930F930F9474
:10916000D547D8011C96ED91FC9181E08283DF9276
:10917000CF9289E79BE19F938F931F930F930F9457
:10918000D547D8011C96ED91FC911282AF92BF9207
:1091900083E49BE19F938F931F930F930F94D54785
:1091A0000FB6F894DEBF0FBECDBFB12C8AE3C82E38
:1091B0008BE1D82E8B2D94E08902F0011124A5E8D3
:1091C000B0E0AC0FBD1FEA0FFB1F808191810097BB
:1091D000A9F12281338121153105C9F33F932F93E2
:1091E0009F938F93DF92CF921F930F930F94D54746
:1091F000B3940FB6F894DEBF0FBECDBFDBCF40E215
:1092000050E060E47CE1C8010F947B4662E27CE1BF
:1092100088E89EE00F94C91CB80188E89EE00F948E
:10922000721C88E89EE00F94CA1B4DCEF70161893D
:109230007289A501C7010F940C3075CF8EE79BE1B1
:109240009F938F931F930F930F94D547D7015896F1
:109250001C921E925797D8011C96ED91FC91C080EC
:10926000D1800F900F900F900F9043E3A42EB12C5C
:10927000D601ED91FC910084F185E02DC601199590
:1092800041975CF4B1E0AB1AB10839F064E170E0E9
:1092900080E090E00E9479BEEBCFD601ED91FC9189
:1092A0000084F185E02DC6011995419734F4C80179
:1092B0000F94412510E000E05AC06FE479E0CE0140
:1092C00083579F4F0F946A19912CA12CD601ED91D1
:1092D000FC910688F789E02DC60119958823E1F1F4
:1092E000BDE0AB1201C0A92CD601ED91FC9106881E
:1092F000F789E02DC60119958111BBC0D601ED910A
:10930000FC910084F185E02DC6011995892B09F4A3
:10931000C2C0D601ED91FC910284F385E02DC60117
:109320001995B82EBAE08B1709F4B7C0EDE08E1787
:1093300009F4B3C0FFEF8F1709F4ADC0682FCE0159
:1093400083579F4F0F9456189A2CAB2CBFCFBAE07F
:10935000BB12FACFAB12F8CFCC24C394D12CCE01E0
:1093600083579F4F0F942B19CD2809F4A3CFD70112
:109370005796ED90FC906AEF7BE189E39FE00F94B4
:10938000C91CB70189E39FE00E9457AC89E39FE0C5
:109390000F94CA1B64E670E080E090E00E9479BE02
:1093A0000115110509F461C1B8ECEB16F10409F0DF
:1093B0003AC16EEE7BE188E89EE00F94C91C64EF31
:1093C00071E080E090E00E9479BEEF961FAE1EAE85
:1093D000EF97C158DF4F19821882CF57D0408FEFD7
:1093E0009FEFCF57DF4F99838883C158D0408FEAD2
:1093F00092E0ED969FAF8EAFED97CD57DF4F19837B
:109400000883C358D040F89490E080E00E94DB4588
:109410008111CAC062EE7BE182E99EE00F94C91C13
:1094200082E99EE00F94CA1BC8010F94412524EFE6
:10943000E22EFF24F394CE018D569F4F0F942B19EB
:10944000C701C856DF4F0FB6F894DEBF0FBECDBFC1
:10945000DF91CF911F910F91FF90EF90DF90CF9010
:10946000BF90AF909F908F907F906F905F904F9044
:109470000895D601ED91FC910084F185E02DC6019F
:109480001995892B09F03ACF64E670E080E090E00E
:109490000E9479BE29CFBB24BA946EE076E08CE9B5
:1094A0009EE00F94721CBE0163577F4F8CE99EE0D3
:1094B0000F94BB1C8CE99EE00F94CA1B61E37BE117
:1094C000CE0185589F4F0F943319BE0165587F4FC9
:1094D000CE0183579F4F0F949917982ECE01855830
:1094E0009F4F0F942B19992079F1CF56DF4F288188
:1094F0003981C159D04049E050E0BE0163577F4FE8
:10950000CE0185589F4F0F947B19ED968EAD9FAD80
:10951000ED97412C512C3201009719F00F94F6452C
:109520002B014201CE0185589F4F0F942B194114F6
:10953000510429F0D70158965C924E925797B40186
:109540008CE99EE00E946CB0F701878490888114BA
:109550009104D1F0CF56DF4F88819981C159D04015
:10956000892B91F0BE0163577F4FCE0185589F4FE5
:109570000F946119CE0185589F4FF4011995CE01C2
:1095800085589F4F0F942B196FE479E0CE018357D4
:109590009F4F0F94FB18FFEFBF12D9CEC8010F9455
:1095A0004125D12CC12CDBCECE0185589F4F0E9486
:1095B00070B89093280A8093270A7894C8010F9472
:1095C00041258091270A9091280A892BD1F46FE4D4
:1095D00079E0CE0183579F4F0F946A19CE018357CC
:1095E0009F4F0E94E9C8CE0183579F4F0F942B19BC
:1095F0006BEC7BE182E99EE00F94C91CF12CE12C1D
:109600001ACF0E94393A8091260A882329F00E94B5
:10961000AFAF71FF0E94767864EC7BE188E89EE052
:109620000F94C91C08CFE0E3EE16E1E0FE0651F40A
:1096300060EB7BE188E89EE00F94C91CC8010F94A1
:109640004125F9CE68E97BE182E99EE00F94C91CCF
:10965000C8010F944125B70182E99EE00E9457ACF2
:1096600082E99EE00F94CA1BE6CE65E87BE189E3C0
:109670009FE00F94C91CEE24EA94FE2CDCCECF931D
:10968000DF93CDB7DEB72E970FB6F894DEBF0FBECF
:10969000CDBF8091FA10811121C18091FA108F5FA6
:1096A0008093FA1069E279E188E89EE00F94C91C82
:1096B00088E89EE00F94CA1B1092840E1092830ECD
:1096C00080E090E190937F0E80937E0E84E890E09E
:1096D0009093860E8093850E81E08093800E80E0CB
:1096E00090E29093820E8093810E82E78093870EA2
:1096F00082E79EE00E9450DD8B37910509F0C5C0DE
:109700006BE179E189E39FE00F94C91C89E39FE055
:109710000F94CA1B8091270A9091280A892B21F067
:1097200081E090E00E94DB451C821B8285EC92E088
:109730009A83898382E79EE09E838D838FEF9FEFDC
:1097400098878F83CE0101960E9470B89093280A63
:109750008093270A82E79EE00E94ADDA8091270A73
:109760009091280A892B01F56FE079E182E99EE06A
:109770000F94C91C82E99EE00F94CA1B6FE479E044
:10978000CE0109960F946A19CE0109960E94E9C884
:10979000CE0109960F942B198091FA108150809375
:1097A000FA1090E080E019C06CEF78E188E89EE064
:1097B0000F94C91C88E89EE00F94CA1B8091FA1090
:1097C00081508093FA100E94393A8091640E9091F2
:1097D000650E892B59F481E090E02E960FB6F8942F
:1097E000DEBF0FBECDBFDF91CF9108950E9450AD77
:1097F000882389F382E70E943BAD8091640E9091AB
:10980000650EDC01ED91FC910088F189E02D60E6A8
:1098100070E019956091640E7091650E40E0CE0184
:1098200009960F94471BBE01675F7F4F86E69EE057
:109830000F94C917CE0109960F942B198091640ECD
:109840009091650EDC01ED91FC910488F589E02D85
:1098500019956EED78E189E39FE00F94C91C66E6E7
:109860007EE0CE0109960F946119BE01675F7F4FBC
:1098700089E39FE00F94BB1C89E39FE00F94CA1B10
:10988000CE0109960F942B19A6CF82E79EE00E9485
:109890001DDA892BA1F082E79EE00E9447DA6FE48F
:1098A00079E0CE0101960F946A19CE0101960E94CB
:1098B000E9C8CE0101960F942B190E946AC982E76C
:1098C0009EE00E94ADDA6BEE78E188E89EE00F94AE
:1098D000C91C88E89EE00F94CA1B5ECF8FEF9FEFF4
:1098E0007CCF4F925F926F927F928F929F92AF92B6
:1098F000BF92CF92DF92EF92FF920F931F93CF937D
:10990000DF93CDB7DEB7CF52D1400FB6F894DEBFAC
:109910000FBECDBF2091FE103091FF10F90171965E
:10992000E532F10508F041C68827E656F34B8F4F24
:109930000D940E4EEC5BD85BD552D552D552D55214
:10994000345B205BD552D552D552D552D552D55223
:10995000D552D552D552BF4C35543C5415565C5651
:109960001B5A185BD552D552D552D552D5524F5BA2
:10997000615B9A5B775BD552D552D552845B8091FF
:10998000260A0F94FC35029709F40FC686E195E08C
:10999000CC5DDE4F99838883C452D140CA5DDE4FCF
:1099A000188219821A821B82C652D140C25EDE4FD3
:1099B00099838883CE51D140C05EDE4F18821982D0
:1099C0001A821B82C052D140C85EDE4F99838883C1
:1099D000C851D140C65EDE4F188219821A821B829E
:1099E000CA51D140CE5EDE4F99838883C251D140A7
:1099F000CC5EDE4F188219821A821B82C451D1407C
:109A000069E670E188E89EE00F94C91C88E89EE052
:109A10000F94CA1B8091640E9091650E8E010F57B2
:109A20001F4F892B09F45CC00E9450AD882309F4B4
:109A300057C082E70E943BAD8091640E9091650E05
:109A4000DC01ED91FC910088F189E02D60E170E08E
:109A50001995BE016F5F7F4F8091640E9091650EE6
:109A60000E94F1AC89819A81AB81BC81CA5DDE4FD5
:109A700088839983AA83BB83C652D1408091640EA8
:109A80009091650EDC01ED91FC910488F589E02D43
:109A90001995CA5DDE4F8881C652D140882301F1F5
:109AA0008F3FA9F4C95DDE4F8881C752D1408F3FF7
:109AB00071F4C85DDE4F8881C852D1408F3F39F4C0
:109AC000C75DDE4F8881C952D1408F3F49F00E9467
:109AD000AFAF72FFA1C18091180A833008F09CC11A
:109AE0006DE570E188E89EE00F94C91C0FB6F8940C
:109AF000A89580916000886180936000109260005A
:109B00000FBE80910D0A81112AC01092F5091092A2
:109B1000F40988EE93E0A0E0B0E08093F60990931A
:109B2000F709A093F809B093F9098CEE94E09093AB
:109B3000F3098093F20986E195E09093010A8093FE
:109B4000000A1092020A1092030A1092040A10925C
:109B5000050A88E080930A0A81E080930D0A8FEA63
:109B600099E09093170A8093160A0F942D29F12CEF
:109B7000E12C882309F4AEC080E591E00E9418B87A
:109B800046E050E06CE67EE089E090E00F94E2264B
:109B900086E195E09A8389831B821C821D821E8246
:109BA000CE0103960F9417290F942C298091160A41
:109BB0009091170AFC0112A213A214A215A2DC01B3
:109BC00016A217A210A611A612A613A614A615A6D1
:109BD00040EE5EE260E070E046AB57AB60AF71AF65
:109BE00040EA5FE060E070E042AF53AF64AF75AF52
:109BF000189626E0FD01322F11923A95E9F7AC0153
:109C0000425F5F4F34E1FA0111923A95E9F7ECE6D1
:109C1000FEE001900D922A95E1F7FC01EE5BFF4F0B
:109C200010820F941D337C01019709F053C080E529
:109C300091E00E9418B86091160A7091170A625F4D
:109C40007F4FCE0101960F94091DCE0103960F940C
:109C500017296091160A7091170A6A5E7F4FCE012C
:109C600001960F94091DCE0103960F94252960914A
:109C7000160A7091170A6E5E7F4FCE0101960F94FF
:109C8000091DCE0103960F941E290F942C29609173
:109C9000160A7091170A625E7F4FCE0101960F94EB
:109CA000091D8B819C81AD81BE8180937B0C90933B
:109CB0007C0CA0937D0CB0937E0C0E9461BD7F73E1
:109CC0008091010290910202682779277093020225
:109CD0006093010288E199E20FB6F894A895809309
:109CE00060000FBE90936000A895EF2809F4EAC2C7
:109CF00064EB7FE088E89EE00F94C91CCE010196DA
:109D00000F94E0358B819C81AD81BE81CA5DDE4FB1
:109D100088839983AA83BB83C652D14056E1E52E3E
:109D200055E0F52EFA82E982CE0101960E948775F0
:109D300088E89EE00F94CA1BCE018C5D9E4F0E9466
:109D40005BAE80917B0C90917C0CA0917D0CB091CE
:109D50007E0C8B839C83AD83BE83C05EDE4F888385
:109D60009983AA83BB83C052D140CE01825E9E4FAD
:109D70000E9405AFFA82E9821B821C821D821E822C
:109D800080E591E00E9418B844E050E0BE016D5FAC
:109D90007F4F81E090E00F941E260F942C298B8139
:109DA0009C81AD81BE81C65EDE4F88839983AA8384
:109DB000BB83CA51D140CE01885E9E4F0E945AAFEC
:109DC000FA82E9821B821C821D821E8280E591E05C
:109DD0000E9418B844E050E0BE016D5F7F4F85E0FF
:109DE00090E00F941E260F942C298B819C81AD81CD
:109DF000BE81CC5EDE4F88839983AA83BB83C45126
:109E0000D140CE018E5E9E4F0E94B0AE81E00E9496
:109E100044B01092180AD7C167E470E188E89EE068
:109E20000F94C91C86E195E09A838983CA5DDE4F51
:109E300088819981AA81BB81C652D1408B839C8342
:109E4000AD83BE83CE0101960E9487758091640E1A
:109E50009091650E892B09F420C20E9450AD882391
:109E600009F41BC282E70E943BAD8091640E909181
:109E7000650EDC01ED91FC910088F189E02D64E133
:109E800070E01995BE016F5F7F4F8091640E9091D5
:109E9000650E0E94F1AC89819A81AB81BC81C05E64
:109EA000DE4F88839983AA83BB83C052D1408091BF
:109EB000640E9091650EDC01ED91FC910488F589AA
:109EC000E02D1995C05EDE4F8881C052D1408823B5
:109ED00009F4E3C18F3FB1F4CF5DDE4F8881C152F9
:109EE000D1408F3F79F4CE5DDE4F8881C252D140A0
:109EF0008F3F41F4CD5DDE4F8881C352D1408F3F0B
:109F000009F4CBC161E470E188E89EE00F94C91CBC
:109F100086E195E09A838983C05EDE4F88819981CE
:109F2000AA81BB81C052D1408B839C83AD83BE8309
:109F3000CE0101960E9487758091640E9091650E06
:109F4000892B09F483C10E9450AD882309F47EC196
:109F500082E70E943BAD8091640E9091650EDC011A
:109F6000ED91FC910088F189E02D68E170E0199590
:109F7000BE016F5F7F4F8091640E9091650E0E94CD
:109F8000F1AC89819A81AB81BC81C65EDE4F88834A
:109F90009983AA83BB83CA51D1408091640E90916A
:109FA000650EDC01ED91FC910488F589E02D199591
:109FB000C65EDE4F8881CA51D140882309F446C16C
:109FC0008F3FB1F4C55EDE4F8881CB51D1408F3FCA
:109FD00079F4C45EDE4F8881CC51D1408F3F41F48B
:109FE000C35EDE4F8881CD51D1408F3F09F42EC131
:109FF0006CE370E188E89EE00F94C91C86E195E06F
:10A000009A838983C65EDE4F88819981AA81BB814C
:10A01000CA51D1408B839C83AD83BE83CE01019610
:10A020000E9487758091640E9091650E892B09F4CA
:10A03000CDC00E9450AD882309F4C8C082E70E94B9
:10A040003BAD8091640E9091650EDC01ED91FC9129
:10A050000088F189E02D6CE170E01995BE016F5F19
:10A060007F4F8091640E9091650E0E94F1AC8981C2
:10A070009A81AB81BC81CC5EDE4F88839983AA83B1
:10A08000BB83C451D1408091640E9091650EDC0178
:10A09000ED91FC910488F589E02D1995CC5EDE4F99
:10A0A0008881C451D140882309F490C08F3FB1F416
:10A0B000CB5EDE4F8881C551D1408F3F79F4CA5EB7
:10A0C000DE4F8881C651D1408F3F41F4C95EDE4FDB
:10A0D0008881C751D1408F3F09F478C065E370E1B2
:10A0E00088E89EE00F94C91C66E1E62E65E0F62E36
:10A0F000FA82E982CC5EDE4F88819981AA81BB8198
:10A10000C451D1408B839C83AD83BE83CE01019625
:10A110000E948775FA82E982CC5EDE4F8881998140
:10A12000AA81BB81C451D1408B839C83AD83BE8304
:10A13000F801F182E082C65EDE4F88819981AA81B2
:10A14000BB81CA51D14082839383A483B583CE530C
:10A15000DF4FF982E882C25CD040C05EDE4F88816A
:10A160009981AA81BB81C052D140CC53DF4F8883F3
:10A170009983AA83BB83C45CD040CE5FDE4FF98253
:10A18000E882C250D140CA5DDE4F88819981AA81A0
:10A19000BB81C652D140CC5FDE4F88839983AA83AE
:10A1A000BB83C450D1409E012F5F3F4FA801BE0129
:10A1B0006E537F4FCE018E5F9E4F0E94DBB888E8C2
:10A1C0009EE00F94CA1B82E090E08FC086E195E08C
:10A1D0009A838983C65EDE4F488159816A817B817B
:10A1E000CA51D1404B835C836D837E83D8018D93AC
:10A1F0009C93C05EDE4F488159816A817B81C05249
:10A20000D140F8014283538364837583CE53DF4F7B
:10A2100099838883C25CD040CA5DDE4F8881998172
:10A22000AA81BB81C652D140CC53DF4F888399832A
:10A23000AA83BB83C45CD040AE014F5F5F4FB801BF
:10A24000CE018E539F4F0E941AB9B9CF86E195E097
:10A250009A838983C05EDE4F488159816A817B8100
:10A26000C052D1404B835C836D837E83D8018D9334
:10A270009C93CA5DDE4F88819981AA81BB81C652B9
:10A28000D140F80182839383A483B583BE016F5FBD
:10A290007F4FC8010E946CB992CF86E195E09A8306
:10A2A0008983CA5DDE4F88819981AA81BB81C652AC
:10A2B000D1408B839C83AD83BE83CE0101960E94E7
:10A2C000B7B97DCF63EF7FE082E99EE00F94C91CB0
:10A2D00064EC7FE082E99EE00F94C91C8091180A2B
:10A2E0008F5F8093180A86EF9FEF9093FF10809303
:10A2F000FE1089E0E9E2F2E0D80101900D928A9522
:10A30000E1F787E1F8013996DF011D928A95E9F7B7
:10A3100080E79EE0009731F0A801485F5F4F62E060
:10A320000E94496ACE018E539F4F0F94E0350E94E0
:10A33000ACBE683B7B408105910538F464E670E073
:10A3400080E090E00E9479BEF2CFCC53DF4F88814D
:10A350009981AA81BB81C45CD0408093DA0D90932F
:10A36000DB0DA093DC0DB093DD0DC8010E94A0B8F9
:10A37000892BC9F0E090D60DF090D70DD701ED9163
:10A38000FC91C088D18863E072E0CE0101960F9401
:10A39000091D49EE54E1BE016F5F7F4FC701F60111
:10A3A000199581113CC263E97FE082E99EE00F9438
:10A3B000C91C82E99EE00F94CA1B4AEEA42E4DE010
:10A3C000B42E7501D12CC12CD7018D919C91892B74
:10A3D00049F1960143E050E060E070E0CB010E945B
:10A3E000E1C9D701ED91FC9180859185009711F02D
:10A3F0000F94A744D701ED91FC9186819781009736
:10A4000011F00F94A744D701ED91FC9184819581BF
:10A410000F94A744F701808191810F94A744D7013D
:10A420001D921C92BFEFCB1ADB0AE2E0EE0EF11C8C
:10A43000F8E0CF16D10441F686E0E9E4F2E09E01AF
:10A440002F5F3F4F4901D90101900D928A95E1F7A5
:10A45000FE0137968AE1DF011D928A95E9F7AE0188
:10A460004A5F5F4F8BE1FA0111928A95E9F78CE61A
:10A470009EE0009719F066E00E94496A61E176E08B
:10A48000C8010F945952D12CC12CD5018D919D91A9
:10A490005D01892B09F0CCC18AE090E00F940B4458
:10A4A0007C01009709F4C4C1FC0117821682118651
:10A4B000108615821482D8010D900020E9F7CD0195
:10A4C0000197801B910B0F940B445C01F70195835E
:10A4D0008483892B11F40C945C5CD4010D900020D2
:10A4E000E9F7CD010197881999090F940B44F701F9
:10A4F00091878087009711F40C94595CB4010F94F4
:10A50000785280E590E0D70111969C938E93139634
:10A510001C921E921297B801C5010F947852F50152
:10A5200001900020E9F73197AE16BF0620F431976D
:10A5300081818E32C9F75F01B2E0AB0EB11CF5012B
:10A5400001900020E9F7CF018A199B090B960F941F
:10A550000B444C01D70117969C938E931697009746
:10A5600041F0B5010F94785268E176E0C4010F9490
:10A570005952F601EE0FFF1FE651F24FF182E082D1
:10A58000960142E050E060E070E0CB010E94E1C93A
:10A59000019709F456C164E276E082E99EE00F94E7
:10A5A000721C82E99EE00F94CA1B0FB6F894A8951E
:10A5B00080916000886180936000109260000FBEFF
:10A5C0008091FE109091FF1002970CF401C18091D0
:10A5D000180A81110C941F5C0091160A1091170A39
:10A5E0000115110511F40C941F5C0E94ACBE4B01C7
:10A5F0005C017801FEE3EF0EF11CF701808191818F
:10A60000A281B381A5019401281B390B4A0B5B0B76
:10A61000CA01B901683E33E0730781059105B0F1C5
:10A6200028EE33E040E050E00F94834D861A970AFD
:10A63000A80AB90AD7018D929D92AD92BC92139748
:10A64000F80186A597A5A0A9B1A969017A01CC0C4A
:10A65000DD1CEE1CFF1C8C159D05AE05BF0510F022
:10A660000C94075C16A617A610AA11AAF80182A9D5
:10A6700093A9A4A9B5A98C159D05AE05BF0510F039
:10A680000C94115C12AA13AA14AA15AAF80186A5A3
:10A6900097A5A0A9B1A9892B8A2B8B2B11F00C941B
:10A6A0001B5CEE5BFF4F8081833011F00C941B5CD0
:10A6B00084E08083C8010F941D3301967C01F8016A
:10A6C00082A993A9A4A9B5A9892B8A2B8B2BA1F4C4
:10A6D000EE5BFF4F8081833011F081110DC010823D
:10A6E000F8013E9684E1DF011D928A95E9F7C801E1
:10A6F0000F941D3303967C01B2E0EB16F10429F0B0
:10A70000E4E0EE16F10409F046C080E591E00E9415
:10A7100018B86091160A7091170A625F7F4FCE01D8
:10A7200001960F94091DCE0103960F94172960918D
:10A73000160A7091170A6A5E7F4FCE0101960F9438
:10A74000091DCE0103960F9425296091160A709178
:10A75000170A6E5E7F4FCE0101960F94091DCE0140
:10A7600003960F941E290F942C296091160A70915C
:10A77000170A625E7F4FCE0101960F94091D8B81EF
:10A780009C81AD81BE8180937B0C90937C0CA093C7
:10A790007D0CB0937E0C0F94FC35029711F40C9451
:10A7A0002D5CF3E0EF16F10411F40C94425C14F00C
:10A7B0000C94235C31E0E316F10411F40C943F5C3B
:10A7C00069ED72E142E0E416F10411F40C94475C87
:10A7D00088E199E20FB6F894A895809360000FBEC7
:10A7E000909360002091FE103091FF10C901C15D6F
:10A7F000DE4F0FB6F894DEBF0FBECDBFDF91CF9115
:10A800001F910F91FF90EF90DF90CF90BF90AF908E
:10A810009F908F907F906F905F904F9008956BE71F
:10A820007FE088E89EE00F94C91C88E89EE0C3CDD5
:10A83000BFEFCB1ADB0AE8E0CE16D10409F025CE33
:10A84000AACE6AE67FE088E89EE00F94C91CB801B2
:10A8500088E89EE00F94721C63E67FE088E89EE043
:10A860000F94C91C88E89EE09ECE82E090E0909311
:10A87000FF108093FE1099CE80911E0A8111D2C1E3
:10A880000E94501D6EEF73E189E39FE00F94C91C95
:10A8900089E39FE00F94CA1B8091640E9091650E2E
:10A8A000892B09F432C10E9450AD882309F42DC1CF
:10A8B00082E70E943BAD8091640E9091650EDC01B1
:10A8C000ED91FC910088F189E02D60E570E019952B
:10A8D0004FE050E0BE016F5F7F4F8091640E90911A
:10A8E000650E0E9495AD8C018091640E9091650E6D
:10A8F000DC01ED91FC910488F589E02D1995011595
:10A90000110509F402C1E1E0F0E0EC0FFD1FE00FDA
:10A91000F11F1082BE016F5F7F4F89E39FE00F94AC
:10A92000721C89E39FE00F94CA1BCE01865D9E4F87
:10A930000F94E035C45DDE4F88819981AA81BB8187
:10A94000CC52D1408093430E9093440EA093450E79
:10A95000B093460E65E476E083E39EE00F94FB1827
:10A96000BE016F5F7F4FCE01825E9E4F0F946A19CA
:10A970006FEB70E1CE01885E9E4F0F94331965E452
:10A9800076E0CE018E5F9E4F0F946A19BE016E5F16
:10A990007E4FCE018E5E9E4F0F946119BE01685EA0
:10A9A0007E4FCE018E5E9E4F0F94C718BE01625E31
:10A9B0007E4F0F94C7188C016FE479E0CE018C5D57
:10A9C0009E4F0F946A19F80184819581880F991F11
:10A9D000880F991F63E070E00F94E64DCE018C5D07
:10A9E0009E4F0F940218F12CE12CD80114968D91F2
:10A9F0009C91E816F90608F0B7C0B701C8010F949A
:10AA00008817E82F880FFF0BF595E795F595E795E3
:10AA1000EF73FF27EA58FF4E6491CE018C5D9E4F85
:10AA20000F945618B701C8010F948817B0E18B0234
:10AA300050011124E0E3AE22BB246701FFEFCF1ADF
:10AA4000DF0AD80114968D919C91C816D90608F09A
:10AA500078C0B601C8010F948817E82F880FFF0B44
:10AA6000B4E0F595E795BA95E1F7EF70FF27EA298D
:10AA7000FB29EA58FF4E6491CE018C5D9E4F0F94E6
:10AA80005618B601C8010F948817B4E08B02500124
:10AA90001124ECE3AE22BB246701F2E0CF0ED11CFF
:10AAA000D80114968D919C91C816D90608F03EC025
:10AAB000B601C8010F948817E82F880FFF0BA6E096
:10AAC000F595E795AA95E1F7E370FF27EA29FB29B9
:10AAD000EA58FF4E6491CE018C5D9E4F0F9456183C
:10AAE000B601C8010F948817E82FEF730E2E000CE3
:10AAF000FF0BEA58FF4E6491CE018C5D9E4F0F9480
:10AB00005618B3E0EB0EF11C70CF6AE071E1CE0194
:10AB100001960F944D4662ED70E182E99EE00F943C
:10AB2000C91C82E99EE00F94CA1BF4CEF501EA58D5
:10AB3000FF4E6491CE018C5D9E4F0F9456186DE3CD
:10AB4000DBCFF501EA58FF4E6491CE018C5D9E4F3C
:10AB50000F94561842E050E06DE476E0CE018C5D33
:10AB60009E4F0F942A18CDCF68EB70E1CE018F571E
:10AB70009F4F0F943319BE016F577F4FCE018E53F5
:10AB80009F4F0F946119BE016C5D7E4FCE018E53B5
:10AB90009F4F0F94C718BC0189E39EE00F941419CE
:10ABA000CE018E539F4F0F942B19CE018F579F4F7D
:10ABB0000F942B19CE018C5D9E4F0F942B19CE0153
:10ABC0008E5E9E4F0F942B19CE018E5F9E4F0F9479
:10ABD0002B19CE01885E9E4F0F942B19CE01825EF9
:10ABE0009E4F0F942B1984E59CE09093400E809328
:10ABF0003F0E82E79EE09093420E8093410E8FE4D9
:10AC00009EE00F94A13486E990E490934E0E8093D9
:10AC10004D0E61EC70E188E89EE00F94C91C81E064
:10AC200080931E0A83E090E022CE8091260A8091D4
:10AC3000FA108111DBCD0E94AFAF70FD2DC0809165
:10AC40001D0A81111EC00E940347883C910519F41A
:10AC500084E090E00CCE8091260A67ED73E18111CB
:10AC600012C0CE0101960F94E0358B819C81AD819D
:10AC7000BE81892B8A2B8B2B09F43BC28FE090E09D
:10AC8000F6CD67EC73E188E89EE00F94C91C88E874
:10AC90009EE00F94CA1BDCCF8091260A882349F0DE
:10ACA00084E090E09093FF108093FE106DE873E1D4
:10ACB000D5CD8FE090E0F6CFA8958091260A8091BF
:10ACC000210A9091220A009721F00E94E1AC823083
:10ACD00068F46AE773E188E89EE00F94C91C88E88D
:10ACE0009EE00F94CA1B87E090E0C1CDC85EDE4FA6
:10ACF0001882C851D140FE01EE5FFE4F11921192B1
:10AD00008EE0DF011D928A95E9F70E94E4AB88236B
:10AD100019F085E090E0ABCDE090210AF090220A96
:10AD2000E114F10441F0C7010E94E1AC082F10E0EA
:10AD3000023011055CF46BE372E182E99EE00F944E
:10AD4000C91C82E99EE00F94CA1B98CF70E060E0B6
:10AD5000C7010E94A76A009709F489C09093300A3E
:10AD600080932F0A6EE272E188E89EE00F94C91C7E
:10AD700060912F0A7091300A88E89EE00F94721C4F
:10AD800088E89EE00F94CA1B80912F0A9091300AA8
:10AD90000E94A0B8892B09F06DC060E576E082E9D9
:10ADA0009EE00F94721C82E99EE00F94CA1BE09013
:10ADB000210AF090220A61E070E0C7010E94A76AB0
:10ADC0005C010230110509F46CC062E0C7010E9409
:10ADD0003EACFC01C184D2840330110509F46AC081
:10ADE00063E070E0C7010E94A76A7C018091640E55
:10ADF0009091650E892B09F462C00E9450AD8823A2
:10AE000009F45DC082E70E943BAD8091640E909191
:10AE1000650EDC01ED91FC910088F189E02D60E484
:10AE200070E019954FE050E0BE016E5F7E4F80915B
:10AE3000640E9091650E0E9495AD4C018091640E58
:10AE40009091650EDC01ED91FC910488F589E02D6F
:10AE500019958114910499F1E2E0F1E0EC0FFD1FE6
:10AE6000E80DF91D10828E010E5F1E4F3EC080E777
:10AE700092E074CF6AE172E188E89EE00F94C91C09
:10AE800060912F0A7091300A88E89EE00F94721C3E
:10AE900063E172E188E89EE00F94C91C88E89EE0B7
:10AEA00084CF7BE5C72E77E0D72E9E01285E3E4FEC
:10AEB00079019CCFAE01485E5E4F7A0197CF053095
:10AEC00011058CF264E070E08091210A9091220AD1
:10AED0000E94A76A8C0163EF71E188E89EE00F94FD
:10AEE000C91C88E89EE00F94CA1BB092AD0CA092DA
:10AEF000AC0CD092AF0CC092AE0C87E794E4909368
:10AF0000A50C8093A40C40E150E066EE71E1CE0107
:10AF10008E539F4F0F947B4630E020E041E050E09D
:10AF200060E2CE018F579F4F0E94787240E250E05E
:10AF300060E073E3CE018F579F4F0F945D4665EC41
:10AF400071E188E89EE00F94C91CB50188E89EE095
:10AF50000F94721C63EC71E188E89EE00F94C91CA9
:10AF6000B60188E89EE00E9457AC6CEB71E188E87E
:10AF70009EE00F94C91CB70188E89EE00F94721CF4
:10AF800067EB71E188E89EE00F94C91CF7018081AE
:10AF9000811104C010E000E0F12CE12CA0902F0AF8
:10AFA000B090300A0E94E4AB8111C6C180918F0C31
:10AFB0009091900CDC01ED91FC910688F789E02DD1
:10AFC0001995882309F498C081E090E090939A0C39
:10AFD0008093990C87E0E9E6F2E0DE01119601909A
:10AFE0000D928A95E1F7FE01319685E090E021917E
:10AFF000A091910CB091920CA80FB91F2C930196BF
:10B000008C309105A1F786E3E114F10429F086EB79
:10B010000115110509F086EFC090910CD090920CAB
:10B02000F60184878091960C85878091950C8687A0
:10B030008090930C9090940CB401C5010F948E46AF
:10B0400041968816990608F08EC080918F0C9091D9
:10B05000900CDC01ED91FC910488F589E02D1995A7
:10B0600064E771E182E99EE00F94C91C6091B20C23
:10B070007091B30C82E99EE00E9457AC6CE571E1DF
:10B0800082E99EE00F94C91C82E99EE00F94CA1BDE
:10B090008091230A882379F0E091210AF091220A15
:10B0A000828193819093220A8093210A892B09F04F
:10B0B000B4C10E94491A0E94ACBE6093190A7093F1
:10B0C0001A0A80931B0A90931C0A8091150A8F5FBD
:10B0D0008093150A83330CF4ABC16EE271E182E90F
:10B0E0009EE00F94C91C82E99EE00F94CA1B109247
:10B0F000150A86EF9FEFBBCB6091AC0C7091AD0C45
:10B1000080918F0C9091900CDC01ED91FC9140911D
:10B11000AE0C5091AF0C6115710571F00088F1898A
:10B12000E02D1995019709F44FCF8EEF9FEF909383
:10B13000B30C8093B20C94CF0684F785E02D26E102
:10B1400035E03A8329834090A80C5090A90C609078
:10B15000AA0C7090AB0C4B825C826D827E82BE0129
:10B160006F5F7F4FDECF4FE050E0B601C5010E9418
:10B170001CAC6C01A090930CB090940CB501CE0166
:10B180008F579F4F0F948E468C0D9D1D0296A816CB
:10B19000B90608F45ACF6091910C7091920CA601F7
:10B1A000CE018F579F4F0E941CAC6C01A090930C56
:10B1B000B090940CB501CE018E539F4F0F948E46E4
:10B1C0008C0D9D1D0296A816B90608F43ECF60911D
:10B1D000910C7091920CA601CE018E539F4F0E944C
:10B1E0001CAC6C01E114F104B9F1A090930CB09087
:10B1F000940CB501C7010F948E4696012E5F3F4F08
:10B20000820F931FA816B90608F41FCF6091910C06
:10B210007091920CA601C7010E941CAC6C01011533
:10B220001105D1F0E090930CF090940CB701C80197
:10B230000F948E4696012E5F3F4F820F931FE816A4
:10B24000F90608F402CF6091910C7091920CA6015E
:10B25000C8010E941CAC6C01A601455051096091C7
:10B26000910C7091920C80E10E94B8BE0E94ACBE1D
:10B2700060939B0C70939C0C80939D0C90939E0C00
:10B2800060939F0C7093A00C8093A10C9093A20CE0
:10B2900080918F0C9091900CDC01ED91FC910084D9
:10B2A000F185E02D1995892B21F50E94ACBE009106
:10B2B0009F0C1091A00C2091A10C3091A20C6B015D
:10B2C0007C01C01AD10AE20AF30A2091970C30914E
:10B2D000980CA8EEB3E00F94D74DC616D706E80633
:10B2E000F906B0F28CEF9FEF9093B30C8093B20C01
:10B2F000ACCECE018E5E9E4F0E945FC3643071055E
:10B300008105910509F0A1CEE091910CF091920C8C
:10B31000838190E08111E8CF0E94ACBE60939F0CC6
:10B320007093A00C8093A10C9093A20C1092A30C8C
:10B330001092B30C1092B20C1092150A69EA71E1E6
:10B3400088E89EE00F94C91C60912F0A7091300A22
:10B3500088E89EE00F94721C88E89EE00F94CA1B58
:10B3600081E080931D0A30E020E043E050E061E49A
:10B37000CE0101960E9478726AE676E0CE010196CF
:10B380000F945952CE0101960E94B3BF30E020E0E5
:10B3900042E050E061E4CE0101960E9478726EE6D0
:10B3A00076E0CE0101960F945952BE016F5F7F4F38
:10B3B00089E39FE00F94CE1BCE0101960E94B3BF9C
:10B3C00030E020E041E050E061E4CE0101960E94CF
:10B3D00078726EE676E0CE0101960F945952BE0166
:10B3E0006F5F7F4F89E39FE00F94CE1BCE010196E4
:10B3F0000E94B3BF85E090E09093FF108093FE1011
:10B400000E94ACBE6093190A70931A0A80931B0ABB
:10B4100090931C0A66E871E121CA63E171E188E852
:10B420009EE00F94C91C88E89EE00F94CA1B43CE8F
:10B430008CE090E01CCA0E94ACBE0091190A1091E9
:10B440001A0A20911B0A30911C0A601B710B820B97
:10B45000930B60347F418105910508F4A6C830E064
:10B4600020E043E050E061E4CE018F579F4F0E94FF
:10B4700078726AE676E0CE018F579F4F0F9459524B
:10B480000091930C1091940CB801CE018F579F4FEF
:10B490000F948E4609960817190790F10E94E4ABA5
:10B4A000882371F18091990C90919A0C019609F47E
:10B4B000BCC090939A0C8093990CE091910CF09100
:10B4C000920C80919A0C8583E091910CF091920CF2
:10B4D0008091990C86836091910C7091920C47E059
:10B4E00050E0CE018F579F4F0E941CACAC014550DD
:10B4F00051096091910C7091920C82EA0E94B8BE41
:10B50000FE01EE53FF4F119211928EE3DF011D9267
:10B510008A95E9F71A821982FE0133968EE7DF01D8
:10B520001D928A95E9F730E020E041E050E060E4C8
:10B53000CE018E539F4F0E9478724FE350E060E03F
:10B5400073E3CE018E539F4F0F945D464FE750E05B
:10B550006AEF72E3CE0101960F947B4641E0BE0193
:10B560006F5F7F4FCE018E539F4F0E947ABF30E0B6
:10B5700020E041E050E060E4CE018E539F4F0E94F6
:10B5800078724FE350E064EA72E1CE018E539F4F30
:10B590000F945D464FE750E06AE972E1CE010196F3
:10B5A0000F947B464FE750E067E872E1CE010196C9
:10B5B0000F945D4641E0BE016F5F7F4FCE018E5319
:10B5C0009F4F0E947ABF30E020E041E050E060E40D
:10B5D000CE018E539F4F0E9478724FE350E067E197
:10B5E00073E3CE018E539F4F0F945D464FE750E0BB
:10B5F00067E772E1CE0101960F947B4641E0BE0100
:10B600006F5F7F4FCE018E539F4F0E947ABF86E0BF
:10B6100090E09093FF108093FE106DE573E188E851
:10B620009EE00F94C91C0C94D55281E090E041CF6C
:10B630008091260A0E94E4AB81110C94D55208CB6C
:10B640000E94ACBE6093190A70931A0A80931B0A79
:10B6500090931C0A85EF9FEF9093FF108093FE104C
:10B660008091260A0C94D5520E94ACBE0091190A12
:10B6700010911A0A20911B0A30911C0A601B710B51
:10B68000820B930B683873418105910510F40C947B
:10B69000D5521092FF101092FE100C94D5520E94B9
:10B6A000E4AB81110E9449C60E94ACBE6093190AA6
:10B6B00070931A0A80931B0A90931C0A8DE090E005
:10B6C000D6C80E94ACBE0091190A10911A0A2091A6
:10B6D0001B0A30911C0A601B710B820B930B6031AB
:10B6E00077428105910508F0B3CA0C94D5520E94A7
:10B6F000ACBE6093190A70931A0A80931B0A909348
:10B700001C0A8EE090E0B3C80E94ACBE0091190AFA
:10B7100010911A0A20911B0A30911C0A601B710BB0
:10B72000820B930B603C744D8140910508F0E1CC95
:10B730000C94D5520E943F4B009741F18130910506
:10B7400009F486CA019611F00C94D5520E94ACBE41
:10B750000091190A10911A0A20911B0A30911C0AB3
:10B76000601B710B820B930B60337547810591054C
:10B7700010F40C94D5526AE373E182E99EE00F94D1
:10B78000C91CF0E0E0E019950C94D55283E190E0FB
:10B790009093FF108093FE100E94ACBE6093190A34
:10B7A00070931A0A80931B0A90931C0A0C94D5522A
:10B7B0000E94E4AB81110E9449C60E94491A0E946E
:10B7C000ACBE6093190A70931A0A80931B0A909377
:10B7D0001C0A8FEE9FEF4BC88091260A8091FA10C9
:10B7E00081110C94F65382E190E09093FF108093C6
:10B7F000FE100E940347883C910509F429CA8091F4
:10B80000260A882309F42DCA63E173E13CCA821B2E
:10B81000930BA40BB50B86A797A7A0ABB1AB0C9469
:10B820003653821B930BA40BB50B82AB93ABA4AB2B
:10B83000B5AB0C944653F12CE12C0C945F53F12CD6
:10B84000E12C0C94CB5354E0E516F104F1F085E0C3
:10B85000E816F10411F00C94E8536AE073E182E910
:10B860009EE00F94C91C82E99EE00F94CA1B86EFEC
:10B870009FEF9093FF108093FE100C94E85366EFB7
:10B8800072E1EDCF66EC72E1EACF6AEA72E188E834
:10B890009EE00F94C91CCE0101960F94E035CE01B5
:10B8A00001960E94877588E89EE00F94CA1B0C944D
:10B8B000E853C5010F94A744D70118968D919C9128
:10B8C000009711F00F94A744C7010F94A7440C945C
:10B8D000CB528F929F92AF92BF92DF92EF92FF92E4
:10B8E0000F931F93CF93DF93CDB7DEB7A7970FB614
:10B8F000F894DEBF0FBECDBF7C0108A319A32AA315
:10B900003BA34CA35DA36EA37FA3CE0180960E94B0
:10B9100098234B015C01D7011496ED91FC91808531
:10B920008F70843009F0E9C0102F409100115091C0
:10B93000011161857285CE0101960E94DAE2CE0185
:10B9400001960E94FBDE882309F446C08B8589306E
:10B9500009F042C070E060E0CE0101960E9418E05C
:10B96000082FD92E6EE87AE089E39FE00F94C91C76
:10B97000602F7D2D89E39FE00E9457AC6CE87AE050
:10B9800089E39FE00F94C91CB501A40189E39FE0FE
:10B990000E94A2B066E87AE089E39FE00F94C91C98
:10B9A000612F70E089E39FE00E9457AC89E39FE03C
:10B9B0000F94CA1B80912C0A90912D0A892B29F192
:10B9C00040E050E3B701CE0180960E94A32070E0D2
:10B9D00060E0C7010E94121E10E000E0CE01019657
:10B9E0000E9477E3C801A7960FB6F894DEBF0FBE9A
:10B9F000CDBFDF91CF911F910F91FF90EF90DF901E
:10BA0000BF90AF909F908F90089581E090E09093C9
:10BA10002D0A80932C0A26E040E855E260E070E0B1
:10BA200087EB9BE00F94D51D0093B60C87EB9BE052
:10BA30009093B50C8093B40C1092C40D1092C60D67
:10BA40001092C50DEB81FC81153021F01F3011F0F3
:10BA5000123011F580858F70808770E060E083ED93
:10BA600097E090933F0D80933E0D1092410D109200
:10BA7000400D7093430D6093420D86E00E9406C016
:10BA800010922D0A10922C0A01E010E0882309F48C
:10BA9000A5CF682F70E09DCF80858F7080618087F3
:10BAA00022E538EB42E152E4C501B4010F942D4E7A
:10BAB00020E030E040E251E40F949F4C2DEE3EE94F
:10BAC0004CE35EE30F94994E4B015C0120E030E0C3
:10BAD000A9010F94414F20E030E040E05FE387FD93
:10BAE00007C0C501B4010F942D4E0F940B4FB7CF73
:10BAF000C501B4010F942C4EF8CF10E000E072CFD6
:10BB00002091BB0A260F3327331F21323105ECF475
:10BB10002091750BFC0190E080E0243069F082E018
:10BB20000895A091BB0A2191AC014556554FA40F31
:10BB3000B52FB11D2C930196861798F38091BB0AFF
:10BB4000680F6093BB0A80E0089581E0089508952E
:10BB50000895E091A40B8091A30BE81730F4F0E076
:10BB6000E252F54F808190E008958FEF9FEF0895A6
:10BB70009091A40B8091A30B2FEF3FEF981748F4FF
:10BB8000E92FF0E0E252F54F208130E09F5F909383
:10BB9000A40BC90108958091A30B9091A40B891B5C
:10BBA000990B0895CF92DF92EF92FF920F931F931C
:10BBB000CF93DF937C01CB018A0120917B0B222361
:10BBC00089F0EB016B01C40ED51ECC15DD0569F0C3
:10BBD0006991D701ED91FC910190F081E02DC701B1
:10BBE0001995F3CF642F0E94805DC801DF91CF913A
:10BBF0001F910F91FF90EF90DF90CF900895CF931A
:10BC0000DF931F92CDB7DEB7698320917B0B222390
:10BC1000F9F02091A10B203258F021E030E0FC0136
:10BC20003383228390E080E00F90DF91CF910895DD
:10BC30008091A20BE82FF0E0E458F44F99819083B3
:10BC40008F5F8093A20B8093A10B81E090E0ECCFFB
:10BC500061E0CE0101960E94805DF7CF90E0FC018B
:10BC6000EE56F74DE491F0E0EE0FFF1FE858F74D68
:10BC7000A591B4912C918852974DFC018491822317
:10BC800091E009F490E0892F089590E080E0089514
:10BC9000DC01ED91FC910284F385E02D1994DF9293
:10BCA000EF92FF920F931F93CF93DF93EC010C89D8
:10BCB0001D890115110559F01D8A1C8AC801DF91E3
:10BCC000CF911F910F91FF90EF90DF900895EC8539
:10BCD000FD858E859F85DF01A80FB91F2C91243229
:10BCE00009F055C011962C912B3709F050C00296DF
:10BCF000E80FF91FF12CE12CDF01D190DD2009F4D0
:10BD000046C08DE7D816E9F08FEFE81AF80AF4CFAD
:10BD1000198A188A2C853D852115310579F08E8583
:10BD20009F85280F391FF9012081222321F00196D8
:10BD30009F878E873EC01D861C86C0CF0FEF1FEFEA
:10BD4000BDCFE114F10419F11C928E859F850296F6
:10BD50006C857D85680F791FE881F9810684F785F8
:10BD6000E02DCE011995998B888B1B8A1A8AEC8558
:10BD7000FD858E859F85E80FF91FEE0DFF1DD28290
:10BD80008E859F850396E80EF91EFF86EE8628892C
:10BD900039892115310509F4BDCF8A899B89280F7E
:10BDA000391FF9012081222309F4B2CF01969B8B20
:10BDB0008A8B022F220F110B81CFDC011C96ED9193
:10BDC000FC911D971E968D919C91E80FF91F808123
:10BDD000082E000C990B0895DC0115968D919C910D
:10BDE000009739F0DC01ED91FC910680F781E02DA0
:10BDF0001994089583E090E00895DC011296ED9186
:10BE0000FC9113973097B9F016968D919C918430E0
:10BE1000910541F08530910541F0039749F482E0A6
:10BE200090E0089581E090E0089581E190E0089528
:10BE3000828590E0089590E080E0089585E090E0AC
:10BE400008951F93CF93DF930097A1F0FC01108515
:10BE5000212F2F70223071F4EC016185728583856A
:10BE600094850F94404C69877A878B879C87107FD5
:10BE700013601887DF91CF911F9108958EE090E0B5
:10BE80000895CF93DF93FC01C681D78180858F70A1
:10BE9000853079F08630E1F42097D1F0E881F9819E
:10BEA000309719F080818F7B79F40A80DB81C02D77
:10BEB000F3CF209769F0CE010E94415F811105C048
:10BEC0000A80DB81C02DF5CF81E0DF91CF9108950D
:10BED00080E0FBCF84E190E00895DC01ED91FC91DE
:10BEE0000484F585E02D60E0199581E090E00895E7
:10BEF000ECEBF0E080818A7B808360E084E10E944B
:10BF000003BC60E085E10C9403BC60E08DE00C9420
:10BF100003BC61E08DE00C9403BC0F931F93CF939F
:10BF2000DF930097D1F0FC0120852F702630A9F413
:10BF30008B01EC010E94C6AB009789F40E946BB1A3
:10BF4000AC01B801CE010E94A8B7B801CE01DF91C3
:10BF5000CF911F910F910C94C6AB90E080E0DF91E0
:10BF6000CF911F910F910895CF92DF92EF92FF92A0
:10BF7000CF93DF9369017A010E948D5FEC01892BD9
:10BF8000C9F08885982F9F70923039F0933071F006
:10BF9000911110C0807F82608887C701B6010F941D
:10BFA0000B4F69877A878B879C8704C0C986DA869E
:10BFB000EB86FC86CE01DF91CF91FF90EF90DF9072
:10BFC000CF900895CF92DF92EF92FF9269017A01AC
:10BFD000009791F0FC0120852F70253069F40E94B4
:10BFE0003EACFC01892B41F090859F70933059F451
:10BFF000C184D284E384F484C701B601FF90EF903A
:10C00000DF90CF9008959230B9F76185728583856E
:10C0100094850F94404C6B017C01EECFCF93DF935E
:10C02000EC0168E776E289E39FE00F94C91C6CE6B7
:10C0300076E289E39FE00F94C91C6C817D8189E3DE
:10C040009FE00E9457AC66E676E289E39FE00F949A
:10C05000C91C89E39FE00F94CA1B60E08C810E9499
:10C0600031BCE881F9810484F585E02D60E0CE01E2
:10C07000199581E090E0DF91CF910895CF93DF9300
:10C08000EC016FE376E289E39FE00F94C91C6C81B9
:10C090007D8189E39FE00E9457AC6DE376E289E3FE
:10C0A0009FE00F94C91CEA81FB810280F381E02D9F
:10C0B0006081718189E39FE00F94721C67E376E2EF
:10C0C00089E39FE00F94C91C89E39FE00F94CA1B8A
:10C0D000E881F981008CF18DE02DCE011995813038
:10C0E000910529F0029759F060E08C811AC063E055
:10C0F00070E0CE010F94B41060E00E9431BC60E0AB
:10C100008C810E9431BC61E070E0CE010F94B410CC
:10C1100060E00E9431BC62E070E0CE010F94B41088
:10C1200060E00E9431BCE881F9810484F585E02D4E
:10C1300060E0CE01199581E090E0DF91CF91089504
:10C14000CF93DF93EC016BED7EE189E39FE00F94E9
:10C15000C91CEA81FB810280F381E02D608171813D
:10C1600089E39FE00F94721C89E39FE00F94CA1B40
:10C17000E881F9810484F585E02D60E0CE01199510
:10C1800081E090E0DF91CF9108950D94A7440D9444
:10C19000A7440D94A7440D94A744EF92FF920F93E8
:10C1A0001F93CF93DF938C016DE873E289E39FE0E7
:10C1B0000F94C91C89E39FE00F94CA1BD801149601
:10C1C000ED91FC91309749F1C681D781209729F1F3
:10C1D000E881F9813097E9F080818823D1F060E728
:10C1E00076E0CE010E94C6AB7C01009791F0FC0185
:10C1F00081859285A385B4850097A105B10549F095
:10C200000F94A744D70119961D921D921D921C925E
:10C210001C970A80DB81C02DD9CFD801ED91FC910C
:10C220000484F585E02D60E0C801199581E090E077
:10C23000DF91CF911F910F91FF90EF9008950D9492
:10C24000A7440D94A7440D94A7440D94A744EF92DE
:10C25000FF920F931F93CF93DF93EC018B0180919B
:10C26000310A9091320A0097A9F0FC0120852F70C5
:10C27000263081F40E94C6ABFC0190859F709430FB
:10C2800049F481859285DF91CF911F910F91FF90A5
:10C29000EF900895EE88FF88C70101970D97D0F4BD
:10C2A00064E776E0C8010F946F52892B99F48FE20E
:10C2B000888F85E08E9DB0018F9D700D1124675988
:10C2C000784D46E050E0CE0149960F947B46CE0172
:10C2D0004896D9CF90E080E0D6CFFC01828193814F
:10C2E0000E948EE221E030E0823011F430E020E064
:10C2F000C90108950F931F93CF93DF938C01D0E072
:10C30000C0E001151105B1F0BE016150714EC801C8
:10C310000F944446892B51F4FE01ED5FF04E849159
:10C3200090E0DF91CF911F910F9108952596C23330
:10C33000D10539F781E090E0F4CFAF92BF92CF9270
:10C34000DF92EF92FF920F931F93CF93DF93CDB7BE
:10C35000DEB768970FB6F894DEBF0FBECDBFFC0105
:10C36000098B1A8B2B8B3C8B4D8B5E8B6F8B788F55
:10C3700082819381009709F49DC024813581232B0C
:10C3800009F498C0CC2009F495C06F0170E060E01A
:10C390000E9418E0192FD601ED91FC91008CF18DCF
:10C3A000E02DC60119955C018230910509F476C033
:10C3B000039709F445C095E0F1E0AF16B10409F028
:10C3C00091E019861A861B861C861D861E861F868E
:10C3D000188A8A85807F892B8A87EE24EA94FE2C2E
:10C3E00009891A892B893C894D895E896F89788DE5
:10C3F000CE0109960E943027F1E0AF16B10409F48E
:10C400004FC082E0A816B10409F045C06F8570E006
:10C41000D60114968C910E946DBC61E070E0C6015B
:10C420000F94B4106E8570E00E946DBC62E070E005
:10C43000C6010F94B4106D8570E00E946DBC2BC0D6
:10C44000612F661F6627661FCE0141960E947922E2
:10C450005C01BC01D60114968C910E946DBC6BE40A
:10C4600076E289E39FE00F94C91CF601648175812F
:10C4700089E39FE00E9457AC69E476E289E39FE09C
:10C480000F94C91CB50189E39FE00E9457AC89E372
:10C490009FE00F94CA1B81E090E00EC094E091CF22
:10C4A00063E070E0C6010F94B410688970E00E94E8
:10C4B0006DBCACCF90E080E068960FB6F894DEBF1C
:10C4C0000FBECDBFDF91CF911F910F91FF90EF90E5
:10C4D000DF90CF90BF90AF900895CF92DF92EF9210
:10C4E000FF920F931F93CF93DC011296ED91FC9175
:10C4F00060E0848195810E943EAC8C01009729F018
:10C50000FC0180858F708530D1F063E975E282E9A6
:10C510009EE00F94C91C82E99EE00F94CA1BC12CB7
:10C52000D12C90E8E92E9FEBF92EC701B601CF91EF
:10C530001F910F91FF90EF90DF90CF900895C80169
:10C540000E94E1AC813040F18630A8F1893020F5BD
:10C5500065E0C8010E943EACFC0190859F7093305D
:10C56000F9F4C184D284E384F484C1E060E0C801BA
:10C570000E943EACFC0190859F70933009F5618567
:10C5800072858385948520E030E0A9010F94394CB1
:10C5900087FF1FC0C111C9CFC12CD12C7601C5CFD7
:10C5A000923049F461857285838594850F94404C5F
:10C5B0006B017C01DACFC0E0C12CD12C7601D6CF43
:10C5C000923039F461857285838594850F94404C4F
:10C5D000DACFC111AACFC12CD12C8FE7E82E83E48A
:10C5E000F82EA3CFCF93DF93EC0161E675E289E3E8
:10C5F0009FE00F94C91CEA81FB810280F381E02D4A
:10C600006081718189E39FE00F94CE1BEC81FD81F5
:10C61000309721F0808191810F94A7448C819D8176
:10C620000F94A74470E060E08A819B810E9408DF3C
:10C630001D821C8281E090E0DF91CF910895CF931D
:10C64000DF93EC0168E776E089E39FE00F94CE1B6F
:10C6500040E050E0BA018A819B810E944BDFE88173
:10C66000F9810484F585E02D60E0CE0119956D8592
:10C670008C810E9403BC6D858D810E9403BC81E08A
:10C6800090E0DF91CF910895CF93DF93EC0167E8BD
:10C6900076E089E39FE00F94721CEA81FB810280BF
:10C6A000F381E02D6081718189E39FE00F94CE1BBF
:10C6B0008C819D81009711F00F94A74470E060E099
:10C6C0008A819B810E9408DF1D821C8281E090E0AC
:10C6D000DF91CF910895CF92DF92EF92FF920F9367
:10C6E0001F93CF93DF93009701F1DC011896EC9133
:10C6F000EF70E630D1F469017A018B01EC010E9400
:10C70000C6AB0097A1F4A7019601B801CE010E9423
:10C71000F4B7B801CE01DF91CF911F910F91FF9037
:10C72000EF90DF90CF900C94C6AB90E080E0DF916B
:10C73000CF911F910F91FF90EF90DF90CF900895D0
:10C74000CF92DF92EF92FF920F931F93CF93DF93DD
:10C75000009701F1DC011896EC91EF70E630D1F40E
:10C7600069017A018B01EC010E94C6AB0097A1F42C
:10C77000A7019601B801CE010E94D0B7B801CE0141
:10C78000DF91CF911F910F91FF90EF90DF90CF90AD
:10C790000C94C6AB90E080E0DF91CF911F910F9198
:10C7A000FF90EF90DF90CF9008958F929F92AF927D
:10C7B000BF92CF92DF92EF92FF920F931F93CF938E
:10C7C000DF93CDB7DEB760970FB6F894DEBF0FBE2C
:10C7D000CDBFE986FA860B871C872D873E874F875A
:10C7E000588B6115710511F0011103C090E080E0D4
:10C7F000CCC07B015C01DB018D909C9019821A8278
:10C800001B821C821D821E821F8218868A81807F65
:10C810008A836FE875E0C7010E94C6AB6C0166E9C8
:10C8200076E0C7010E94C6AB7C01C114D10451F16E
:10C83000F60180858F70843029F5818592850E946C
:10C840007A61182F8930B1F134F48130E4F4C12CCD
:10C85000D12C760168C08A30D1F7B701CE01099694
:10C860000E944B2F29833A834B835C836D837E83A5
:10C870008F8398873F7009F4B9CFCE0101960E944B
:10C88000222415C011E0B701CE0109960E944B2F5A
:10C8900029833A834B835C836D837E838F83988760
:10C8A0003F7009F4A3CFCE0101960E94DE236B01F5
:10C8B0007C0139C0B701CE0109960E944B2F298314
:10C8C0003A834B835C836D837E838F8398873F702D
:10C8D00009F48CCF31503B3008F0B9CFE32FF0E0B2
:10C8E0008827EA58FB498F4F0D940E4E8A648A645C
:10C8F000276481648164E564D864D864D864816401
:10C9000081642D813E814F815885AAE0B0E00F946B
:10C91000C44DCDCFCD80FAE0CF9E600111240D2C07
:10C92000000CEE08FF0880911E02893020F48091EF
:10C930001D028930E8F06CEF72E289E39FE00F940A
:10C94000C91CB40189E39FE00F94721C65EF72E289
:10C9500089E39FE00F94C91C2AE030E0B701A601EB
:10C9600089E39FE00F94EC1B89E39FE00F94CA1BBF
:10C97000D5011296ED91FC9162E0848195810E942F
:10C980003EAC009779F581E090E060960FB6F894A0
:10C99000DEBF0FBECDBFDF91CF911F910F91FF90F2
:10C9A000EF90DF90CF90BF90AF909F908F900895C1
:10C9B00020E030E040E251E46D817E818F819885F6
:10C9C0000F949F4C0F940B4F72CF6D817E818F819E
:10C9D00098852AE030E040E050E00F94A54D6901D1
:10C9E0007A01A1CFFC0120852F70263061F6B401B9
:10C9F0000E94C6AB5C01009731F2DC0118968C9165
:10CA000018978F709BEF980F923008F0BCCF4501BC
:10CA1000853029F416968C90169717969C90F50100
:10CA20008085806880876AE976E0C4010E94C6AB91
:10CA3000FC01892B61F0C186D286E386F486812FC2
:10CA40008295807F10851F70182B10879CCF6CEE0D
:10CA500072E289E39FE00F94C91CD5016D917C912E
:10CA600089E39FE00F94721C89E39FE00F94CA1B37
:10CA7000A70196016AE976E0C4010E94D0B76AE98D
:10CA800076E0C4010E94C6ABFC01892B09F47BCF80
:10CA90001295107F90859F70192BD7CF2F923F92C0
:10CAA0004F925F927F928F929F92AF92BF92CF925E
:10CAB000DF92EF92FF920F931F93CF93DF9300D0FB
:10CAC00000D01F921F92CDB7DEB709831A832B8344
:10CAD0003C834D835E836F837887DC011496ED91F0
:10CAE000FC910FEF1FEF3097F9F057014C01C2880E
:10CAF000D388E114F10489F1F7018081882369F179
:10CB0000C114D10489F1B701C6010E94C6ABE98006
:10CB1000FA800B811C812D813E814F815885BC019B
:10CB2000C4010E94D5638C01C80128960FB6F89401
:10CB3000DEBF0FBECDBFDF91CF911F910F91FF9050
:10CB4000EF90DF90CF90BF90AF909F908F907F90AD
:10CB50005F904F903F902F900895C114D10421F021
:10CB6000D6011696CD90DC907B80F12C0FEF1FEF55
:10CB7000272C312C512C412CC114D10449F161E7EF
:10CB800076E0C6010E94C6AB0097E9F0FC01208563
:10CB90002F702230C1F481859285A385B4858215DA
:10CBA0009305A405B50579F4E980FA800B811C8111
:10CBB0002D813E814F815885B601C4010E94D56305
:10CBC0008C01FF24F394D6011296CD90DC90D4CF43
:10CBD000F110AACF67E173E282E99EE00F94C91CCD
:10CBE000B50182E99EE00F94721C6BE073E282E96A
:10CBF0009EE00F94C91C672D70E082E99EE00E94C0
:10CC000057AC82E99EE00F94CA1B8ECFCF93DF937F
:10CC1000EC01EC81FD8140815181052E000C660BF9
:10CC2000770B228187EB9BE00F94D51D70E060E0CD
:10CC30008A819B810E9418E0E4EBFCE0828387EB11
:10CC40009BE0918380831092C40D1092C60D1092C8
:10CC5000C50DDF91CF910895CF93DF9361157105D5
:10CC600089F0EB01DC011296ED91FC9162E0848188
:10CC700095810E943EACBE010E94C6ABDF91CF9170
:10CC80000C945ABA90E080E0DF91CF9108954F92D2
:10CC90005F926F927F928F929F92AF92BF92CF924C
:10CCA000DF92EF92FF920F931F93CF93DF93CDB755
:10CCB000DEB768970FB6F894DEBF0FBECDBF098B05
:10CCC0001A8B2B8B3C8B4D8B5E8B6F8B788FDC01A3
:10CCD00012962D913C911397232B09F4DEC0CC20A2
:10CCE00009F4DBC06C01ED91FC91008CF18DE02D1D
:10CCF00019955C0164EF7EE189E39FE00F94C91C04
:10CD0000CE0141960E94AE26A114B10471F460E0F8
:10CD1000CE0141960E947922682FF6018481958187
:10CD20000F940C3781E090E0BAC0CE0141960E948A
:10CD30006D244C0194E0F2E0AF16B10459F081E1AA
:10CD4000A816B10409F445C091E0A1E0AA16B10407
:10CD500009F495E019861A861B861C861D861E8698
:10CD60001F86188A8A85807F892B8A87EE24EA9419
:10CD7000FE2C09891A892B893C894D895E896F8926
:10CD8000788DCE0109960E9430276AEE7EE189E314
:10CD90009FE00F94C91CCE0109960E94AE26B2E016
:10CDA000AB16B10489F0E1E1AE16B104B1F0AA947A
:10CDB000AB2809F0B7CF188963E070E0C6010F9483
:10CDC000B410612F0F940C376F85F6018481958123
:10CDD00051C0888D8170888FBCCF0FE710E08FEF36
:10CDE00088169806A9F0092C000CAA08BB08A50112
:10CDF00094012959310941095109AFEFB0E00F946D
:10CE0000C44D2BE531E040E050E00F94A54D890181
:10CE100063E070E0C6010F94B4105C01288930E033
:10CE2000D8010F94254E412C512C32014A94A30174
:10CE300092010F94A54D622FC5010F940C3764E049
:10CE400070E0C6010F94B4105C01AFEFB0E0A01B1E
:10CE5000B10B288930E00F94254EA30192010F9465
:10CE6000A54D622FC5010F940C376F85D60114961E
:10CE70008D919C910F940C371E8561E070E0C60186
:10CE80000F94B410612F0F940C371D8562E070E091
:10CE9000C6010F94B410612F43CF90E080E06896F4
:10CEA0000FB6F894DEBF0FBECDBFDF91CF911F91BB
:10CEB0000F91FF90EF90DF90CF90BF90AF909F9039
:10CEC0008F907F906F905F904F900895FC018181CB
:10CED00091E090937B0B80939C0B1092A20B10928D
:10CEE000A10B0895CF93C62F0E94666761EE8FE76E
:10CEF0009CE00E94FF5D6C2F8FE79CE00E94FF5D2D
:10CF0000CF910C9476BECF93DF93EC010E946667BD
:10CF100040E060EFCE010F943A37DF91CF910C944F
:10CF200076BE0E94666781E00E9486BD91E0811115
:10CF300090E0892F08951092750B81E08093740B17
:10CF400010924F0B61E084E10E9403BC61E085E137
:10CF50000E9403BCE9EBF0E080818E7F80838081BA
:10CF60008D7F808388E48093B80085E48093BC0043
:10CF70000895CF93DF9391E090939A0A882361F00C
:10CF8000C091B800D091BA000E94785F0E949B6760
:10CF9000D093BA00C093B800DF91CF910895CF929B
:10CFA000DF92EF92FF920F931F93CF93FC01C18109
:10CFB0000E9461BD6B017C018091750B811164C081
:10CFC00081E08093750B8093740B9FEF9093730BAC
:10CFD0001092720B1092710B8093500B8091500B3A
:10CFE000CC0FC82BC093500B80914F0B813009F0B0
:10CFF00081C010924F0B0E9461BD6B017C0180913A
:10D00000500B8093BB008091770B9091780BA0918F
:10D01000790BB0917A0B892B8A2B8B2BA1F00E9474
:10D0200061BD0091770B1091780B2091790B3091B5
:10D030007A0B6C197D098E099F09061717072807B7
:10D04000390708F442C08091BC0083FDD8CF85EC3D
:10D050008093BC000E9461BD6B017C018091750BC7
:10D06000813009F449C08091720B811167C08091B1
:10D07000720BE1E5FBE0AEEDBAE090E0981751F1FC
:10D0800021912D939F5FFACF8091770B9091780B30
:10D09000A091790BB0917A0B892B8A2B8B2B09F4F9
:10D0A0008BCF0E9461BD0091770B1091780B20917E
:10D0B000790B30917A0B6C197D098E099F0906173F
:10D0C00017072807390708F077CF8091760B0E9461
:10D0D000B96780E01092A40B8093A30B8FE79CE0CC
:10D0E0000E94B85DCF911F910F91FF90EF90DF905C
:10D0F000CF90089585EEACCF8091770B9091780B0F
:10D10000A091790BB0917A0B892B8A2B8B2B09F488
:10D11000A5CF0E9461BD0091770B1091780B2091F3
:10D12000790B30917A0B6C197D098E099F090617CE
:10D1300017072807390708F091CFC7CF81E099CFAB
:10D140008F929F92AF92BF92EF92FF921F93CF93D5
:10D15000DF93EC010E94ACBE4B015C0110E08BE45C
:10D16000E82EF12C0E94ACBE681979098A099B0946
:10D17000683E73408105910510F5ED85FE85309779
:10D1800009F0199560EFCE010E947267CE010E94EE
:10D19000CF67182F80FD0FC08A81813009F41A8271
:10D1A000812FDF91CF911F91FF90EF90BF90AF90B3
:10D1B0009F908F900895C7010197F1F7D3CF81E039
:10D1C0008A83EECFCF93DF93EC0163EC0E9472670A
:10D1D000CE01DF91CF910C94CF6785ED8093BC0099
:10D1E0008091770B9091780BA091790BB0917A0B8D
:10D1F0000796A11DB11D23E0B695A7959795879534
:10D200002A95D1F72091BC0024FD03C01092750B24
:10D2100008954091770B5091780B6091790B709144
:10D220007A0B452B462B472B69F30097A105B105D7
:10D2300041F02AE22A95F1F700C00197A109B1094E
:10D24000E1CF8091760B0C94B9671F920F920FB6C5
:10D250000F9211240BB60F922F933F934F935F932E
:10D260006F937F938F939F93AF93BF93EF93FF93AE
:10D270008091B900887F803609F44DC008F040C025
:10D28000883209F4A9C028F5803109F49DC0C8F49A
:10D29000882309F4FBC0883009F496C0FF91EF9110
:10D2A000BF91AF919F918F917F916F915F914F91BE
:10D2B0003F912F910F900BBE0F900FBE0F901F90BC
:10D2C0001895883109F488C0803241F78093730B38
:10D2D00014C0803409F49DC040F48033B9F388331E
:10D2E000E9F68093730B85ECB0C0803509F485C0F6
:10D2F000883509F496C0883489F60E94ED68CECF4F
:10D30000883909F48CC038F5883729F050F488360C
:10D3100011F0803719F683E08093750B1092DD0AC7
:10D3200057C0883809F47BC0803919F0803809F07B
:10D33000B5CF8091DD0A803208F071C0E091DD0A3E
:10D3400081E08E0F8093DD0A8091BB00F0E0E35412
:10D35000F54F80833DC0803B39F0E0F4803A09F41A
:10D3600079C0883A09F09ACF84E08093750B1092C7
:10D37000BC0A1092BB0AE0919F0BF091A00B19958B
:10D380008091BB0A81110FC081E08093BB0A10928B
:10D390009B0A09C0803C09F4A6CF883C09F4A3CFBE
:10D3A000883B09F07BCFE091BC0A81E08E0F80932F
:10D3B000BC0AF0E0E556F54F80818093BB00909168
:10D3C000BC0A8091BB0A29C08091500B8093BB009E
:10D3D00085EC8093BC0062CF9091720B8091710BB1
:10D3E000981758F5E091720B81E08E0F8093720BC5
:10D3F000F0E0EF5AF44F8081E9CFE091720B81E0C9
:10D400008E0F8093720B8091BB00F0E0EF5AF44FC7
:10D4100080839091720B8091710B9817C8F285E808
:10D42000D8CFE091720B81E08E0F8093720B8091C8
:10D43000BB00F0E0EF5AF44F80838091740B8111B0
:10D440005CCF81E080934F0B84EA8093BC00109204
:10D45000750B24CF85EC8093BC001092750B8091E6
:10D46000DD0A803230F4E091DD0AF0E0E354F54F5C
:10D4700010826091DD0A70E0E0919D0BF0919E0BAF
:10D480008DEB9AE019951092DD0A08CF1092730B7C
:10D4900034CFCF93DF93EA01282FDC01ED91F0E048
:10D4A00094E0F595E7959A95E1F7E551FD4F808178
:10D4B0008883FD013197E081EF70F0E0E551FD4F89
:10D4C0008081898322968A2F821B861738F36150C8
:10D4D00070E0660F771F460F571FFA011282DF9127
:10D4E000CF910895CF92DF92EF92FF9269017A0176
:10D4F000009791F0FC0120852F70263069F40E947E
:10D50000C6ABFC01892B41F090859F709230A1F44D
:10D51000C184D284E384F484C701B601FF90EF9004
:10D52000DF90CF90089561857285838594850F94EF
:10D530000B4F6B017C01F0CF9330A9F3913061F771
:10D54000C1840C2C000CDD08EE08FF08E5CF009725
:10D5500089F0FC0120852F70253061F40E943EACDB
:10D56000009741F0FC0120852F70243019F481854B
:10D570009285089590E080E008950F931F93CF93D4
:10D58000DF9364E578E289E39FE00F94ED1C81E08E
:10D590000E9486BD0E94785F61E085E10E9431BCF7
:10D5A00060E084E10E9431BCC4E1D0E010E001E021
:10D5B000612F85E10E9403BC10276AE070E080E0E3
:10D5C00090E00E9479BE219799F764E170E080E0D5
:10D5D00090E00E9479BE0E9459B88091F510909118
:10D5E000F610009729F10E949167882309F1809134
:10D5F000F5109091F6100E94836769E378E289E361
:10D600009FE00F94ED1CE091F510F091F61000836F
:10D610008091F5109091F6100F947F3765E278E2D3
:10D62000811102C060E178E289E39FE00F94ED1C74
:10D6300081E0DF91CF911F910F910895CF92DF92FA
:10D64000EF92FF920F931F93182F6A017B010E94A4
:10D65000ACBE04C096958795779567951A95D2F7D5
:10D660006C217D218E219F218B019C01015011098C
:10D67000210931090E3F1F4F2F4F3F4F20F061E02E
:10D6800070E080E090E01F910F91FF90EF90DF90AD
:10D69000CF9008953F924F925F926F927F928F92B8
:10D6A0009F92AF92BF92CF92DF92EF92FF920F9331
:10D6B0001F93CF93DF9300D000D0CDB7DEB77C01AE
:10D6C000362E80912E0A882309F40AC1D7011496B8
:10D6D0009C9180911D02891708F402C18091980ADB
:10D6E0009091990ABAE06B1312C28D5B954FFC01C1
:10D6F0001082D70118968D919C91892B09F4ECC06A
:10D7000080913F0A9091400AA091410AB091420A4B
:10D71000892B8A2B8B2B09F0CBC00E94ACBE2B012E
:10D720003C01F70100851185D80119966D917C9116
:10D730006115710599F4F80185809680A780B08401
:10D740008091750C9091760CA091770CB091780C2B
:10D7500088169906AA06BB0609F484C0D8011B9650
:10D760004D915C911C974115510509F47BC0F7015F
:10D77000248153968C91539790E0322F377002C0DA
:10D78000959587953A95E2F780FF6CC0C22ED12C13
:10D79000C601887F9370892B39F451968D919C91A5
:10D7A000887F9370C82AD92AD8018D919C91DC0179
:10D7B000ED91FC916115710509F4C1C00688F789E6
:10D7C000E02D1995019709F04DC06CE3F8018081B7
:10D7D00091810F94E51BB601D8018D919C910E9417
:10D7E0009CB0F8012281808191816BE177E2222354
:10D7F00011F069E177E20F94C91CD8011D966D9173
:10D800007C911E978D919C910F94721C60E2F8019F
:10D81000808191810F94E51BD8011F966D917C91B9
:10D8200050978D919C910F94721CF80122818081F8
:10D8300091816EE077E2222311F068E077E20F94A5
:10D84000C91C63E47AE0D8018D919C910F94721CFD
:10D85000F80180819181DC01ED91FC91008CF18DCA
:10D86000E02D19950E94ACBEAB01BC0144195509CD
:10D8700066097709F701858196814536510561056D
:10D88000710508F472C0009721F068E577E20F9403
:10D89000ED1C4FEF5FEFBA0180E00E941E6B6093BA
:10D8A0003F0A7093400A8093410A9093420A14C041
:10D8B0000E94ACBE00913F0A1091400A2091410A9B
:10D8C0003091420A601B710B820B930B60337547DA
:10D8D0008105910508F021CF1092990A1092980ABB
:10D8E000D70115968D919C911697009771F014961B
:10D8F0003C9120911E02231740F0DC01ED91FC9138
:10D900000190F081E02D632D199581E090E026963D
:10D910000FB6F894DEBF0FBECDBFDF91CF911F9140
:10D920000F91FF90EF90DF90CF90BF90AF909F90BE
:10D930008F907F906F905F904F903F9008950488F4
:10D94000F589E02D26E135E03A832983D801159643
:10D950008D909D90AD90BC9018978B829C82AD82EB
:10D96000BE82BE016F5F7F4F2CCF40913F0A509126
:10D97000400A6091410A7091420A452B462B472B81
:10D9800009F4AACF009721F069E477E20F94ED1C27
:10D9900010923F0A1092400A1092410A1092420AD5
:10D9A000D70118960D911C91F8016185728561155A
:10D9B000710591F445805680678070848091750C64
:10D9C0009091760CA091770CB091780C481659067E
:10D9D0006A067B0609F480CFD8011B964D915C91B5
:10D9E0001C974115510509F477CFF701248153960F
:10D9F0008C91539790E0322F377002C095958795A0
:10DA00003A95E2F780FF68CFC22ED12CC601887FFD
:10DA10009370892B39F451968D919C91887F9370E6
:10DA2000C82AD92AD8018D919C91DC01ED91FC91F5
:10DA30006115710509F455C00688F789E02D19951F
:10DA4000019709F049CF6CE3F801808191810F942F
:10DA5000E51BB601D8018D919C910E949CB0F80104
:10DA600022818081918164E377E2222311F062E3D5
:10DA700077E20F94C91CD8011D966D917C911E9779
:10DA80008D919C910F94721C60E2F80180819181CC
:10DA90000F94E51BD8011F966D917C9150978D9145
:10DAA0009C910F94721CF80122818081918167E220
:10DAB00077E2222311F061E277E20F94C91C6AE356
:10DAC00077E2D8018D919C910F94C91CF801808157
:10DAD0009181DC01ED91FC91008CF18DE02D199587
:10DAE000FBCE0488F589E02D26E135E03A832983D1
:10DAF000D80115964D905D906D907C9018974B8253
:10DB00005C826D827E82BE016F5F7F4F98CF8435CD
:10DB100091050CF0E5CEBDE06B1709F4E1CE9C0158
:10DB20002F5F3F4F3093990A2093980A8D5B954F52
:10DB3000FC016083D5CECF92DF92FF920F931F93AB
:10DB4000CF93DF9300D000D01F921F92CDB7DEB7E6
:10DB50006C01F02E1A83022F10E0FF2029F001152E
:10DB6000110511F401E010E040E050E061E070E0E8
:10DB7000F601828193810E94EBE001301105A9F149
:10DB80000230110541F0012BB1F569E473E289E33C
:10DB90009FE00F94C91C8A818F70B9F1F601028150
:10DBA0001381C8010E948CDF672B682B692B89F4D5
:10DBB00001E010E0C80128960FB6F894DEBF0FBE52
:10DBC000CDBFDF91CF911F910F91FF90DF90CF904C
:10DBD00008954FEF5FEFBA0180E00E941E6BAB012A
:10DBE000BC01C8010E944BDFE3CFF1E0FF1681F0DA
:10DBF00082E0F81669F06DE373E289E39FE00F9429
:10DC0000C91C89E39FE00F94CA1B10E000E0D2CF4B
:10DC1000F601C280D380C6010E948CDF672B682B7F
:10DC2000692B31F24FEF5FEFBA0180E00E941E6B6B
:10DC3000AB01BC01C6010E944BDFBCCF2F923F92CB
:10DC40004F925F926F927F928F929F92AF92BF920C
:10DC5000EF92FF920F931F93CF93DF93CDB7DEB771
:10DC60002C970FB6F894DEBF0FBECDBF61307105A3
:10DC700009F463C18C01FC01E280F38040E050E0D4
:10DC800061E070E0C7010E9414E1672B682B692BEB
:10DC900009F453C140E050E062E070E0C7010E9427
:10DCA00014E1672B682B692B89F48091000288238B
:10DCB00009F443C140E050E062E070E0C7010E9417
:10DCC000EBE080910002815080930002F801E28035
:10DCD000F380C7010E948CDF4B015C0119821A821C
:10DCE0001B821C821D821E821F8218868A81807F71
:10DCF0008A8340E050E2B701CE0101960E94B6212E
:10DD000060E0CE0101960E9479227C01F8018281B7
:10DD100093810E948EE2823011F0853011F4F12C53
:10DD2000E12CF80186819AEC980F903108F0B7C188
:10DD300021853285A90170E060E049875A876B87A9
:10DD40007C8743845484712C612C0E9444BD9C01C7
:10DD5000990F440B550B2419350946095709AFEFA4
:10DD6000B0E00F94C44D29853A854B855C85241914
:10DD70003509460957090F94A54D390137FDB9C139
:10DD80005FEF6516710411F00CF0B6C181149104B7
:10DD9000A104B10409F08BC1E618F70856EFE516A7
:10DDA0005FEFF5060CF0F6C0F801658585810E94ED
:10DDB00003BCF801A280B380C5010E948CDF672BF1
:10DDC000682B692B59F44FEF5FEFBA0180E00E9496
:10DDD0001E6BAB01BC01C5010E944BDFF801B48092
:10DDE00065858EEF8B0D8C3028F084ED8B0D8330A4
:10DDF00008F070C0AA27BB27AE19BF09662309F433
:10DE00005CC09D01A1E0BFEF0F941D4E29E130E001
:10DE100040E050E00F94A54DBA01A90141505F4F79
:10DE20006F4F7F4F942F852F692F782F6F3F71058C
:10DE300019F014F06FEF70E06634710514F466E4C5
:10DE400070E08B2D78C06EE273E289E39FE00F945F
:10DE5000C91C89E39FE00F94CA1B6DE976E089E352
:10DE60009FE00F94CE1BF801658584810E9403BC5E
:10DE7000F801658585810E9403BC40E050E0BA014D
:10DE8000F801828193810E944BDF40E050E061E025
:10DE900070E0F801828193810E94C2E040E050E08E
:10DEA00062E070E0F801828193810E94C2E080917B
:10DEB00000028F5F8093000240C02FEF30E00F948C
:10DEC000254E29E130E040E050E00F94A54D922F1F
:10DED000832FAACF858191E069279EEF980F9C3010
:10DEE00020F08C52833008F0D6C08B2D0E9403BCEA
:10DEF000AA27BB27AE19BF09F80185858823B1F190
:10DF00002FEF30E00F94254E29E130E040E050E063
:10DF10000F94A54D922F832F692F782F6F3F710596
:10DF200019F014F06FEF70E06634710514F466E4D4
:10DF300070E0F80185810E946DBC90E080E02C9635
:10DF40000FB6F894DEBF0FBECDBFDF91CF911F910A
:10DF50000F91FF90EF90BF90AF909F908F907F9028
:10DF60006F905F904F903F902F9008959D01A1E09A
:10DF7000BFEF0F941D4E29E130E040E050E00F94D8
:10DF8000A54DBA01A90141505F4F6F4F7F4F942FAC
:10DF9000852FC2CFFBE0EF16F1040CF45ECFF80141
:10DFA000658584810E9403BCF801A280B380C5010D
:10DFB0000E948CDF672B682B692B59F44FEF5FEFC2
:10DFC000BA0180E00E941E6BAB01BC01C5010E943A
:10DFD0004BDFF801B58065858EEF8B0D8C3020F01E
:10DFE00084ED8B0D8330B0F4662351F09701A1E0EE
:10DFF000BFEF0F941D4E23E330E040E050E00ACF26
:10E000002FEF30E0D7010F94254E23E330E040E0BE
:10E0100050E05BCF848191E069279EEF980F9C30A0
:10E0200018F08C528330B8F58B2D0E9403BCF80198
:10E0300085858823E1F02FEF30E0D7010F94254E3E
:10E0400029E130E040E050E00F94A54D922F832F5E
:10E05000692F782F77FF02C070E060E06F3F710595
:10E0600019F014F06FEF70E0F801848164CF97012C
:10E07000A1E0BFEF0F941D4E29E130E040E050E0F9
:10E080000F94A54DBA01A90141505F4F6F4F7F4FCB
:10E09000942F852FDDCF8B2D0E9403BC4ECF66249D
:10E0A0006A94762C81149104A104B104F1F0F80172
:10E0B00027803084032C000C440855080E94ACBE15
:10E0C000211431044104510409F4BDCE68197909C1
:10E0D0008A099B09621573058405950508F0B3CE7E
:10E0E000FFEF6F167F0609F057CE4FE7E41AF108ED
:10E0F00055CE712C612C4ACE66246A94712C46CE82
:10E100001F93CF93DF9300D000D0CDB7DEB761303F
:10E11000710509F46BC05CF4672B09F45DC06AE912
:10E1200070E289E39FE00F94C91C80E04BC062302D
:10E13000710571F06330710591F79093B90C80937C
:10E14000B80C55275093BB0C4093BA0C84E009C01F
:10E150009093B90C8093B80C5093BB0C4093BA0CBD
:10E1600083E00E9406C0182F4FEF5FEFBA0180E0F6
:10E170000E941E6B60933B0A70933C0A80933D0A99
:10E1800090933E0A1123D9F065E870E282E99EE09F
:10E190000F94C91C812F90E0B0E0A0E089839A839E
:10E1A000AB83BC8380E190E09E838D83BE016F5F73
:10E1B0007F4F82E99EE00E94D1FA0F94CA1B81E052
:10E1C0001111B3CF26960FB6F894DEBF0FBECDBFA8
:10E1D000DF91CF911F9108959093B90C8093B80C63
:10E1E0005093BB0C4093BA0C81E0BBCF9093B90C19
:10E1F0008093B80C5093BB0C4093BA0C82E0B1CF23
:10E20000CF92EF92FF920F931F93CF93DF9300D0A3
:10E2100000D01F921F92CDB7DEB77C0109831A830D
:10E220002B833C834D835E836F83788762EC7EE132
:10E2300089E39FE00F94C91CCE0101960E94AE268F
:10E24000898181112CC00B81013089F128F010E007
:10E250000230F1F5CC2001F160E0CE0101960E9480
:10E260007922F70102811381892B81F0C8010E9474
:10E270008CDF672B682B692B79F44FEF5FEFBA01C6
:10E2800080E00E941E6BAB01BC0103C040E050E087
:10E29000BA01C8010E944BDF81E090E02AC08031C2
:10E2A000B0F58E30B8F58130A9F18230B9F165EB67
:10E2B0007EE189E39FE00F94C91C698189E39FE0B7
:10E2C0000E9450AC89E39FE00F94CA1B01E010E06C
:10E2D00065EA7EE189E39FE00F94C91CB80189E3F8
:10E2E0009FE00E9457AC89E39FE00F94CA1B90E027
:10E2F00080E028960FB6F894DEBF0FBECDBFDF9149
:10E30000CF911F910F91FF90EF90CF90089583517F
:10E31000843068F6F70102811381A8CF40E050E015
:10E32000BA01F70182819381B5CF8F929F92AF920C
:10E33000BF92CF92DF92EF92FF920F931F93CF93F2
:10E34000DF9300D000D01F921F92CDB7DEB76D7F54
:10E350006130710509F4B7C0FC01E280F380E1147B
:10E36000F10409F4B0C08C01C7010E948CDF4B019D
:10E370005C0161E070E0C7010E94D2DF811491046A
:10E38000A104B10409F49FC020E030E04AE754E45E
:10E390000F949F4C0F94124F6B017C01C114D10458
:10E3A000E104F10409F48FC00E94ACBE6819790938
:10E3B0008A099B096C157D058E059F0508F483C0AD
:10E3C000F801A280B38070E060E0C5010E94D2DF56
:10E3D00020E030E048EC52E40F949F4C0F94124F31
:10E3E0006B017C014FEF5FEFBA0180E00E941E6B72
:10E3F000AB01BC01C5010E944BDF19821A821B824E
:10E400001C821D821E821F8218868A81807F8A83D9
:10E41000F8016281738140E050E3CE0101960E94D1
:10E42000B621CE0101960E9422244B015C016BEAC9
:10E4300076E089E39FE00F94721CB501A40189E3A3
:10E440009FE00E944DAC6AEB76E089E39FE00F9479
:10E45000721CB701A60189E39FE00E944DAC89E3DD
:10E460009FE00F94CA1BC80CD91CEA1CFB1C8A81B4
:10E47000807F86608A83CD82DE82EF82F886F80113
:10E480006281738140E050E2CE0101960E94A32098
:10E490006EEB76E089E39FE00F94721CB701A60152
:10E4A00089E39FE00E944DAC89E39FE00F94CA1B73
:10E4B00030E020E040E050E260E070E0F80182816E
:10E4C00093810E94C43790E080E028960FB6F894BC
:10E4D000DEBF0FBECDBFDF91CF911F910F91FF9097
:10E4E000EF90DF90CF90BF90AF909F908F90089566
:10E4F0008F929F92AF92BF92CF92DF92EF92FF9254
:10E500000F931F93CF93DF937C014A015901C09170
:10E51000310AD091320A062F660F110B209709F4A9
:10E520005CC088858F70863009F055C063ED76E059
:10E53000CE010E94C6AB6C0182E08816910449F0BE
:10E5400068ED76E0E3E08E16910429F0D0E0C0E0BB
:10E5500006C06CED76E0CE010E94C6ABEC01C114A2
:10E56000D104D9F1F60180858F708430B1F56185D1
:10E570007285A801C7010F949D52A80161EA75E058
:10E58000C7010F947F52209779F188858F7084306E
:10E5900059F569857A85A801C7010F947F52A801B2
:10E5A00061EA75E0C7010F947F52A114B10429F00C
:10E5B000A801B501C7010F947F52C701DF91CF9128
:10E5C0001F910F91FF90EF90DF90CF90BF90AF9091
:10E5D0009F908F900895D0E0C0E0A8016CEB77E2A7
:10E5E000C7010F947B46C9CFF2E08F16910481F0EA
:10E5F00083E08816910429F060912F0A7091300A07
:10E60000CACFA80166EB77E2C7010F945D46C7CF7A
:10E61000A80163EB77E2F8CFFF920F931F93CF939C
:10E62000DF93CDB7DEB7C455D1090FB6F894DEBF7E
:10E630000FBECDBF8C01F62EDC0116966C91FF202B
:10E6400011F081E06827F80184810E9403BCF80181
:10E6500087819085A185B285883E9340A105B1054B
:10E6600008F49BC068EB76E289E39FE00F94C91C35
:10E6700063EB76E289E39FE00F94C91CD8011496FE
:10E680006D917C9189E39FE00E9457AC6EEA76E23F
:10E6900089E39FE00F94C91C6F2D70E089E39FE030
:10E6A0000E9457AC89E39FE00F94CA1BFE01E55B13
:10E6B000FF4F8FE290E08193919388E0DF011D92FC
:10E6C0008A95E9F767EA76E2CE01855B9F4F0F9462
:10E6D0003946F801828193810E948EE2FF2009F47D
:10E6E00069C06FE976E2853151F068E976E28631FA
:10E6F00031F06CE876E28F3011F464E976E2CE0115
:10E700008F5B9F4F0F944D468091FE109091FF10AC
:10E71000059709F442C0D8011296ED91FC91028050
:10E72000F381E02D0081118101151105B1F140E463
:10E7300050E0B801CE0101960F949D526FE270E057
:10E74000CE0101960F946452892B41F4980143E065
:10E7500050E060E4CE0101960E9478724FE350E0F1
:10E76000BE01655B7F4FCE0101960F947F520E94E0
:10E77000E4AB882391F08091FE109091FF100697F2
:10E7800061F48091F910811108C041E0BE016F5B16
:10E790007F4FCE0101960E947ABFCC5ADF4F0FB651
:10E7A000F894DEBF0FBECDBFDF91CF911F910F91C7
:10E7B000FF90089568E876E2823009F4A0CF63E81C
:10E7C00076E29DCFAF92BF92CF92EF92FF920F93DE
:10E7D0001F93CF93DF9300D000D01F921F92CDB72D
:10E7E000DEB75C0109831A832B833C834D835E83F0
:10E7F0006F8378876DEF76E289E39FE00F94C91C01
:10E80000CE0101960E94AE26E114F10439F066EFC4
:10E8100076E2C7010F944446009749F1F501028161
:10E8200013810115110509F18981811163C08B8163
:10E83000813009F467C068F1823049F1082F10E097
:10E8400063ED76E289E39FE00F94C91C63EC76E206
:10E8500089E39FE00F94C91CB80189E39FE00E94FF
:10E8600057AC89E39FE00F94CA1B90E080E02896A4
:10E870000FB6F894DEBF0FBECDBFDF91CF911F91D1
:10E880000F91FF90EF90CF90BF90AF900895CC2064
:10E89000D9F060E0CE0101960E947922892B09F41B
:10E8A0004EC0C8010E948CDF672B682B692BF9F4DE
:10E8B0004FEF5FEFBA0180E00E941E6BAB01BC011D
:10E8C000C8010E944BDF13C0C8010E948EE28E3047
:10E8D00019F050F4813059F460E0CE0101960E94A5
:10E8E0007922892B21F0DDCF83518430A8F381E098
:10E8F00090E0BDCF8031F0F48E3098F6813089F20F
:10E900008230E9F06BEE76E289E39FE00F94C91C58
:10E910006EED76E289E39FE00F94C91C698189E37B
:10E920009FE00E9450AC89E39FE00F94CA1B01E076
:10E9300010E086CF8351843008F4B3CFE3CF40E0BA
:10E9400050E0BA01C8010E944BDF60E0C5010E949F
:10E950000C73CDCF4F925F926F927F928F929F9266
:10E96000AF92BF92CF92DF92FF920F931F93CF93FC
:10E97000DF9300D000D01F921F92CDB7DEB7613079
:10E98000710509F482C0FC01628173816115710512
:10E9900009F47BC08C0119821A821B821C821D82A1
:10E9A0001E821F8218868A81807F8A8340E050E21F
:10E9B000CE0101960E94B62160E0CE0101960E9430
:10E9C00079226C01F801828193810E948CDF2B01F6
:10E9D0003C01F8012781308541855285D6010F948D
:10E9E000CF4D2FEF30E040E050E00F94834D4901D0
:10E9F0005A010E94ACBEFF24F39481149104A10437
:10EA0000B10461F06419750986099709FF24F3942C
:10EA1000681579058A059B0508F4F12C4114510409
:10EA20006104710491F1F80187809084A184B2841B
:10EA30000E94ACBEF80181149104A104B10451F00C
:10EA40006419750986099709681579058A059B0572
:10EA500008F449C0A280B3804FEF5FEFBA0180E0B5
:10EA60000E941E6BAB01BC01C5010E944BDFCD288B
:10EA700061F0F80184810E942E5EF801968189136D
:10EA800004C061E0C8010E940C7390E080E0289609
:10EA90000FB6F894DEBF0FBECDBFDF91CF911F91AF
:10EAA0000F91FF90DF90CF90BF90AF909F908F908D
:10EAB0007F906F905F904F900895FF20D9F060E0B5
:10EAC000C8010E940C73F801828193810E94B3E413
:10EAD000892BD9F640E050E0BA01F8018281938198
:10EAE0000E944BDFD2CF84810E942E5EF801968176
:10EAF0008913E3CFCD2849F2F80184810E942E5E6C
:10EB0000F80196818913C1CFF110BFCFBACFAF9270
:10EB1000BF92CF92DF92EF92FF921F93CF93DF933A
:10EB200000D000D0CDB7DEB76C017C0110E08AE0E8
:10EB3000A82EB12C133061F1F701828190E0B0E092
:10EB4000A0E089839A83AB83BC83BE82AD82BE0181
:10EB50006F5F7F4F88E89EE00E94D1FA61EB77E219
:10EB60000F94C91C1F5FFFEFEF1AFF0A143011F753
:10EB700026960FB6F894DEBF0FBECDBFDF91CF91C2
:10EB80001F91FF90EF90DF90CF90BF90AF900895CE
:10EB9000F601858190E0B0E0A0E089839A83AB83A1
:10EBA000BC83BE82AD82BE016F5F7F4F88E89EE06E
:10EBB0000E94D1FA6FEA77E2D3CFFC01DC018D919C
:10EBC0008111FDCF30E020E050E040E08AE09191FB
:10EBD000992301F1443051055CF59E3271F42F3FC9
:10EBE000310509F02CF5DB01A40FB51F12962C930B
:10EBF0004F5F5F4F30E020E0EACF829FD001839FDC
:10EC0000B00D1124292F990F330B205331092A0FEE
:10EC10003B1FDDCF2F3F310509F054F4443051053F
:10EC20003CF4640F751FFB01228381E090E008959E
:10EC300090E080E00895CF93DF931F921F92CDB7AD
:10EC4000DEB78091B1119091B211009711F48DEB64
:10EC500091E1BE016F5F7F4F681B790B072E000C9F
:10EC6000880B990B0F900F90DF91CF9108954F92E1
:10EC70005F926F927F929F92AF92BF92CF92DF92FC
:10EC8000EF92FF920F931F93CF93DF93CDB7DEB731
:10EC900068970FB6F894DEBF0FBECDBFFC01198A8E
:10ECA0001A8A1B8A1C8A1D8A1E8A1F8A188E8A89C4
:10ECB000807F8A8BA081B181109709F47AC08C91F2
:10ECC000882309F476C000811181D8019C91992391
:10ECD00009F443C09D3209F4DAC090539A3028F009
:10ECE0000F5F1F4F11830083EECFC801912CDC0111
:10ECF0006D01C81AD90A2D91022E000C330B205336
:10ED000031092A303105A0F37F016EE270E0C801BD
:10ED10000F946452FC01009709F448C0DC015D01C6
:10ED2000AE1ABF0A11968C911197082E000C990B00
:10ED3000C09711960A9798F38181282F082E000C0E
:10ED4000330B205331092A30310518F480330CF08D
:10ED500057C020E030E0A90108C0912CD12CC12C73
:10ED6000D3CF29E030E040E050E0AAE0B0E00F94DB
:10ED7000C44D2B013C012281822F022E000C990BE5
:10ED8000C0978A30910570F420330CF441C02A33C7
:10ED90000CF042C0092E000CAA0BBB0B480E591EEA
:10EDA0006A1E7B1EA114B10409F088C0CD2809F0A9
:10EDB00073C088E0FE017196DE01199601900D92F4
:10EDC0008A95E1F729853A854B855C856D857E8539
:10EDD0008F85988968960FB6F894DEBF0FBECDBFB9
:10EDE000DF91CF911F910F91FF90EF90DF90CF9027
:10EDF000BF90AF909F907F906F905F904F900895DD
:10EE00008A330CF0AECF032E000C440B550BADCF64
:10EE100080E090E0DC01C2CF89E090E0A0E0B0E0CB
:10EE2000BDCFB8E0CB16D1040CF04DC0C8010F9493
:10EE3000F6459B01AC01A4E6B0E00F94C44D9920C7
:10EE400041F07094609450944094411C511C611C9A
:10EE5000711C2A89207F26602A8B460E571E681E49
:10EE6000791E4D8A5E8A6F8A788E6CE270E0F701B7
:10EE7000808191810F946452009721F4D7011D92F3
:10EE80001C9297CF0196F7019183808392CFC8019E
:10EE90000196992493942BCFC8010F94F645AB01AA
:10EEA000BC01CE0141960E948D2129833A834B8378
:10EEB0005C836D837E838F839887D7CFF3E0AF1613
:10EEC000B1040CF4AECFC8010F94D4452A89207F39
:10EED00027602A8B6D8B7E8B8F8B988FC6CFCF92BE
:10EEE000DF92EF92FF920F931F93CF93DF93EC018A
:10EEF000A881B981109781F18C91882369F10881EB
:10EF00001981F8019081992351F09D3241F090537D
:10EF10009A3028F00F5F1F4F19830883F0CFC80184
:10EF20000F94F6456B017C016CE270E0C8010F9410
:10EF30006452009769F419821882C701B601DF9103
:10EF4000CF911F910F91FF90EF90DF90CF90089598
:10EF5000019699838883F1CFC12CD12C7601EDCF16
:10EF60000097B1F1FC01DB01AC01405F5F4F80E035
:10EF700090812FE9290F263098F497559295907F2C
:10EF80009C9321813FE9320F3630B0F42755922B04
:10EF90009D933296E417F50759F791E08927089574
:10EFA0002FEB290F263010F49753E8CF90539A3067
:10EFB00028F381E090E0E2CF3FEB320F363010F4DF
:10EFC0002753E5CF20532A3010F381E020E0DFCF34
:10EFD00080E008950097D1F0DC011696ED91FC9148
:10EFE0003097A1F080858F70843021F481859285DF
:10EFF000009771F40680F781E02D309739F0808515
:10F000008F70843019F481859285089590E080E0B6
:10F01000089508950895089508950F931F93CF9329
:10F02000DF93EC011D860A811B8170E060E0C8015E
:10F030000E9418E087FD44C08C838C818150853408
:10F0400010F080E28C8361E070E0C8010E9418E05B
:10F0500087FD3BC08D838D818150853410F081E226
:10F060008D8362E070E0C8010E9418E0863490F55C
:10F070008E8363E070E0C8010E9418E09C0121507B
:10F0800031092115344040F59A87898764E070E0A2
:10F09000C8010E9418E0813024E0920700F59C87A7
:10F0A0008B8765E070E0C8010E9418E01816190609
:10F0B000CCF498878F83DF91CF911F910F910895A2
:10F0C00081958C8381E08D87B8CF81958D8381E098
:10F0D0008D87C1CF1E82CDCF1A861986D7CF80E00B
:10F0E00094E0DDCF80E197E2E4CF0895CF93DF9302
:10F0F00000D000D01F921F92CDB7DEB7E2E7FEE04E
:10F10000128A118A80E090E19587848784E890E0F4
:10F11000948B838B81E0868780E090E2908B878759
:10F1200087E7858B1C821B8285EC92E09A8389831A
:10F13000FE83ED838FEF9FEF98878F836BE87EE1EF
:10F1400088E89EE00F94C91C6091270A7091280AF4
:10F15000CE0101960E94AAB282E79EE00E94ADDA3B
:10F160006BE77EE188E89EE00F94C91C88E89EE08A
:10F170000F94CA1B0E946AC928960FB6F894DEBF86
:10F180000FBECDBFDF91CF910895EF92FF921F93F5
:10F19000CF93DF93192F7B01C82FD92FD7FF03C03F
:10F1A000D195C195D10961E08C2F0E9431BC82E0DC
:10F1B000E816F10499F460E08C2F0E9403BC63E729
:10F1C0007EE189E39FE00F94C91C89E39FE0DF9112
:10F1D000CF911F91FF90EF900D94CA1B612FEF28E4
:10F1E00051F46095661F6627661F8C2F0E9403BC32
:10F1F0006FE67EE1E6CF661F6627661F8C2F0E94B2
:10F2000003BC6AE67EE1DDCFBF92CF92DF92EF9240
:10F21000FF920F931F93CF93DF93CDB7DEB72E9757
:10F220000FB6F894DEBF0FBECDBF2091FC10309119
:10F23000FD10232B09F4A6C02091FB102111A2C0C0
:10F240007C018091FB108F5F8093FB108091FA10FE
:10F250008F5F8093FA100E94ACBE0091370A109124
:10F26000380A2091390A30913A0A601B710B820BDF
:10F27000930B6B3071058105910508F479C083E02B
:10F28000E816F104A9F00E94ACBE0091330A109177
:10F29000340A2091350A3091360A601B710B820BBB
:10F2A000930BBB24B394643671058105910508F472
:10F2B000B12CE091FC10F091FD1006811781011531
:10F2C0001105C1F1F80180858F70863079F51987B5
:10F2D000088770E060E0CE0108960F94B901B7018D
:10F2E000CE0108960F94EA0469EC75E0C8010E940B
:10F2F000C6ABFC01892BD1F090859F709550923060
:10F30000A8F4C680D780C114D10481F0DA82C98202
:10F31000B801CE0101960F94B901B701CE01019653
:10F320000F94EA04F601C280D380EDCFF801028188
:10F330001381C5CFF3E0EF16F10451F00E94ACBE8B
:10F340006093370A7093380A8093390A90933A0A87
:10F35000BB2051F00E94ACBE6093330A7093340A14
:10F360008093350A9093360A1092A60F1092A70F39
:10F370008091FA1081508093FA108091FB10815097
:10F380008093FB102E960FB6F894DEBF0FBECDBF54
:10F39000DF91CF911F910F91FF90EF90DF90CF9071
:10F3A000BF900895A8950F943E2382E090E00E94BC
:10F3B00004790E94714C039724F00E94B0C40E940B
:10F3C000D4CC0D940D0FA89582E090E00C940479B4
:10F3D0008091F9108F5F8093F910A89583E090E0F9
:10F3E0000E9404790F943E238091F91081508093FC
:10F3F000F910089568E47EE188E89EE00F94C91C46
:10F4000065E37EE188E89EE00F94C91C67E27EE137
:10F4100088E89EE00F94C91C6FE17EE188E89EE0D9
:10F420000F94C91C88E89EE00F94CA1B6FE07EE130
:10F4300088E89EE00F94C91C63E07EE188E89EE0C6
:10F440000F94C91C66EF7DE188E89EE00F94C91C0B
:10F4500061EE7DE188E89EE00F94C91C62ED7DE1DC
:10F4600088E89EE00F94C91C6AEC7DE188E89EE084
:10F470000F94C91C69EB7DE188E89EE00F94C91CDC
:10F4800063E97DE188E89EE00F94C91C66E87DE1B0
:10F4900088E89EE00F94C91C6CE77DE188E89EE057
:10F4A0000F94C91C6DE67DE188E89EE00F94C91CAD
:10F4B00065E67DE188E89EE00F94C91C69E57DE181
:10F4C00088E89EE00F94C91C6FE37DE188E89EE028
:10F4D0000F94C91C60E27DE188E89EE00F94C91C8E
:10F4E0006BE07DE188E89EE00F94C91C6EEF7CE143
:10F4F00088E89EE00F94C91C60EF7CE188E89EE0FC
:10F500000F94C91C64EE7CE188E89EE00F94C91C4E
:10F510006CED7CE188E89EE00F94C91C61ED7CE114
:10F5200088E89EE00F94C91C64EC7CE188E89EE0CA
:10F530000F94C91C6CEB7CE188E89EE00F94C91C19
:10F5400061EB7CE188E89EE00F94C91C62EA7CE1F3
:10F5500088E89EE00F94C91C69E97CE188E89EE098
:10F560000F94C91C6BE87CE188E89EE00F94C91CED
:10F570006DE77CE188E89EE00F94C91C61E77CE1BF
:10F5800088E89EE00F94C91C69E67CE188E89EE06B
:10F590000F94C91C66E57CE188E89EE00F94C91CC5
:10F5A0006CE47CE188E89EE00F94C91C88E89EE04A
:10F5B0000D94CA1BCF93DF93EC016BE576E289E3F0
:10F5C0009FE00F94C91C66E576E289E39FE00F9403
:10F5D000C91C6C817D8189E39FE00E9457AC60E586
:10F5E00076E289E39FE00F94C91C89E39FE00F94C2
:10F5F000CA1B61E08C810E9431BC6E818C810E94AB
:10F6000003BC8A819B81009729F040E050E0BA0159
:10F610000E944BDFE881F9810484F585E02D62E0EA
:10F62000CE0119958A819B81009799F00E94B3E4DD
:10F630001816190674F40A80DB81C02D4FEF5FEFB6
:10F64000BA0180E00E941E6BAB01BC01CE010E949A
:10F650004BDF81E090E0DF91CF910895CF93DF936E
:10F66000EC016DE276E289E39FE00F94C91C6C81A6
:10F670007D8189E39FE00E9457AC6BE276E289E3EB
:10F680009FE00F94C91CEA81FB810280F381E02D89
:10F690006081718189E39FE00F94721C65E276E2DC
:10F6A00089E39FE00F94C91C89E39FE00F94CA1B74
:10F6B0008A819B81892B09F451C08C819D81892B82
:10F6C00009F04CC0E881F981008CF18DE02DCE016C
:10F6D00019958130910529F0029759F061E08C81EC
:10F6E0001AC063E070E0CE010F94B41061E00E9494
:10F6F00031BC61E08C810E9431BC61E070E0CE01E0
:10F700000F94B41061E00E9431BC62E070E0CE0161
:10F710000F94B41061E00E9431BC8091A100887FF9
:10F720008093A10080919100887F809391008091C7
:10F73000A10082608093A1008091910082608093FB
:10F740009100E881F9810484F585E02D62E0CE0125
:10F75000199581E090E0DF91CF91089590E080E0ED
:10F76000FACF2F923F924F925F926F927F928F9239
:10F770009F92AF92BF92CF92DF92EF92FF920F9340
:10F780001F93CF93DF93CDB7DEB760970FB6F89492
:10F79000DEBF0FBECDBF9A838983DC011496ED9145
:10F7A000FC91309709F45DC18680978081149104A3
:10F7B00009F41DC1D401ED91FC91309709F413C1F6
:10F7C0008081882309F40FC12FEF3FEFA90169E77A
:10F7D00075E0C4010E94A06322E030E040E050E008
:10F7E00066E577E0C4010E94A0632FEF3FEFA90117
:10F7F00068ED76E0C4010E94A06360E776E0C40192
:10F800000E94C6AB988B8F87009709F4ECC0FC016F
:10F8100080858F70853009F0E6C0CF010E94E1AC91
:10F82000833008F4E0C020E030E040EA51E461EECB
:10F8300076E0C4010E946B638C010E94215F20E08E
:10F8400030E040EA51E46DE775E0C4010E946B636B
:10F850006C010E94215F20E030E040E050EC65EE5A
:10F8600076E0C4010E946B637C010E94215F20E06E
:10F8700030E040E85FE370E060E08F8598890E94A7
:10F88000E25F2B013C0120E030E0A9010F94394CEC
:10F89000B12C87FF06C077FA709477F87094BB2478
:10F8A000B39420E030E0A90161E070E08F85988991
:10F8B0000E94E25F6B837C838D839E8320E030E037
:10F8C000A90162E070E08F8598890E94E25F6F83F2
:10F8D000788789879A8720E030E040EA50E463E047
:10F8E00070E08F8598890E94E25F6B877C878D87A7
:10F8F0009E878CE390E00F940B441C019801275FD6
:10F900003F4FA701475F5F4FB601675F7F4F1F9271
:10F91000BF92FA85FF9389858F9398859F93AF81D6
:10F92000AF93AB80BC80CD80DE8083017201C101CA
:10F930000F947420C101032C000CAA0BBB0BEF85A4
:10F94000F88981879287A387B48761E070E0C1015D
:10F950000F94D51F20E030E04AE754E46B857C85A6
:10F960008D859E850F949F4C0F940B4FAF85B88962
:10F9700019968D919C910F94272060E873E289E39A
:10F980009FE00F94C91CB301A20189E39FE00E948C
:10F99000A2B068EE76E089E39FE00F94721C4B8181
:10F9A0005C816D817E8189E39FE00E94A2B06CEE54
:10F9B00076E089E39FE00F94721C3F81288599854A
:10F9C0008A85432F522F692F782F89E39FE00E9469
:10F9D000A2B089E39FE00F94CA1B0F900F900F9085
:10F9E0000F900F900F90F40182809380DFCE65E737
:10F9F00073E289E39FE00F94C91C89E39FE00F94B1
:10FA0000CA1B40E050E0BA01A981BA8112968D91DB
:10FA10009C910E944BDFA981BA81ED91FC911197D5
:10FA20000484F585E02D62E0CD01199581E090E038
:10FA300060960FB6F894DEBF0FBECDBFDF91CF91B9
:10FA40001F910F91FF90EF90DF90CF90BF90AF90FC
:10FA50009F908F907F906F905F904F903F902F90EE
:10FA6000089561E673E289E39FE00F94C91C89E37E
:10FA70009FE00F94CA1B90E080E0DACFCF93DF9332
:10FA8000EC010E940D7860EF76E089E39FE00F942F
:10FA9000CE1B61E08C810E9431BC61E08D810E94AF
:10FAA00031BC6D858C810E9403BC6D858D810E9467
:10FAB00003BC60E08E810E9431BC40E050E0BA019E
:10FAC0008A819B810E944BDF40E050E061E070E062
:10FAD0008A819B810E94C2E040E050E062E070E0D9
:10FAE0008A819B810E94C2E0E881F9810484F585C6
:10FAF000E02D62E0CE01199582E08093000281E062
:10FB000090E0DF91CF9108956F927F928F929F92B4
:10FB1000AF92BF92CF92DF92EF92FF920F931F931B
:10FB2000CF93DF933C01DC0114968D919C91159746
:10FB3000892B71F41296CD91DC9184E190E00F94C1
:10FB40000B44BC01CE010E9408DFE3019D838C833E
:10FB5000F301C481D581209769F461E770E282E9FD
:10FB60009EE00F94C91C82E99EE00F94CA1B90E0AE
:10FB700080E0A7C24FEF5FEFBA0180E00E941E6BEA
:10FB80006E837F8388879987D3011496ED90FC90CC
:10FB90001597E114F104D1F01296ED91FC91309794
:10FBA000A9F0C481D581209789F088858F70853030
:10FBB00069F4CE010E94E1AC823040F000912A0A43
:10FBC00010912B0A0115110509F08CC064E370E255
:10FBD00082E99EE00F94C91C61E070E0E3018C8132
:10FBE0009D81892B11F470E060E082E99EE00E9423
:10FBF00057AC62E370E282E99EE00F94C91C61E0B9
:10FC000070E0F30182819381892B11F470E060E050
:10FC100082E99EE00E9457AC60E370E282E99EE0D8
:10FC20000F94C91CD3011296ED91FC9161E070E034
:10FC300084819581892B11F470E060E082E99EE077
:10FC40000E9457AC6EE270E282E99EE00F94C91CFC
:10FC5000E301EA81FB810480F581E02D80858F70CE
:10FC600061E070E0853011F470E060E082E99EE0D0
:10FC70000E9457AC6CE270E282E99EE00F94C91CCE
:10FC8000D3011296ED91FC91848195810E94E1ACA3
:10FC900061E070E0823010F070E060E082E99EE0A8
:10FCA0000E9457AC82E99EE00F94CA1B69E470E29F
:10FCB00082E99EE00F94C91C82E99EE00F94CA1B62
:10FCC000D301ED91FC910484F585E02D61E0C30141
:10FCD0001995E301E881F9810084F185E02DC301E4
:10FCE000199545CF61E0CE010E943EACEC018885BC
:10FCF0008F70843029F469857A856115710539F42E
:10FD000064E170E282E99EE00F94C91CCBCFC80188
:10FD10000E94C6AB8C01009769F462EF7FE182E933
:10FD20009EE00F94C91C69857A8582E99EE00F9454
:10FD3000721CB8CF6CEF76E00E94C6AB009709F456
:10FD4000D2C0EC0128852F70243009F0CCC0C984C2
:10FD5000DA84D0E0C0E0C114D10409F4B7C0BE0118
:10FD6000625B704EC6010F944446892B09F0A9C00E
:10FD7000FE01EE5AF04E25913491922F832FF70118
:10FD80009283838363E077E0C8010E94C6ABE301FE
:10FD9000EC81FD81009709F4AEC0DC0118962C912E
:10FDA00018972F70223009F0A6C019968D919D9159
:10FDB0000D90BC91A02D0097A105B10509F49BC041
:10FDC0009183808340815181052E000C660B770B57
:10FDD000228187EB9BE00F94D51D68E077E0C80196
:10FDE0000E94C6AB7C01F301C481D581009709F460
:10FDF00088C0DC0118968C918F70863009F081C024
:10FE00006DE077E0C7010E94C6AB9B878A8762E1FD
:10FE100077E0C7010E94C6AB9D878C8766E177E0DB
:10FE2000C7010E94C6AB9F878E876CE177E0C70150
:10FE30000E94C6AB998B888B61E277E0C7010E9474
:10FE4000C6AB009709F45AC0FC01818592859D8359
:10FE50008C8367E277E0C8010E94C6AB9B8B8A8BDC
:10FE6000892B09F40CC16CED7FE189E39FE00F94CD
:10FE7000C91C89E39FE00F94CA1BD3011496ED912E
:10FE8000FC910288F389E02DC681D781209709F47F
:10FE900041C06BE277E0CE010E94C6AB009769F0EB
:10FEA000FC0120852F70213041F48185882329F0C1
:10FEB00068817981C3010E942C660A80DB81C02D94
:10FEC000E5CF2696C834D10509F045CF61E37FE13F
:10FED00089E39FE00F94C91C89E39FE00F94CA1B3C
:10FEE00096E080E04CCF86E090E0D70113969C939B
:10FEF0008E93129747CF80E895E262CF88EE93E029
:10FF0000A6CF1B861A8688EE93E09D838C831D8680
:10FF10001C869FCF66EC7FE189E39FE00F94C91CAC
:10FF200089E39FE00F94CA1BD3011496ED91FC91D5
:10FF30000288F389E02DE680F780E114F10409F4EA
:10FF400078C066E976E0C7010E94C6AB009709F465
:10FF500065C064E377E00E94C6AB8C01009709F4AA
:10FF60005DC0EC0188858F70823009F04BC0C98478
:10FF7000DA84D3011496ED91FC910288F389E02D87
:10FF8000309709F453C0C681D78146010D2C000C6F
:10FF9000AA08BB08209709F449C068E377E0CE01BE
:10FFA0000E94C6AB0097F1F1FC0120852F70223032
:10FFB000C9F581859285A385B48588159905AA051B
:10FFC000BB0581F565EA7FE189E39FE00F94C91CD9
:10FFD0006881798189E39FE00F94721C66E97FE173
:10FFE00089E39FE00F94C91CB60189E39FE00E945A
:10FFF00057AC89E39FE00F94CA1B68817981C301E4
:020000021000EC
:100000000E942C66F80180858F70843039F4D80105
:1000100019966D917C91C3010E942C66E701EA80DC
:10002000FB808BCF0A80DB81C02DB4CF70E060E015
:10003000E6CF6CEA7FE189E39FE00F94C91C89E376
:100040009FE00F94CA1BD3011296ED91FC9162E0E0
:10005000848195810E943EAC009789F0FC01C681A5
:10006000D781209761F0CE010E94415F882319F06B
:10007000CE010E945ABA0A80DB81C02DF2CF6CE516
:1000800070E288E89EE00F94C91CD3011296ED91AE
:10009000FC910280F381E02D6081718188E89EE00F
:1000A0000F94721C88E89EE00F94CA1BE301E8815C
:1000B000F9810484F585E02D62E0C301199581E0A2
:1000C00090E0DF91CF911F910F91FF90EF90DF9023
:1000D000CF90BF90AF909F908F907F906F9008953A
:1000E000CF93DF93EC016CEC7EE189E39FE00F940A
:1000F000C91CEA81FB810280F381E02D608171815E
:1001000089E39FE00F94721C89E39FE00F94CA1B60
:10011000E881F9810484F585E02D62E0CE0119952E
:1001200081E090E0DF91CF910895DC01ED91FC91A9
:100130000484F585E02D62E0199581E090E0089552
:100140002F923F924F925F926F927F928F929F92E7
:10015000AF92BF92CF92DF92EF92FF920F931F93D5
:10016000CF93DF93CDB7DEB7CB57D1090FB6F89455
:10017000DEBF0FBECDBFE296EFAEE297E396FFAED5
:10018000E397E4960FAFE497E5961FAFE597E69601
:100190002FAFE697E7963FAFE797E8964FAFE89720
:1001A000E9965FAFE9970097B9F124012B2CEC9603
:1001B000AFAEEC97EB96DFAEEB97EA96CFAEEA9751
:1001C000362E8C0180911E02893020F480911D0210
:1001D0008930C0F0C8010E94EBB37C01892B91F0FB
:1001E0006CE377E089E39FE00F94721CB70189E329
:1001F0009FE00F94721C89E39FE00F94CA1BC70114
:100200000F94A744F80180858F70843009F45FC192
:1002100028F4882309F464C180E02FC0853009F4F4
:1002200046C08630C9F769EC75E0C8010E94C6ABCC
:100230003C01009709F476C0912C812CB12CA12CA3
:10024000D12CC12CE296EFACE297E396FFACE3979A
:10025000E4960FADE497E5961FADE597E6962FADD2
:10026000E697E7963FADE797E8964FADE897E996B2
:100270005FADE997632D0E94A080C558DF4F0FB690
:10028000F894DEBF0FBECDBFDF91CF911F910F91CC
:10029000FF90EF90DF90CF90BF90AF909F908F90A6
:1002A0007F906F905F904F903F902F900895809136
:1002B000FA108F5F8093FA10668077806114710462
:1002C00059F14201EC96AFACEC97B22CEA96CFAC68
:1002D000EA97EB96DFACEB97E296EFACE297E3960A
:1002E000FFACE397E4960FADE497E5961FADE59775
:1002F000E6962FADE697E7963FADE797E8964FADC8
:10030000E897E9965FADE997632DC3010E94A0804D
:10031000F30162807380D2CF8091FA108150809374
:10032000FA107ACF62E477E0C8010E94C6AB2C01D4
:1003300067E477E0C8010E94C6AB7C016CE477E01B
:10034000C8010E94C6AB332039F0F1E03F1609F432
:100350009FC0D12CC12C0CC060E577E0C8010E9481
:10036000C6AB3C0165E577E0C8010E94C6AB6C01F5
:100370006114710409F43801C114D10409F468014D
:100380004114510431F4EA964FACEA97EB965FAC16
:10039000EB97E114F10421F4EC96EFACEC97F22C1E
:1003A0006114710409F4A5C0F30180858F70843055
:1003B00009F09FC061847284C114D10409F49CC007
:1003C000F60180858F70843009F096C0C184D28494
:1003D00010E000E04114510409F4F3C06114710409
:1003E00009F4B1C069E078E289E39FE00F94C91C89
:1003F000F2016185728589E39FE00F94721C64E0CD
:1004000078E289E39FE00F94C91CB30189E39FE080
:100410000F94721C89E39FE00F94CA1BCE018F5882
:100420009F4F0E94AE26E114F10409F0D3C0F201FF
:1004300080858F70843009F083C140910011509104
:10044000011161857285CE0101960E94DAE2CE012A
:1004500001960E94FBDE8823B1F00E941B766B019F
:10046000683C71050CF083C063EC77E282E99EE0A2
:100470000F94C91CB60182E99EE00E9457AC82E944
:100480009EE00F94CA1BCE0101960E9477E358C1EB
:100490006AE577E0C8010E94C6AB3C016FE577E0F2
:1004A000C8010E94C6AB6C016114710409F04AC115
:1004B00060E577E0C8010E94C6AB3C01C114D104DD
:1004C00009F450CF892B09F05BCF380159CFD12CDB
:1004D000C12C712C612CF12CE12C512C412C48CFDA
:1004E000D12CC12C712C612CF12CE12C512C412CE4
:1004F00047CF712C612C60CF00E020E030E340E179
:1005000050E0BE016F597F4FCE018F589F4F0E9420
:100510008E246C01E4960FADE49710E001151105EF
:1005200009F058CFE2968FADE297811109C0E396AA
:100530008FADE3978F7009F44DCF02E010E04ACF02
:1005400001E010E047CF6AEF77E289E39FE00F9484
:10055000C91CF2016185728589E39FE00F94721CCA
:1005600065EF77E289E39FE00F94C91C57CF6114D0
:10057000710431F0B301CE0101960E942AB483CFF9
:10058000A12CC12CF12CE12CE2960FADE297E39661
:100590001FADE397E4962FADE497E5963FADE59761
:1005A000E6964FADE697E7965FADE797E8966FADB5
:1005B000E897E9967FADE997CE0101960E94C3E5E1
:1005C00062CFE114F10409F4BBC0C114D10409F4F1
:1005D000B7C004C0C114D10409F429CFF701808544
:1005E0008F70843009F0A8C08185928525961FAE52
:1005F0001EAE259748EE53E060E070E029964CAFC0
:100600005DAF6EAF7FAF29972BED32E023963FAF02
:100610002EAF23972F969FAF8EAF2F9761961FAE69
:100620001EAE619763961FAE1EAE639765961FAEB2
:100630001EAE659767961FAE1EAE679769961FAF91
:100640000EAF69976A961FAE6A9740E450E0BE010C
:100650006F5F7F4FCE018F5B9F4F0E9495AD21E072
:1006600030E02C0F3D1F820F931FFC0110826DEEB6
:1006700077E289E39FE00F94C91CF70161857285D9
:1006800089E39FE00F94721C64E677E089E39FE0C2
:100690000F94721CBE016F5F7F4F89E39FE00F9440
:1006A000721C68EE77E289E39FE00F94C91CB601E3
:1006B00089E39FE00F94721C89E39FE00F94CA1BAB
:1006C0000E94E4AB8823C1F18091F910811134C0FC
:1006D0006FE270E0CE0101960F946452892B51F4C1
:1006E000F7012185328543E050E060E4CE010196B8
:1006F0000E94787261EE77E289E39FE00F94C91C53
:10070000BE016F5F7F4F89E39FE00F94721C6CED19
:1007100077E289E39FE00F94C91CB60189E39FE06B
:100720000F94721C89E39FE00F94CA1B41E0B6014D
:10073000CE0101960E947ABF4114510409F077CE90
:1007400081E09BCD892B09F01BCE0CCE8F929F921E
:10075000AF92BF92CF92DF92EF92FF920F931F93CF
:10076000CF93DF9300D000D01F921F92CDB7DEB79A
:10077000DC011296ED91FC91309709F468C0248158
:100780003581232B09F463C08C01662309F472C000
:100790000E946D62E62EB72E6C01D8011296ED9183
:1007A000FC910280F381E02D6081718182E99EE0FD
:1007B0000F94721C69EB75E282E99EE00F94C91CEC
:1007C00082E99EE00F94CA1B20E030E0A9016E2D63
:1007D0007B2DC6010F94414F87FD39C06DEA75E24C
:1007E00082E99EE00F94C91C4E2D5B2DB60182E973
:1007F0009EE00E94A2B082E99EE00F94CA1BD8013D
:100800001296ED91FC9161E0848195810E943EAC4D
:1008100019821A821B821C822A81207F2760F22E75
:100820002E2D4E2D5B2DB6014D835E836F83788711
:10083000912C812CB12CA12CD12CC12CE9800B81C5
:100840001C813E814F8158856FEF0E94A0802896C1
:100850000FB6F894DEBF0FBECDBFDF91CF911F91D1
:100860000F91FF90EF90DF90CF90BF90AF909F904F
:100870008F9008950280F381E02D6081718188E876
:100880009EE00F94721C66EC75E288E89EE00F947F
:10089000C91C88E89EE028960FB6F894DEBF0FBE0C
:1008A000CDBFDF91CF911F910F91FF90EF90DF901F
:1008B000CF90BF90AF909F908F900D94CA1B4F9296
:1008C0005F926F927F928F929F92AF92BF92CF92E0
:1008D000DF92EF92FF920F931F93CF93DF93CDB7E9
:1008E000DEB7E8970FB6F894DEBF0FBECDBF09ABF9
:1008F0001AAB2BAB3CAB4DAB5EAB6FAB78AFDC0157
:100900001496ED91FC91309719F490E080E0C9C005
:1009100020813181232BC9F33C01DC01ED91FC9155
:100920000284F385E02D1995029779F78BA9E82EBB
:10093000F12C19A9112321F0E114F10409F431C1BA
:10094000823009F4D7C0A8F4882309F4D3C08130D9
:10095000A9F069ED75E289E39FE00F94C91CB70126
:1009600089E39FE00E9457AC89E39FE00F94CA1B84
:10097000CCCF833009F447C0893059F7D3011296A0
:10098000ED91FC9161E0848195810E943EAC2C0147
:1009900019A61AA61BA61CA61DA61EA61FA618AA47
:1009A0008AA5807F8AA719A761E0CE0189960E9457
:1009B000492129A33AA34BA35CA36DA37EA38FA3D4
:1009C00098A71150163108F0FDC1E12FF0E08827FB
:1009D000E351FB478F4F0D940E4E1786D585E28667
:1009E000E286E286E286E286E286E2864686A6869F
:1009F000E286E28617861786E286E286E286178618
:100A00001786178617868AA98F7009F47ECFCE01C4
:100A1000C1960E949823D3011496ED91FC916683B0
:100A20007783808791876FE176E289E39FE00F9477
:100A3000C91CD3011296ED91FC910280F381E02D47
:100A40006081718189E39FE00F94721C61E176E21D
:100A500089E39FE00F94C91CD3011496ED91FC919A
:100A6000468157816085718589E39FE00E94A2B02D
:100A700089E39FE00F94CA1BF301E480F5800E9494
:100A8000ACBED70152966D937D938D939C935597F1
:100A9000D3011496ED91FC918689811119C081E0F2
:100AA00090E0E8960FB6F894DEBF0FBECDBFDF91A1
:100AB000CF911F910F91FF90EF90DF90CF90BF905B
:100AC000AF909F908F907F906F905F904F90089520
:100AD000168A60E0C3010E94A683D3011496ED91AB
:100AE000FC9180E090E0A0E0B0EC86879787A08B37
:100AF000B18BD5CF8AA98F7009F407CFCE01C196EB
:100B00000E949823D3011496ED91FC91628773871C
:100B1000848795876BE076E289E39FE00F94C91C98
:100B2000D3011296ED91FC910280F381E02D60815A
:100B3000718189E39FE00F94721C60E076E289E3A3
:100B40009FE00F94C91CD3011496ED91FC9142854E
:100B500053856485758589E39FE00E94A2B089E38F
:100B60009FE00F94CA1BD3011296ED91FC9162E0B5
:100B7000848195810E943EAC009709F490CF912C1E
:100B8000812CB12CA12CD12CC12CE9A8FAA80BA93D
:100B90001CA92DA93EA94FA958AD6FEF0E94A080B6
:100BA0007ECFEE24E394F12CE9CE8091FE1090915B
:100BB000FF100597F1F019821A821B821C821D8298
:100BC0001E821F8218868A81807F8A836BE0CE0115
:100BD00001960E946B21912C812CB12CA12CD12C3F
:100BE000C12C79018A019B01AC016FEFC2010E9407
:100BF000A080912C812CB12CA12CD12CC12CE9A44A
:100C0000FAA40BA51CA52DA53EA54FA558A96FEFCD
:100C1000C2010E94A08030E020E040E050E460E0AB
:100C200070E0F301828193810E94C43738CF19822A
:100C30001A821B821C821D821E821F8218868A8154
:100C4000807F8A8340E051E060E070E0D30112963B
:100C50008D919C910E9414E1672B682B692BA1F068
:100C60006BE0CE0101960E946B21912C812CB12C5E
:100C7000A12CD12CC12C79018A019B01AC016FEF11
:100C8000C2010E94A080BBCF6AE0EBCF8091FE1032
:100C90009091FF10059791F061E0D30112968D912C
:100CA0009C910E946FE230E020E040E050E160E083
:100CB00070E0F301828193810E94C43740E050E0EC
:100CC00061E070E0D30112968D919C910E94EBE05F
:100CD000912C812CB12CA12CD12CC12CE9A4FAA4EB
:100CE0000BA51CA52DA53EA54FA558A96FEFC201C8
:100CF0000E94A080D301ED91FC910288F389E02D40
:100D0000C3011995892B09F4E8CE19821A821B8236
:100D10001C821D821E821F8218868A81807F8A83A0
:100D200061E0CE0101960E946B2129873A874B87AB
:100D30005C876D877E878F87988B79018A019B01FD
:100D4000AC016FEFC2010E94A080C7CE912C812C14
:100D5000B12CA12CD12CC12CE9A4FAA40BA51CA563
:100D60002DA53EA54FA558A96FEFC2010E94A080F6
:100D7000D301ED91FC910288F389E02DC30119950F
:100D8000892B09F08CCE19861A861B861C861D8637
:100D90001E861F86188A8A85807F8A8762E0CE0138
:100DA00009960E946B2129833A834B835C836D8370
:100DB0007E838F83988779018A019B01AC016FEF55
:100DC000C201ECCE6EEE75E289E39FE00F94C91C80
:100DD00069A989E39FE00E9450AC89E39FE00F94EA
:100DE000CA1BB7CD2F923F924F925F926F927F9224
:100DF0008F929F92AF92BF92CF92DF92EF92FF922B
:100E00000F931F93CF93DF93CDB7DEB764970FB6E1
:100E1000F894DEBF0FBECDBF1C01DC0114968D918E
:100E20009C911597892B99F41296ED91FC91FA8378
:100E3000E98389E190E00F940B44BC0189819A8198
:100E40000E9408DFD10115969C938E931497F101AF
:100E5000048115810115110569F46EE475E282E9DA
:100E60009EE00F94C91C82E99EE00F94CA1B90E09B
:100E700080E092C3D8011D921C920280F381E02D84
:100E8000FC8BEB8B309791F0848195819A838983D9
:100E9000009761F0DC0118968C9118978F7085305F
:100EA00029F4CD010E94E1AC811186C064E175E2B4
:100EB00082E99EE00F94C91C61E070E0F101848139
:100EC0009581892B11F470E060E082E99EE00E9438
:100ED00057AC62E175E282E99EE00F94C91C61E0C3
:100EE00070E0D10112968D919C91892B11F470E0E4
:100EF00060E082E99EE00E9457AC60E175E282E921
:100F00009EE00F94C91CD1011296ED91FC9161E015
:100F100070E084819581892B11F470E060E082E9B2
:100F20009EE00E9457AC6EE075E282E99EE00F946D
:100F3000C91CD1011296ED91FC910480F581E02D40
:100F400080858F7061E070E0853011F470E060E0C2
:100F500082E99EE00E9457AC6CE075E282E99EE077
:100F60000F94C91CD1011296ED91FC918481958159
:100F70000E94E1AC61E070E0823010F070E060E06F
:100F800082E99EE00E9457AC82E99EE00F94CA1B62
:100F900068E275E282E99EE00F94C91C82E99EE056
:100FA0000F94CA1BD101ED91FC910484F585E02DCD
:100FB00061E0C10119955BCF60E089819A810E944F
:100FC0003EAC9F838E83009729F0FC0180858F7053
:100FD000853039F062EF74E282E99EE00F94C91C1B
:100FE000D3CF8E819F810E94E1AC8150883008F080
:100FF000A3C1E82FF0E08827EF5FF7478F4F0D94EC
:101000000E4E6D894389168991887988798862881E
:10101000098867E08E819F810E943EACFC0190852B
:101020009F70933009F041C041845284638474847A
:10103000F1E0FD8366E08E819F810E943EACFC0161
:1010400090859F70933009F045C081859285A38576
:10105000B48589839A83AB83BC8391E09D8364E0EC
:101060008E819F810E943EACFC0190859F709330E1
:1010700009F050C061857285838594850F94124F65
:101080004B0163E08E819F810E943EACFC01808514
:101090008F70833009F060C081859285A385B48507
:1010A0008A879B87AC87BD8764C0923059F461857D
:1010B0007285838594850F94404C2B013C0181E01F
:1010C0008D83B8CF412C512C8FE7682E83E4782E86
:1010D0001D82B0CF9230C9F4618572858385948575
:1010E0000F94404C69837A838B839C83A1E0AD830A
:1010F000B6CF412C512CBFE76B2EB3E47B2E198267
:101100001A821B821C821D82AACF19821A821B821C
:101110001C82A5CF9230C1F481849284A384B484CC
:10112000B0CFF0EC8F2EF7E29F2EF9E0AF2EB12C6E
:10113000412C512CAFE76A2EA3E47A2E19821A8231
:101140001B821C821D829DCFE0EC8E2EE7E29E2E3C
:10115000E9E0AE2EB12C95CF823009F082C06185D6
:101160007285838594850F94404C6A877B878C8732
:101170009D8762E08E819F810E943EACFC0180854C
:101180008F70833009F072C091859E87A285AF87EA
:10119000B385B88B8485898B61E08E819F810E94A5
:1011A0003EACFC0180858F70833009F08BC0C18418
:1011B000D284E384F48460E08E819F810E943EACFF
:1011C000FC0180858F70833009F0A9C081859285EC
:1011D000A385B4858E839F83A887B98720E030E0FC
:1011E000A9016E817F81888599850F94394C87FF8D
:1011F000D0C08E819F81A885B985B0588E839F838A
:10120000A887B98791E09A8BAB89BC891696ED9136
:10121000FC9180858F70823009F4BDC0833009F461
:10122000D4C180E090E0A0EAB1E4D3C160EC862EA6
:1012300067E2962E69E0A62EB12C80E090E0A0EA4D
:10124000B0E48A879B87AC87BD87412C512C7FE710
:10125000672E73E4772E19821A821B821C821D82EC
:1012600088CF80E090E0A0EAB0E41ACF823029F580
:1012700061857285838594850F94404C6E877F8746
:10128000888B998B89CF40EC842E47E2942E49E0DD
:10129000A42EB12C80E090E0A0EAB0E48A879B877E
:1012A000AC87BD87412C512C5FE7652E53E4752E2A
:1012B00019821A821B821C821D821E861F86188A32
:1012C000198A6ACF823039F5618572858385948564
:1012D0000F94404C6B017C016ECF20EC822E27E2F4
:1012E000922E29E0A22EB12C80E090E0A0EAB0E49A
:1012F0008A879B87AC87BD87412C512C3FE7632EA3
:1013000033E4732E19821A821B821C821D821E8670
:101310001F86188A198AC12CD12C76014CCF8230B5
:1013200091F561857285838594850F94404C6E8319
:101330007F838887998752CF80EC882E87E2982E0A
:1013400089E0A82EB12C80E090E0A0EAB0E48A8782
:101350009B87AC87BD87412C512C9FE7692E93E476
:10136000792E19821A821B821C821D821A8A1E867D
:101370001F86188A198AC12CD12C7601CE82DF8271
:10138000E886F98641CF1A8A1E821F82188619863E
:101390003BCF1A8A39CF61857285838594850F94F6
:1013A000404CF8016287738784879587D801169629
:1013B0001D921D921D921C921997F80112821382A0
:1013C000148215820E94ACBED80152966D937D9313
:1013D0008D939C935597D1011496ED91FC9181E0EA
:1013E000868B908E878A61E0C1010E94A683F101FD
:1013F00004811581D8018D919C9169ED74E2892B4E
:1014000009F0EACD8CE390E00F940B449C8B8B8B1E
:101410009801265F3F4FA8014E5F5F4FB8016A5F9A
:101420007F4F1F92BA89BF93E989EF93F889FF93A1
:101430008F858F939E859F9356016701EE80FF8075
:10144000088519858B899C890F947420D101149685
:10145000ED91FC918B899C89918380830F900F90F3
:101460000F900F900F900F90009709F491CD61E0CD
:1014700070E00F94D51FD1011496ED90FC90BD81C2
:10148000BB2309F44AC0A301920169817A818B814F
:101490009C810F94414F87FF40C0F7010190F0817C
:1014A000E02DFF83EE8389819A81AB81BC8182AB81
:1014B00093ABA4ABB5AB46AA57AA60AE71AE82ADF2
:1014C000882359F1068D178DF80180809180A280C4
:1014D000B380A5019401C301B2010F94394C87FF79
:1014E0007EC0D8014D925D926D927C921397AE8131
:1014F000BF8196968D909D90AD90BC909997A501D7
:101500009401C301B2010F94394C87FF7DC0EE8175
:10151000FF8146A257A260A671A620E030E04AE70C
:1015200054E46A857B858C859D850F949F4C0F9430
:101530000B4FD7018D919C910F9427206AE375E2A0
:1015400088E89EE00F94C91CD1011296ED91FC91A0
:101550000280F381E02D6081718188E89EE00F9424
:10156000721C88E89EE00F94CA1BD1011496ED917D
:10157000FC9180E090E0A0E0B0EC86879787A08B9C
:10158000B18BD101ED91FC910484F585E02D62E0F1
:10159000C101199581E090E064960FB6F894DEBF22
:1015A0000FBECDBFDF91CF911F910F91FF90EF90B4
:1015B000DF90CF90BF90AF909F908F907F906F9073
:1015C0005F904F903F902F90089581859285A385DD
:1015D000B485F80182879387A487B587E7CEA501F4
:1015E000940169817A818B819C810F94414F1816F7
:1015F0000CF07DCF89819A81AB81BC81F801808319
:101600009183A283B38373CFA501940169817A8109
:101610008B819C810F94414F18160CF07ECF8981ED
:101620009A81AB81BC81EE81FF8186A397A3A0A79D
:10163000B1A773CF4F925F926F927F928F929F92DA
:10164000AF92BF92CF92DF92EF92FF920F931F93D0
:10165000CF93DF93CDB7DEB760970FB6F894DEBFB8
:101660000FBECDBF6130710509F4DBC1DC011496FA
:10167000ED91FC913097C9F481E090E060960FB64F
:10168000F894DEBF0FBECDBFDF91CF911F910F91B8
:10169000FF90EF90DF90CF90BF90AF909F908F9092
:1016A0007F906F905F904F90089520813181232B20
:1016B00019F33C01DC01ED91FC910284F385E02DEE
:1016C00019950297C9F6F301E280F380E114F10461
:1016D00099F2C7010E948EE2823071F240E051E03F
:1016E00060E070E0C7010E9414E1672B682B692B52
:1016F00019F6D3011496ED91FC9180819181FC0142
:1017000022AD222309F455C10F94371E882309F412
:1017100050C1D3011496ED91FC9186898823A1F0E4
:10172000C3010E946D626B017C0120E030E0A901E1
:101730000F94414F87FD08C0D3011496ED91FC91A1
:10174000C282D382E482F5826DE875E289E39FE08C
:101750000F94C91CD3011296ED91FC910280F38184
:10176000E02D6081718189E39FE00F94721C67E82E
:1017700075E289E39FE00F94C91CD3011496ED91A3
:10178000FC91428553856485758589E39FE00E94BD
:10179000A2B062E875E289E39FE00F94C91CD3010F
:1017A0001496ED91FC91468157816085718589E39E
:1017B0009FE00E94A2B067E677E089E39FE00F9484
:1017C000721CD3011496ED91FC9142815381648186
:1017D000758189E39FE00E94A2B06EE775E289E31C
:1017E0009FE00F94C91CD3011496ED91FC910190D8
:1017F000F081E02D408151816281738189E39FE016
:101800000E94A2B06AE775E289E39FE00F94C91CC9
:10181000D3011496ED91FC910190F081E02D44816B
:1018200055816681778189E39FE00E94A2B066E7D7
:1018300075E289E39FE00F94C91CD3011496ED91E2
:10184000FC910190F081E02D408551856285738582
:1018500089E39FE00E94A2B0D3011496ED91FC9120
:101860008689882331F06FE675E289E39FE00F9463
:10187000C91C89E39FE00F94CA1BF301E480F58043
:10188000D70156968C918111F7CE0281138161E0C8
:10189000F801848195810E943EAC2C0120E030E06B
:1018A000A901D7011E966D917D918D919C915197C3
:1018B0000F94394C81110CC020E030E0A901F701F0
:1018C00062817381848195810F94414F18165CF079
:1018D00040E050E061E070E0C8010E9414E1672B35
:1018E000682B692B31F119861A861B861C861D868A
:1018F0001E861F86188A8A85807F8A8761E0CE01CE
:1019000009960E946B2129833A834B835C836D8304
:101910007E838F839887912C812CB12CA12CD12C84
:10192000C12C79018A019B01AC016FEFC2010E94B9
:10193000A08040E050E061E070E0D30112968D910C
:101940009C910E94C2E0D3011496ED91FC913281EA
:1019500063815481458119861A861B861C868A8577
:10196000807F8760F82E8A87232F832F962FA52FBD
:10197000B42F8D879E87AF87B88B912C812CB12C8B
:10198000A12CD12CC12CE9840B851C853E854F856B
:1019900058896FEFC2010E94A080D3011496ED9187
:1019A000FC9182819381A481B58186879787A08BE2
:1019B000B18BD3011496ED91FC91868981115CCE97
:1019C0008789908D009709F457CE28EE33E0829FE7
:1019D0002001839F500C929F500C11240E94ACBE9A
:1019E000D3011496ED91FC914114510499F06201D8
:1019F000F12CE12C0289138924893589AB01BC01C2
:101A0000401B510B620B730B4C155D056E057F057A
:101A100008F432CE81E0868B61E0C3010E94A68388
:101A20002BCE90E080E02ACE2F923F924F925F9291
:101A30006F927F928F929F92AF92BF92CF92DF92DE
:101A4000EF92FF920F931F93CF93DF93CDB7DEB743
:101A5000C458D1090FB6F894DEBF0FBECDBFFC014C
:101A6000902FA2960FAFA297A3961FAFA397A4960D
:101A70002FAFA497A5963FAFA597A6964FAFA69771
:101A8000A7965FAFA797A8966FAFA897A9967FAFC5
:101A9000A99786EF800F823008F492C6EB96FFAECE
:101AA000EEAEEB97AD96FFAFEEAFAD97822F422E25
:101AB000512C002309F492C64114510409F483C641
:101AC000EB96AEADBFADEB97AB2B09F48EC687306E
:101AD00051F5913109F427C2923109F444C2903191
:101AE000F9F46FEF70E0CE018F599F4F0E944522AD
:101AF0006A962FAF6A976B963FAF6B976C964FAF16
:101B00006C976D965FAF6D976E966FAF6E976F9691
:101B10007FAF6F97A0968FAFA097A1969FAFA19729
:101B200067E0462E512CAD96AEADBFADAD97149685
:101B3000ED91FC91309709F472C466807780CF579D
:101B4000DF4F19821882C158D040E9961FAE1EAEF1
:101B5000E997E3961FAE1EAEE397312C212CE79652
:101B60001FAE1EAEE7976114710409F466C469E7FD
:101B700075E0C3010E94C6ABE1969FAF8EAFE197BF
:101B800066E577E0C3010E94C6ABAB969FAF8EAF10
:101B9000AB976BE777E0C3010E94C6ABCD57DF4F31
:101BA00099838883C358D04060E776E0C3010E94E0
:101BB000C6ABED969FAF8EAFED97E196EEADFFAD64
:101BC000E197309709F4C0C0AB962EAD3FADAB970F
:101BD0002115310509F4B8C080858F70823009F075
:101BE000B3C0D90118968C918F70823009F0ACC0C7
:101BF0002CE330E040E050E06BE976E0C3010E9466
:101C0000726AC358DF4F688379838A839B83CD5779
